:100000000C94FD060C942E070C942E070C942E07CE
:100010000C942E070C942E070C942E070C942E078C
:100020000C942E070C942E070C942E070C942E077C
:100030000C942E070C94C4780C942E070C942E0765
:100040000C942E070C949E710C942E070C942E0782
:100050000C942E070C942E070C942E070C94C66F4C
:100060000C942E070C9454680C942A680C942E0758
:100070000C942E070C942E070C942E070C942E072C
:100080000C9470710C942E070C942E070C942E0770
:100090000C9400680C94D6670C942E070C94E779A6
:1000A0000C942E070C942E070C9442710C942E077E
:1000B0000C942E070C942E070C942E070C9414719C
:1000C0000C942E070C942E070C942E070C94AC67FE
:1000D0000C9482670C942E070C9458670C942E672E
:1000E0000C942E070C9434070C943E070C94E9757D
:1000F0000C940D8E0C942E5A0C948D5B0C9440072E
:100100000C9453070C94658F0C94975B0C943007F8
:100110000C94228E0C945B8D0C94755B0C9412766F
:100120000C94918C0C948AA50C94F35A0C942F8CFB
:100130000C94608A0C94685B0C94A0810C945C5BBA
:100140000C94E3760C94715B0C947C070C94708B8C
:100150000C94B0890C94B28D0C94645B0C94D859B7
:100160000C94AD850C943F760C9460660C94518A87
:100170000C94E6750C94F42D0C949B5B0C94605BD2
:100180000C94988A0C941F5A0C9463910C941377D6
:100190000C94108A0C944F070C94A70D0C94E775DF
:1001A0000C941E770C94BE850C9479070C94838F65
:1001B0000C94A88C0C94425A0C94505A0C94C45B26
:1001C0000C94E8750C94D48D0C94965B0C945D2A79
:1001D0000C947F5B0C94BD8F0C9463070C94AA81E4
:1001E0000C94F9760C94835B0C9409820C945877E8
:1001F0000C94DE830C94B1830C94158C0C94F875DC
:100200000C9493760C94FD760C94895B0C94A65A0E
:100210000C9467720C9473760C948E910C94F9265E
:100220000C94915B0C9433910C94508C0C946B5BFC
:100230000C946A070C9443070C940B760C947B5B2C
:100240000C94EE8F0C9482920C947CB00C94565BC0
:100250000C94B98B0C94D9590C948F8B0C94EA1292
:100260000C944B070C94B9914E414E494E49545948
:10027000494E46CDCCCC3D0AD7233C17B7D1387771
:10028000CC2B329595E6241FB14F0A000020410087
:1002900000C84200401C4620BCBE4CCA1B0E5AAED1
:1002A000C59D7400407A10F35A00A0724E180900E0
:1002B00010A5D4E80000E87648170000E40B5402CB
:1002C0000000CA9A3B000000E1F505000080969806
:1002D00000000040420F000000A086010000001056
:1002E0002700000000E80300000000640000000098
:1002F000000A00000000000100000000002C76D879
:1003000088DC674F0823DFC1DFAE59E1B1B796E55E
:10031000E3E453C63AE651997696E8E6C28426EBC2
:10032000898C9B62ED407C6FFCEFBC9C9F40F2BAD5
:10033000A56FA5F490055A2AF75C936B6CF9676D6D
:10034000C11BFCE0E40D47FEF520E6B500D0ED90C2
:100350002E0300943577050080841E080000204E8F
:100360000A000000C80C333333330F986E12831128
:1003700041EF8D2114893BE65516CFFEE6DB18D1FF
:10038000844B381BF77C1D901DA4BBE424203284D1
:10039000725E228100C9F124ECA1E53D2748545446
:1003A000502F312E3020343030204261642052658D
:1003B00071756573740D0A5365727665723A2057CC
:1003C00065626475696E6F2F312E370D0A436F6E4B
:1003D00074656E742D547970653A20746578742F45
:1003E00068746D6C0D0A0D0A3C68313E45504943F6
:1003F000204641494C3C2F68313E00485454502F10
:10040000312E3020323030204F4B0D0A536572763A
:1004100065723A205765626475696E6F2F312E37A9
:100420000D0A4163636573732D436F6E74726F6C55
:100430002D416C6C6F772D4F726967696E3A202A77
:100440000D0A436F6E74656E742D547970653A2091
:1004500000436F6E6E656374696F6E3A20636C6FF4
:1004600073650D0A436F6E74656E742D54797065F3
:100470003A206170706C69636174696F6E2F782DBA
:100480007777772D666F726D2D75726C656E636F01
:1004900064656400506F7374206661696C65640004
:1004A00055706C6F6164204661696C65643A200028
:1004B000234E6F2073656E736F7220666F722074A7
:1004C000656D7020262068756D69646974792100F6
:1004D0004E6F2053656E736F72210020666F72201D
:1004E00074656D7020262068756D69646974792162
:1004F000002353656E736F72204572726F72200015
:1005000053656E736F72204572726F7221002357AC
:10051000726F6E672073656E736F7220666F7220E4
:1005200074656D7020262068756D69646974792121
:100530000057726F6E672053656E736F72210043B0
:1005400020483D00543D0020202020202020202055
:1005500020202020202020002020202020202020BB
:1005600020202020202020002020202020202020AB
:1005700020202020202020004950206164647265E2
:1005800073733A2000416E676C654000496E766176
:100590006C696420534D20737465707320706572AC
:1005A00020616E676C653D00534D207374657073F8
:1005B0002070657220616E676C653D003C68343E5A
:1005C000436F707972696768742843293230313813
:1005D0002D3230323020456455484B20486173201D
:1005E00043656E7472652E3C2F68343E3C2F626FFB
:1005F00064793E3C2F68746D6C3E003C703E4C61EB
:100600006D7020616E64204F746865722053746150
:10061000747573EFBC9A3C2F703E003C68313E43CA
:10062000616E6E6F74206765742073656E736F7290
:100630002072656164696E6773213C2F68313E00EA
:100640003C21646F63747970652068746D6C3E3C06
:1006500068746D6C3E3C686561643E3C6D657461B8
:1006600020636861727365743D227574662D38224B
:100670003E3C7469746C653E4F6E6C696E652065B6
:1006800078706572696D656E74206F6E20706F6C26
:100690006172697A6174696F6E206F66206C696738
:1006A00068743C2F7469746C653E3C2F68656164A6
:1006B0003E3C626F64793E3C68313E4F6E6C696EC1
:1006C00065206578706572696D656E74206F6E2047
:1006D000706F6C6172697A6174696F6E206F6620E9
:1006E0006C696768743C2F68313E00506172616DBF
:1006F000657465727320726573657420646F6E65CE
:100700002100736573757365722F736D6C6967680B
:1007100074706F2F73312F00616E676C6520646990
:1007200072656374696F6E3A200043757272656E0C
:100730007420534D206973202300534D3A54616255
:100740006C652073746570732070657220616E67CC
:100750006C653D00534D3A506F6C61726F69642057
:1007600073746570732070657220616E676C653D8F
:1007700000234448543D00236E65743D424C4500BF
:10078000236E65743D5769466900236E65743D426A
:1007900054002366747020757365726E616D653ADE
:1007A000003A0023486F7374207365727665722077
:1007B000495020616E6420506F72743A0023526574
:1007C0006C617920646576696365733A00235265CC
:1007D0006C617920737461747573206C6162656CEF
:1007E000733A20002352656C6179207374617465DB
:1007F000733A002352656C61792070696E733A0018
:10080000234E6F2E206F662072656C6179733D00F8
:1008100046696E64696E67205769466920495000D1
:100820004E45543D426C7565746F6F7468204C453D
:10083000004E45543D426C7565746F6F7468004E90
:1008400045543D5769466900696E7075742044537C
:100850005463616C6962726174653A005344206F3D
:1008600070656E206661696C004E65772064617406
:100870006120636F6C6C656374696F6E2073746163
:10088000727465640043757272656E74207365746A
:1008900074696E67733A0053797374656D2072657D
:1008A000736574206174200023445320546865727A
:1008B0006D6F6D657465722063616C6962726174DD
:1008C000656420666F72202300496E76616C6964EE
:1008D00020616E676C6520666F72200020737465FE
:1008E00070732070657220616E676C653D002073C7
:1008F000746570732070657220616E676C653D0071
:100900005461626C65205365742030002354757205
:100910006E7461626C6520536574203000506F6C9A
:100920006172697A65722053657420300023506FBC
:100930006C6172697A657220536574203000576962
:1009400046692049503A004C6F67676572204E61D6
:100950006D653A20005265626F6F74696E672E2E66
:100960002E0053657276657220506F727420757018
:1009700064617465640053504F52543D00495020E7
:1009800075706461746564005349503D0074696D0D
:100990006520696E74657276616C3D00005EBCE234
:1009A000613FDD83C29C7E20A3FD1F41009D23BECD
:1009B00046DB65F88C11AF32CA57E974000020009D
:1009C0002300260029002C002F0032000001000027
:1009D00003010601090100000A0B02090C0D0E08B3
:1009E00007030401000000000000000000000000F8
:1009F00000000000000000000000000000000000F7
:100A000000001211100000000000000000000000B3
:100A10000000000000000000000000002346616E9E
:100A200073207377697463686564206F6E20666FE6
:100A3000722000234865617465722073776974635E
:100A4000686564206F6E20666F72200000000100F0
:100A500001001010020001000100B00000001600AB
:100A6000000028000000100000002000000001002D
:100A70000100000000000000000000000000000075
:100A80000000000000000000000000000000FF0067
:100A90000000FFFF0000FFFF0000FFFF0000CFBFCE
:100AA0000000C7BF0000C3BF0000C1BF0000C0BF3F
:100AB000000000000000C0BF0000C1BF0000C3BFB5
:100AC0000000C7BF0000CFBF0000FFFF0000FFFF16
:100AD0000000000000000000000000000000000016
:100AE0000000000000000000000000000000000006
:100AF00000000000000000000000000000000000F6
:100B000000000000000000000000000000000000E5
:100B10000000557365722D6167656E743A202A0D69
:100B20000A446973616C6C6F773A202F0D0A004E8E
:100B30006574776F726B206D61696E7461696E6543
:100B400064206174200000002200250028002B0092
:100B50002E003100340002010000050108010B01E4
:100B600000002100240027002A002D00300033005F
:100B700001010000040107010A0101021020200800
:100B800008102040102040800201020108040201E8
:100B90000102040810204080804020100804020157
:100BA00080040201804020100804020108040201B0
:100BB0000102040810204080010204081020408037
:100BC00005050505070508080808020202020A0AC9
:100BD00008080404040401010101010101010303E7
:100BE000030303030303040707070C0C0C0C0C0C92
:100BF0000C0C0202020206060606060606060B0B8F
:100C00000B0B0B0B0B0B417070656E64206D6561F7
:100C1000732E200053696E676C65206D6561732EBD
:100C2000200053617665206D65617375726520746F
:100C30006F3A00202020202020202020202020206B
:100C400020202000202020202020202020202020C4
:100C500020202020002377656273657276657220FC
:100C6000626567696E73005461626C6520536574D8
:100C7000203000235475726E7461626C6520536578
:100C800074203000506F6C6172697A657220536510
:100C90007420300023506F6C6172697A6572205342
:100CA000657420300053797374656D2072657374B8
:100CB000617274656421002053797374656D2072CC
:100CC0006573746172746564210023436F6D6D6197
:100CD0006E64400054657374204C616D70732F46D0
:100CE000616E7300444843502053756363657373AA
:100CF0000044484350204641494C454400776562D2
:100D0000736572766572202E2E2E006572726F7278
:100D1000206F70656E696E672066696C653A2000A9
:100D20004C616D70204F74686572002354696D6565
:100D30002020202020204461746520202020205382
:100D400065636F6E647320506F6C61726F696420AD
:100D50005461626C652054286F4329204828252956
:100D6000202000646F6E652100696E69742E206416
:100D70006F6E652E00534420696E69742E20666183
:100D8000696C65642100696E69742E206661696C06
:100D90006564210057656C636F6D6520746F204535
:100DA0006455484B00496E697469616C697A696E73
:100DB0006720534420636172642E2E2E0075706C80
:100DC0006F616420627920465450206661696C65C9
:100DD00064210075706C6F61642062792046545004
:100DE000204F4B21007C3C3E5E2B3D3F2F5B5D3B0B
:100DF0002C2A225C00008AA57CB011241FBECFEFF4
:100E0000D1E2DEBFCDBF00E00CBF1AE0A0E0B2E04F
:100E1000ECEEFFE701E00BBF02C007900D92A8398E
:100E2000B107D9F728E1A8E9BAE001C01D92A83CB2
:100E3000B207E1F716E0CCEFD6E000E006C021975C
:100E40000109802FFE010E9457BACB3FD10780E0F5
:100E50000807A9F70E94BBA90C94E4BF0C940000FA
:100E6000FC01768765870895DC01ED91FC91068C85
:100E7000F78DE02D199591E089270895862F089523
:100E800081E08627089521E0FC018485883008F000
:100E900020E0822F0895FC01848595850895FC014A
:100EA00084899589089520E234E0FC013183208310
:100EB000FB014089518962897389FC014283538314
:100EC000648375830895DC01ED91FC91048CF58DAC
:100ED000E02D199490E080E00895CF93DF93EC012A
:100EE000FB01248135810E94A865CE01DF91CF915D
:100EF00008950A960C94108A0A960C941E77EF9225
:100F0000FF920F931F93CF93DF938C01E091DB123D
:100F10008E2F90E0FC01EE0FFF1FE80FF91FE85B3A
:100F2000FD4E808186FD06C069E370E08BED92E1A5
:100F30000E948C7064E670E080E090E00E94C069DE
:100F4000809145029091460297FF04C0109246029C
:100F500010924502C0914502D0914602BE018BED30
:100F600092E10E94107064E670E080E090E00E94E0
:100F7000C069809145029091460208171907C4F094
:100F80007E01C53BD1051CF054EBE52EF12CC017BA
:100F9000D10714F5B7018BED92E10E9410706EE15C
:100FA00070E080E090E00E94C069E7012196E8CF00
:100FB0000C171D078CF4D7FF02C0D0E0C0E0BE01C3
:100FC0008BED92E10E9410706EE170E080E090E0A5
:100FD0000E94C0692197ECCFCE01C53BD10514F02A
:100FE00084EB90E0E091DB122E2F30E0F901EE0F60
:100FF000FF1FE20FF31FE85BFD4E20812F7B208354
:1010000097FF02C090E080E0DF91CF911F910F9198
:10101000FF90EF900895EF92FF920F931F93CF935D
:10102000DF938C01E091D8128E2F90E0FC01EE0F3F
:10103000FF1FE80FF91FE85BFD4E808186FD06C0AB
:1010400069E370E088ED92E10E948C7064E670E0E4
:1010500080E090E00E94C069809143029091440238
:1010600097FF04C01092440210924302C0914302C1
:10107000D0914402BE0188ED92E10E94107064E6B6
:1010800070E080E090E00E94C069809143029091FE
:10109000440208171907C4F07E01C53BD1051CF0B6
:1010A00054EBE52EF12CC017D10714F5B70188EDEC
:1010B00092E10E9410706DE270E080E090E00E948A
:1010C000C069E7012A96E8CF0C171D078CF4D7FFFB
:1010D00002C0D0E0C0E0BE0188ED92E10E94107035
:1010E0006DE270E080E090E00E94C0692A97ECCF4A
:1010F000CE01C53BD10514F084EB90E0E091D8120D
:101100002E2F30E0F901EE0FFF1FE20FF31FE85B17
:10111000FD4E20812F7B208397FF02C090E080E06E
:10112000DF91CF911F910F91FF90EF9008954F9213
:101130005F926F927F928F929F92AF92BF92CF9267
:10114000DF92EF92FF920F931F93CF93DF93EC0107
:101150008090590290905A02E4E9F2E081E090E038
:10116000512C412C8816990654F02191319121304F
:10117000310519F42FEF421A520A0196F3CF1C16CB
:101180001D060CF04AC08C169D060CF446C04E019C
:101190008E01000F111F7E01EE0CFF1CEE0CFF1CD8
:1011A0008C169D060CF4D9C0C701895C9D4F6C015B
:1011B000FC0180819181A281B381970122563D4F2C
:1011C0005901181619061A061B0654F50E94A37237
:1011D000F5012081318142815381621B730B840BA5
:1011E000950BF60120813181428153812617370703
:1011F0004807590758F410821182128213820E9404
:10120000A372F501608371838283938321960E5FBD
:101210001F4FF4E0EF0EF11CC3CFC1E0D0E0B8CF18
:1012200098012D5A3D4F3901F90180819181980132
:101230002E563D4F6901F9012081318182179307B4
:10124000F1F0F3E04F16510414F00097C1F4880F49
:10125000991FFC01E15DF34F6081F801EC5CF34FF5
:1012600080810E94A768F30180819181F6019183BA
:1012700080836CE271E080E090E00E94C069F5013B
:1012800080819181A281B381181619061A061B0666
:101290000CF0BCCF0E94A372F50120813181428104
:1012A0005381621B730B840B950BF701E95BFD4FB8
:1012B000208131814281538126173707480759071A
:1012C00008F0A4CFF50110821182128213829801D6
:1012D00028563D4F5901F90180819181F601208105
:1012E00031818217930709F491CF6091590270916F
:1012F0005A02E4E9F2E041E050E030E020E0641717
:1013000075074CF0A191B191119711F42F5F3F4FE8
:101310004F5F5F4FF4CF233031051CF0009709F089
:1013200075CF880F991FFC01E15DF34F6081F801D3
:10133000EC5CF34F80810E94A768F5018081918168
:10134000F60191838083F301918380836CE271E0E5
:1013500080E090E00E94C06959CFDF91CF911F914A
:101360000F91FF90EF90DF90CF90BF90AF909F9044
:101370008F907F906F905F904F900895CF93DF9301
:10138000FC0124813581232B69F0EC01BC0180E54F
:1013900091E10E94EA66BE0189E79FE0DF91CF916B
:1013A0000C94EA66DF91CF910895CF93DF93FC010F
:1013B00024813581232B69F0EC01BC0180E591E1AA
:1013C0000E94DC66BE0189E79FE0DF91CF910C941B
:1013D000DC66DF91CF91089581E080939002809147
:1013E0009102882341F088E080935D1660E082E5F9
:1013F00096E10C94CC710895809191028823F9F0C4
:10140000809190028823D9F081E00E94F8718BE3EB
:101410009FE10197F1F760E080E00E94097268E6C1
:1014200075E082E596E10E94FE6661E080E00E9440
:10143000097268E575E082E596E10C94FE66089510
:101440008F929F92AF92BF92CF92DF92EF92FF92D4
:101450000F931F93CF93DF938C01862F0B301105D1
:1014600009F092C09091DB15992309F0F89462E19C
:101470000E94F369EC018091DB15882309F07894D0
:10148000209701F180E090ECA9E7B4EC8093CE15B1
:101490009093CF15A093D015B093D1158093D2150A
:1014A0009093D315A093D415B093D515CE3F8FEF5D
:1014B000D80709F49DC0CF3FDC0709F4F5C1CCEF94
:1014C000DFEF24C1C091D615E090D7156E2D70E0E6
:1014D00090E080E00E9472B72DEC3CEC4CEC5DE3B8
:1014E0000E94D1B74B015C016C2F70E090E080E06E
:1014F0000E9472B79B01AC01C501B4010E9419B9E9
:101500006093CE157093CF158093D0159093D1151D
:10151000D091D815F090D9156D2F6F7770E090E0CD
:1015200080E00E9472B74B015C016F2D70E090E08B
:1015300080E00E9472B72DEC3CEC4CEC5DE30E9425
:10154000D1B79B01AC01C501B4010E9419B9D7FD07
:1015500019C06093D2157093D3158093D4159093CE
:10156000D515CE0DCD0FCF0D81E090E02091DA158D
:10157000C21302C090E080E0892B09F487C0CFEF4E
:10158000DFEF92C19058E5CFCFEFDFEF06311105C5
:1015900009F0BCC09091DB15992309F0F89461E043
:1015A0000E94F369EC018091DB15882309F078949F
:1015B000209709F180E090ECA9E7B4EC8093CE1578
:1015C0009093CF15A093D015B093D1158093D215D9
:1015D0009093D315A093D415B093D515CF3FDC07C6
:1015E00009F462C1209709F451C0229609F067CF2F
:1015F000CEEFDFEF8BC0C091D715D091D61560919B
:10160000D6157091D71576276727762790E080E06A
:101610000E9470B72DEC3CEC4CEC5DE30E94D1B71E
:101620006093CE157093CF158093D0159093D115FC
:10163000E090D915F090D8156F2D6F77762F6E2D1D
:1016400090E080E00E9470B72DEC3CEC4CEC5DE348
:101650000E94D1B7F7FC18C06093D2157093D315D0
:101660008093D4159093D5158C2F8D0F8E0D8F0DE3
:10167000C1E0D0E09091DA15891302C0D0E0C0E05B
:10168000D195C195D109AACF9058E6CFC090CE157B
:10169000D090CF15E090D015F090D11520E030E03B
:1016A00048EC52E4C701B6010E942DBAD0E0C0E078
:1016B000181614F4CBEFDFEF20E030E0A901C701EA
:1016C000B6010E946BB787FF02C0CAEFDFEFC09080
:1016D000D215D090D315E090D415F090D51520E018
:1016E00030E048EC52ECC701B6010E946BB787FFAF
:1016F00002C0C9EFDFEF20E030E040EF52E4C70165
:10170000B6010E942DBA18160CF4C9C00C30110590
:1017100009F0CAC081E08093540F8CE58093760F66
:101720001092550F1092770F90E080E00E94405D7C
:1017300081E00E94505C65E08CE50E94455E10925D
:10174000F50C8093F40CC82FD0E0209709F4AAC0C0
:10175000C530D1050CF4B8C008E51BE08DEE91E171
:101760000E94F875F80180870F5F1F4FC8018855E8
:101770009B408C179D0794F3C091600B0091610B07
:10178000602F70E090E080E00E9472B72DEC3CEC9E
:101790004CEC5DE30E94D1B76B017C016C2F70E0D3
:1017A00090E080E00E9472B79B01AC01C701B601D6
:1017B0000E9419B96B017C01C092580BD092590B51
:1017C000E0925A0BF0925B0BD091620B1091630B7D
:1017D0006D2F6F7770E090E080E00E9472B74B0150
:1017E0005C01612F70E090E080E00E9472B72DEC08
:1017F0003CEC4CEC5DE30E94D1B79B01AC01C50110
:10180000B4010E9419B9D7FD5DC060935C0B709361
:101810005D0B80935E0B90935F0BC00FCD0FC10FDC
:101820008091640BC813ABCE20E030E048EC52E46A
:10183000C701B6010E942DBAD0E0C0E0181614F41A
:10184000CBEFDFEF20E030E040EA50E4C701B60123
:101850000E946BB787FF02C0CAEFDFEFC0905C0B3E
:10186000D0905D0BE0905E0BF0905F0B20E030E0DD
:1018700040EF51ECC701B6010E946BB787FF02C071
:10188000C9EFDFEF20E030E040EF52E4C701B601DE
:101890000E942DBA181644F4C8EFDFEF05C0C8EF58
:1018A000DFEF34CFCEEFDFEFCE01DF91CF911F918D
:1018B0000F91FF90EF90DF90CF90BF90AF909F90EF
:1018C0008F9008959058A1CFCDEFDFEFEDCFCF935C
:1018D000DF93FB0122813381DC0113963C932E932D
:1018E0001297448155816681778114964D935D935B
:1018F0006D937C9317974085518562857385189603
:101900004D935D936D937C931B971C96EF012C96E2
:101910009C01275E3F4F49914D93A217B307D9F71A
:10192000218D328DFC01328F218FDF91CF9108956F
:10193000DF92EF92FF920F931F93CF93DF93D82EF6
:1019400004E31CE0E801EE24E394F12C229680915C
:10195000590290915A028E159F059CF061E0888192
:101960000E948F6960912F0C88810E94A76864EFA4
:1019700071E080E090E00E94C0698FEFE81AF80AF9
:10198000E5CFDD2009F45EC0C4E3DCE0EE24E3949F
:10199000F12C22968091590290915A02E816F9068C
:1019A0002CF56091310C88810E94A76868EE73E085
:1019B00080E090E00E94C069AFEFEA1AFA0A6091F5
:1019C000310C8A810E94A76868EE73E080E090E0A5
:1019D0000E94C06960912F0C88810E94A76868EE00
:1019E00073E080E090E00E94C069D3CF68EE73E0BE
:1019F00080E090E00E94C06992E9E92E92E0F92E21
:101A0000C1E0D0E0B2E0EB0EF11C0E5F1F4F809101
:101A1000590290915A028C179D07A4F0D701ED91BD
:101A2000FC91EE0FFF1FE15DF34F6081F8018081B3
:101A30000E94A76868EC70E080E090E00E94C069B6
:101A40002196E0CFDF91CF911F910F91FF90EF9002
:101A5000DF900895CF92DF92EF92FF920F931F9342
:101A6000CF93DF93CDB7DEB7A0970FB6F894DEBF64
:101A70000FBECDBF7C018B0150E040E06C018AE0DD
:101A8000C80ED11CCA010196F8012491E1E0F0E0F2
:101A9000EC0FFD1FE40FF51F2083222389F0803215
:101AA000910551F440E250E0BE016F5F7F4FC601E7
:101AB0000E94108A90E080E00F5F1F4FAC01E2CFE0
:101AC000029738F0BE016F5F7F4FC7010A960E94F0
:101AD000108AA0960FB6F894DEBF0FBECDBFDF917F
:101AE000CF911F910F91FF90EF90DF90CF900895CD
:101AF000EF92FF920F931F93CF93DF93EC018B0133
:101B00007A016BEF73E00E942A0DB801CE010E94AA
:101B1000D4668E01065F1F4F42E050E06AE979E02B
:101B2000C8010E94108AE114F10421F0B701CE012E
:101B30000E94D46642E050E06AE979E0C801DF9192
:101B4000CF911F910F91FF90EF900C94108A6DE947
:101B500073E00C942A0DEF92FF920F931F93CF9393
:101B6000DF9300D000D0CDB7DEB78C017B0166E2F9
:101B700079E00E9493658AE0E816F1042CF464EDA4
:101B800077E0C8010E947464B701CE0101960E94FB
:101B9000D862BE016F5F7F4FC8010E947E64CE0194
:101BA00001960E94FA64C80126960FB6F894DEBF2B
:101BB0000FBECDBFDF91CF911F910F91FF90EF909E
:101BC00008950F931F93CF93DF9300D000D0CDB72C
:101BD000DEB72091330C2223A9F08C016CEC78E065
:101BE000CE0101960E949365B801CE0101960E9434
:101BF0001564BC0180E591E10E94EA66CE01019680
:101C00000E94FA6426960FB6F894DEBF0FBECDBFD1
:101C1000DF91CF911F910F9108950F931F93CF9351
:101C2000DF93CDB7DEB72C970FB6F894DEBF0FBEAB
:101C3000CDBF8C010E940B73BC01C8010E94AB0D8B
:101C40000E940373BC01CE0107960E94AB0D62E0B7
:101C500078E0CE0101960E949365BE01695F7F4FD7
:101C6000CE0101960E941564BC01C8010E947E64E9
:101C7000CE0101960E94FA64CE0107960E94FA6492
:101C80006EE177E0C8010E9474640E94FB72BC019F
:101C9000CE0101960E94AB0DBE016F5F7F4FC80160
:101CA0000E947E64CE0101960E94FA6462E574E0AF
:101CB000C8010E9474640E94F372BC01CE010196B7
:101CC0000E94AB0DBE016F5F7F4FC8010E947E6412
:101CD000CE0101960E94FA6462E574E0C8010E9498
:101CE00074640E94E972BC01CE0101960E94AB0DA2
:101CF000BE016F5F7F4FC8010E947E64CE010196D6
:101D00000E94FA64C8012C960FB6F894DEBF0FBE8D
:101D1000CDBFDF91CF911F910F9108950F931F9326
:101D2000CF93DF93CDB7DEB72C970FB6F894DEBF15
:101D30000FBECDBF8C010E940B73BC01C8010E9475
:101D4000AB0D0E940373BC01CE0107960E94AB0D40
:101D500062E078E0CE0101960E949365BE01695F62
:101D60007F4FCE0101960E941564BC01C8010E94FC
:101D70007E64CE0101960E94FA64CE0107960E940D
:101D8000FA640E94A3720E94CB7760917E0C70E08F
:101D9000CE0107960E94AB0D62E078E0CE0101967D
:101DA0000E949365BE01695F7F4FCE0101960E943C
:101DB0001564BC01C8010E947E64CE0101960E9498
:101DC000FA64CE0107960E94FA646EE177E0C801DA
:101DD0000E9474640E94FB72BC01CE0101960E94B5
:101DE000AB0DBE016F5F7F4FC8010E947E64CE01C4
:101DF00001960E94FA6462E574E0C8010E9474646E
:101E00000E94F372BC01CE0101960E94AB0DBE018F
:101E10006F5F7F4FC8010E947E64CE0101960E94D1
:101E2000FA6462E574E0C8010E9474640E94E97279
:101E3000BC01CE0101960E94AB0DBE016F5F7F4FCA
:101E4000C8010E947E64CE0101960E94FA64C80116
:101E50002C960FB6F894DEBF0FBECDBFDF91CF91A9
:101E60001F910F910895CF92DF92EF92FF920F93FF
:101E70001F93CF93DF9300D000D0CDB7DEB77C01A6
:101E8000FB01848195818A01081B190B101611062C
:101E90009CF0C7010E947865C70126960FB6F8949A
:101EA000DEBF0FBECDBFDF91CF911F910F91FF908D
:101EB000EF90DF90CF900895CE0101960E948A6541
:101EC000CC24C394D12C6EE177E0CE0101960E9420
:101ED0007464FFEFCF1ADF0A0C151D05A4F7BE01CD
:101EE0006F5F7F4FC7010E947865CE0101960E9407
:101EF000FA64D2CFDF92EF92FF920F931F93CF93AA
:101F0000DF93CDB7DEB762970FB6F894DEBF0FBE92
:101F1000CDBF8C011092650B66E279E0CE010D9683
:101F20000E949365FF24F39480E591E10E94505A4A
:101F30002091650B181619067CF521112DC080E53E
:101F400091E10E942E5A8A3009F07EC089899A89CF
:101F5000892B09F481C0F092650B64E574E0CE0131
:101F600001960E949365BE01635F7F4FCE0101968B
:101F70000E941564BC01CE0107960E948A65CE01BD
:101F800007960E94E10DCE0107960E94FA64CE01E9
:101F900001960E94FA6460C0F12CE12CDD24D394F8
:101FA000222309F460C089899A89019709F045C004
:101FB00061EE74E0CE0107960E949365BE01695FF1
:101FC0007F4FCE010D960E94E463F12C811115C064
:101FD00064E674E0CE0101960E949365BE016F5FD6
:101FE0007F4FCE010D960E94E463FF24F39481118C
:101FF000F12CCE0101960E94FA64CE0107960E9450
:10200000FA64FF20A1F050E040E0BE01635F7F4F23
:10201000CE0101960E946D07BE016F5F7F4F8DE874
:1020200093E10E94C164CE0101960E94FA6464E1CA
:1020300070E080E090E00E94C069BE01635F7F4F66
:10204000C8010E94786596C08D3009F47FCF682F53
:10205000CE010D960E9452646AE070E080E090E04C
:102060000E94C06961CF89E79FE00E94505A18160C
:10207000190614F589E79FE00E942E5A8A30A9F0CC
:102080008D3099F09091650B91110FC0682FCE01A2
:102090000D960E9452648FEFE81AF80A65E070E02E
:1020A00080E090E00E94C069DECF89899A89892BFF
:1020B000A9F3D092650BF2CF64E170E080E090E08C
:1020C0000E94C069EF2809F43FC089899A89892B49
:1020D000D9F18091330C882389F16CEC78E0CE0142
:1020E00001960E949365BE016F5F7F4FCE010D96F2
:1020F0000E94E463F82ECE0101960E94FA64F1106A
:102100001DC06DE574E0CE0101960E949365CE017D
:1021100001960E94D509CE0101960E94FA64BE0183
:10212000635F7F4FCE0101960E948A65CE010196C2
:102130000E94BE09CE0101960E94FA6464E170E03B
:1021400080E090E00E94C06989899A892091650B9E
:1021500021112BCF009709F028CF64E670E080E0D2
:1021600090E00E94C0690E948F6C66E279E0C8012D
:102170000E949365CE010D960E94FA64C801629692
:102180000FB6F894DEBF0FBECDBFDF91CF911F9188
:102190000F91FF90EF90DF9008950F931F93CF93CF
:1021A000DF93CDB7DEB72C970FB6F894DEBF0FBE26
:1021B000CDBF2C893D8930935A0220935902FE01EC
:1021C0007496A4E3BCE090E080E0329628173907CB
:1021D00034F0408151814D935D930196F6CF8C8D03
:1021E0009D8D9093300C80932F0C8E8D9F8D9093AE
:1021F000320C8093310CAD968FADAD97BE01645912
:102200007F4F8F3209F0BAC1CE0107960E949365C5
:1022100066E674E0CE0101960E949365BE01695F97
:102220007F4FCE0101960E941564BC018AEF95E1B3
:102230000E94AA64CE0101960E94FA64CE0107961C
:102240000E94FA646AEF75E1CE0101960E948A65E8
:10225000CE0101960E94BE09CE0101960E94FA6449
:102260006CE774E0CE0101960E949365BE016F5F3A
:102270007F4F8AEF95E10E94C463182FCE0101962B
:102280000E94FA644091FE155091FF15112309F444
:102290007CC1BA01625071098AEF95E10E94B36373
:1022A000682FCE0101960E945F65BE016F5F7F4F70
:1022B0008CED95E10E94C164CE0101960E94FA6402
:1022C00064ED74E1CE0107960E9493656EE774E0B9
:1022D000CE0101960E949365BE01695F7F4FCE01DA
:1022E00001960E941564BC0184EF95E10E94AA64E6
:1022F000CE0101960E94FA64CE0107960E94FA640C
:1023000024968FAD24971F928F9323968FAD23979A
:102310001F928F9322968FAD22971F928F932196B3
:102320008FAD21971F928F9384E894E09F938F93B2
:102330008EE69CE09F938F930E940EBDCE52DF4F9E
:1023400088819981C25DD0409093C7028093C60274
:10235000BE016C527F4FCE0101960E949365BE0173
:102360006F5F7F4F8EEE95E10E94C164CE010196B2
:102370000E94FA64BE0161527F4FCE0101960E9415
:102380009365BE016F5F7F4F88EE95E10E94C16447
:10239000CE0101960E94FA644091EC155091ED1522
:1023A0004250510968EE75E1CE0101960E946D0719
:1023B000CE0101960E944B636C5960936802CE0176
:1023C00001960E94FA64CC5EDE4F688179818A8131
:1023D0009B81C451D1400E9472B70FB6F894DEBF02
:1023E0000FBECDBF9B01AC010E9432BA882389F099
:1023F0008CE390E0A0E0B0E0CC5EDE4F8883998370
:10240000AA83BB83C451D140CD5EDE4F1882C35135
:10241000D140CD5EDE4F8881C351D140882399F0F1
:10242000CC5EDE4F88819981AA81BB81C451D140A5
:1024300080935D0290935E02A0935F02B09360026E
:1024400081E08093010DC85EDE4F688179818A81C9
:102450009B81C851D1409B01AC010E9432BA8823B4
:1024600061F080E090E0A0E7B2E4C85EDE4F8883D0
:102470009983AA83BB83C851D140C45EDE4F688173
:102480007981CC51D140072E000C880B990B0E940A
:1024900072B79B01AC010E9432BA882341F082E0FE
:1024A00090E0C45EDE4F99838883CC51D140C45CF8
:1024B000DE4F08811981CC53D140B801012E000CA8
:1024C000880B990B0E9472B79B01AC010E9432BA33
:1024D000811103C01016110644F080E590E0C45C41
:1024E000DE4F99838883CC53D140C45CDE4F888112
:1024F0009981CC53D140909336028093350288E283
:10250000FE01E551FF4FA2E4BCE001900D928A95D7
:10251000E1F7CE5CDE4F88819981AA81BB81C253ED
:10252000D1408093200290932102A0932202B09385
:102530002302CA5CDE4F88819981AA81BB81C65380
:10254000D14080931C0290931D02A0931E02B09371
:102550001F02C65CDE4F88819981CA53D140909397
:10256000AB028093AA022C960FB6F894DEBF0FBE82
:10257000CDBFDF91CF911F910F910895CE010796A6
:102580000E9493656BE674E045CE415051096AEFB5
:1025900075E1CE0101960E946D07BE016F5F7F4F0E
:1025A0008CED95E10E94C164CE0101960E94FA640F
:1025B0006AEF75E1CE0101960E948A656CE774E0CE
:1025C000CE0101960E94FF63BC018AEF95E10E9453
:1025D000AA6472CE6115710519F00A960C94EE6525
:1025E00090E080E00895EF92FF920F931F93CF93B6
:1025F000DF93CDB7DEB7E8970FB6F894DEBF0FBE16
:10260000CDBF66E279E0CE0187960E94936566E2CF
:1026100079E0CE018D960E94936582E0E82EF12C40
:102620002496FFAEEEAE249786E0EDEEF2E0DE01FA
:10263000D39601900D928A95E1F786E0FE01F3961C
:10264000DE01AC5BBF4F01900D928A95E1F72C96AD
:102650001FAE1EAE2C9701E010E02E961FAF0EAFFE
:102660002E9788E0E3EFF2E0DE01599601900D929B
:102670008A95E1F788E0FE017996DE01A25BBF4F03
:1026800001900D928A95E1F788E1EBEFF2E0DE012F
:10269000119601900D928A95E1F788E1FE0131963D
:1026A000DE01AA5ABF4F01900D928A95E1F7809101
:1026B000130390911403A0911503B0911603E296B1
:1026C0008CAF9DAFAEAFBFAFE29760E974E0CE01D3
:1026D00087960E94CE6260E0CE0187960E94526487
:1026E0004BA55CA5BE016E587F4FCE0187960E9418
:1026F000BF5F62E077E0CE018D960E94856468ED51
:1027000074E08CED95E10E94CE6260E0CE018D9682
:102710000E94526449A95AA9BE0166567F4FCE0154
:102720008D960E94BF5F66E279E0CE0187960E9497
:10273000CE6266E279E0CE018D960E94CE62C250F2
:10274000DF4F19821882CE5FD0408091C6029091EF
:10275000C702C050DF4F99838883C050D14080E0CA
:1027600090E0A0E7B2E4CA5BDE4F88839983AA8336
:10277000BB83C654D140C65BDE4FF982E882CA549F
:10278000D14080E090E0A0E2B2E4C45BDE4F8883F9
:102790009983AA83BB83CC54D14080E090E0A4E32A
:1027A000B2E4C05BDE4F88839983AA83BB83C055A4
:1027B000D14084EB90E0CC5ADE4F99838883C45596
:1027C000D14088E790E0CA5ADE4F99838883C65586
:1027D000D1408CE291E0A0E0B0E0C85ADE4F88839F
:1027E0009983AA83BB83C855D140C45ADE4F19834D
:1027F0000883CC55D140C25ADE4FF982E882CE55CB
:10280000D14060E08EEE95E10E94526460E088EE77
:1028100095E10E9452644091F2155091F315BE016A
:102820006E5F7E4F8EEE95E10E94BF5F4091EC158A
:102830005091ED15BE01635F7E4F88EE95E10E94D9
:10284000BF5F88E2E2E4FCE0DE01A75EBE4F0190DC
:102850000D928A95E1F78CE390E0A0E0B0E0CE5BCA
:10286000DE4F88839983AA83BB83C254D140CF5B58
:10287000DE4F1882C154D14084EE98E3AEE8B2E452
:10288000C05ADE4F88839983AA83BB83C056D14048
:1028900084EE98E3AEE8B1E4CC59DE4F88839983A7
:1028A000AA83BB83C456D140C859DE4F198308831D
:1028B000C856D14080E590E0C659DE4F99838883A1
:1028C000CA56D14084EF91E09093DE028093DD02FE
:1028D000BE016E5B7F4F0E94519264EF71E080E019
:1028E00090E00E94C0696BEE76E0CE0181960E9476
:1028F0008165CE0181960E94BE09CE0181960E941B
:10290000FA64CE018D960E94FA64CE0187960E94E9
:10291000FA64E8960FB6F894DEBF0FBECDBFDF9124
:10292000CF911F910F91FF90EF9008959F92AF92DA
:10293000BF92CF92DF92EF92FF920F931F93CF93AC
:10294000DF93CDB7DEB7C859D1090FB6F894DEBF13
:102950000FBECDBF5C017B016A016CEF74E1CE015B
:1029600089579F4F0E9493656CE774E08E010F5F5B
:102970001F4FC8010E949365B801CE0189579F4F30
:102980000E94E463982EC8010E94FA64911014C05A
:102990006CE774E0C8010E949365BE0169577F4FE0
:1029A000C8010E941564BC01CE0189579F4F0E9447
:1029B000AA64C8010E94FA64B501CE0183579F4FF3
:1029C0000E94936568E974E021E0E216F10441F0A9
:1029D00063EA74E032E0E316F10411F06BEA74E0AC
:1029E000CE0189579F4F0E94746460E0CE018957E1
:1029F0009F4F0E945264B601C8010E948A656AE036
:102A0000C8010E946664BC01CE018D569F4F0E9492
:102A10008A65C8010E94FA64C557DF4F4881598111
:102A2000CB58D040B801CE0189579F4F0E94BF5F5D
:102A30008091020D882399F163EB74E0CE018F57EA
:102A40009F4F0E949365CE018F579F4F0E94D509DB
:102A5000CE018F579F4F0E94FA64BE0169577F4F86
:102A6000CE018F579F4F0E948A65CE018F579F4F8F
:102A70000E94D509CE018F579F4F0E94FA64B8017A
:102A8000CE018F579F4F0E949365CE018F579F4F66
:102A90000E94D509CE018F579F4F0E94FA64CC56F1
:102AA000DF4F8881C459D0408F93CD56DF4F888146
:102AB000C359D0408F93C257DF4F8881CE58D04042
:102AC0008F93C357DF4F8881CD58D0408F9383ECCD
:102AD00094E09F938F9388E9E82E8AE0F82EFF9286
:102AE000EF920E940EBD40913502509136026EE683
:102AF0007CE083E894E10E94228E0FB6F894DEBF5A
:102B00000FBECDBF019709F07CC01F930F9389ECD6
:102B100094E09F938F930AE91BE01F930F930E9409
:102B20000EBDB80183E894E10E94C0668EE69CE089
:102B30009F938F938AED94E09F938F931F930F93AE
:102B40000E940EBDB80183E894E10E94C06661E571
:102B500074E083E894E10E94FE666AE979E083E824
:102B600094E10E94EE65F70101900020E9F7CF01A2
:102B700089599A409F938F9383EE94E09F938F930C
:102B80001F930F930E940EBDB80183E894E10E9449
:102B9000C066B70183E894E10E94D46662E370E006
:102BA00080E090E00E94C06983E894E10E94D48DA7
:102BB0000FB6F894DEBF0FBECDBF11E0CE018D562B
:102BC0009F4F0E94FA64CE0183579F4F0E94FA6480
:102BD000CE0189579F4F0E94FA64812FC856DF4F5C
:102BE0000FB6F894DEBF0FBECDBFDF91CF911F911E
:102BF0000F91FF90EF90DF90CF90BF90AF909F909C
:102C0000089564E974E0CE018F579F4F0E9481655B
:102C1000CE018F579F4F0E94BE09CE018F579F4F05
:102C20000E94FA6460EA74E0CE018F579F4F0E94C1
:102C30008165CE018F579F4F0E94D509CE018F57D6
:102C40009F4F0E94FA6468E97AE0CE018F579F4F48
:102C50000E949365CE018F579F4F0E94BE09CE01FF
:102C60008F579F4F0E94FA6410E0A8CFCF92DF9257
:102C7000EF92FF920F931F93CF93DF93CDB7DEB701
:102C800068970FB6F894DEBF0FBECDBF66E279E05D
:102C9000CE0143960E94936560E078E0CE010196F4
:102CA0000E948165CE0101960E94D509CE01019650
:102CB0000E94FA646CA17DA1CE0101960E94D862A7
:102CC000CE0101960E94BE09CE0101960E94FA64CF
:102CD00063EF77E0CE0101960E948165CE010196F7
:102CE0000E94D509CE0101960E94FA647E0188E215
:102CF000E80EF11C01E010E08CA19DA18017910766
:102D00000CF1F701619171917F01CE0101960E9452
:102D1000D862CE0101960E94D509CE0101960E948B
:102D2000FA646EE177E0CE0101960E949365CE01D0
:102D300001960E94D509CE0101960E94FA640F5FA8
:102D40001F4FDACF6EE177E0CE0101960E949365C6
:102D5000CE0101960E94BE09CE0101960E94FA643E
:102D600064EE77E0CE0101960E948165CE01019666
:102D70000E94D509CE0101960E94FA6460912F0C41
:102D80007091300CCE0101960E94D862CE0101965E
:102D90000E94D509CE0101960E94FA646EE177E0A7
:102DA000CE0101960E949365CE0101960E94D5093D
:102DB000CE0101960E94FA646091310C7091320C40
:102DC000CE0101960E94D862CE0101960E94BE09F2
:102DD000CE0101960E94FA646DEC77E0CE01019677
:102DE0000E948165CE0101960E94D509CE0101960F
:102DF0000E94FA64BE01605D7F4FCE0101960E9481
:102E00009365CE0101960E94D509CE0101960E94DC
:102E1000FA646EE177E0CE0101960E949365CE01DF
:102E200001960E94D509CE0101960E94FA64BE0166
:102E30006C5C7F4FCE0101960E949365CE01019696
:102E40000E94BE09CE0101960E94FA646DEB77E004
:102E5000CE0101960E948165CE0101960E94BE09B5
:102E6000CE0101960E94FA648E010C5D1F4FEE2484
:102E7000E394F12C6801F8E0CF0ED11C8CA19DA148
:102E80008E159F050CF449C0B701CE0107960E942C
:102E9000D8626CEC78E0CE0101960E949365BE0189
:102EA000695F7F4FCE0101960E941564BC01CE017F
:102EB0000D960E948A65CE010D960E94D509CE011D
:102EC0000D960E94FA64CE0101960E94FA64CE012A
:102ED00007960E94FA6462E078E0CE0101960E94B3
:102EE0009365CE0101960E94D509CE0101960E94FC
:102EF000FA64B801645E7F4FCE0101960E9493652B
:102F0000CE0101960E94BE09CE0101960E94FA648C
:102F10008FEFE81AF80A8601ADCF63EA77E0CE01B9
:102F200001960E948165CE0101960E94D509CE01CD
:102F300001960E94FA646EE67CE0CE0101960E9442
:102F40009365CE0101960E94D509CE0101960E949B
:102F5000FA6461EA77E0CE0101960E948165CE01B4
:102F600001960E94D509CE0101960E94FA646091F3
:102F7000350270913602CE0101960E94D862CE01D0
:102F800001960E94BE09CE0101960E94FA6462E990
:102F900077E0CE0101960E948165CE0101960E94E4
:102FA000D509CE0101960E94FA64BE016C5A7F4F8A
:102FB000CE0101960E949365CE0101960E94BE0942
:102FC000CE0101960E94FA6468EF74E0CE0101968A
:102FD0000E949365CE0101960E94D509CE0101960B
:102FE0000E94FA64BE0164587F4FCE0101960E9490
:102FF0009365CE0101960E94BE09CE0101960E9402
:10300000FA64C052DF4F88819981C05ED040892B1D
:1030100071F46AE877E0CE0101960E948165CE01E5
:1030200001960E94BE09CE0101960E94FA64C05228
:10303000DF4F88819981C05ED040019771F460E8CC
:1030400077E0CE0101960E948165CE0101960E9433
:10305000BE09CE0101960E94FA64C052DF4F8881FA
:103060009981C05ED040029771F467E777E0CE01A6
:1030700001960E948165CE0101960E94BE09CE0193
:1030800001960E94FA6461E777E0CE0101960E9402
:103090008165CE0101960E94D509CE0101960E945C
:1030A000FA64CE51DF4F68817981C25ED040CE0193
:1030B00001960E94D862CE0101960E94BE09CE01FF
:1030C00001960E94FA644091930C5091940C609187
:1030D000950C7091960C21E0CE0107960E94026536
:1030E00063E075E0CE0101960E949365BE01695FC1
:1030F0007F4FCE0101960E9415646DE075E00E943D
:10310000FF63BC01CE010D960E948A65CE010D962B
:103110000E94BE09CE010D960E94FA64CE0101966E
:103120000E94FA64CE0107960E94FA6440918F0CC7
:103130005091900C6091910C7091920C21E0CE0115
:1031400007960E94026562E175E0CE0101960E9439
:103150009365BE01695F7F4FCE0101960E941564A1
:103160006DE075E00E94FF63BC01CE010D960E94E8
:103170008A65CE010D960E94BE09CE010D960E9471
:10318000FA64CE0101960E94FA64CE0107960E946D
:10319000FA6464E577E0CE0101960E948165CE0174
:1031A00001960E94D509CE0101960E94FA644091D1
:1031B000200250912102609122027091230225E0A9
:1031C000CE0101960E940265CE0101960E94BE09C1
:1031D000CE0101960E94FA646AE377E0CE0101967F
:1031E0000E948165CE0101960E94D509CE0101960B
:1031F0000E94FA6440911C0250911D0260911E02CF
:1032000070911F0225E0CE0101960E940265CE0159
:1032100001960E94BE09CE0101960E94FA646AE2FC
:1032200077E0CE0101960E948165CE0101960E9451
:10323000D509CE0101960E94FA6460915B027091FB
:103240005C02CE0101960E94D862CE0101960E94D6
:10325000BE09CE0101960E94FA6468E177E0CE01D2
:1032600001960E948165CE0101960E94D509CE018A
:1032700001960E94FA64C65BDE4F68817981CA5468
:10328000D140CE0101960E94D862CE0101960E94E3
:10329000BE09CE0101960E94FA64CE0143960E94B7
:1032A000FA6468960FB6F894DEBF0FBECDBFDF910B
:1032B000CF911F910F91FF90EF90DF90CF900895E5
:1032C000DF92EF92FF920F931F93CF93DF93CDB7CF
:1032D000DEB762970FB6F894DEBF0FBECDBF209168
:1032E0009102222379F120919002222359F17A014F
:1032F0008C016F3F7F4FA1F560E080E00E94097272
:10330000D12CB80182E596E10E94DC6667E475E0A5
:1033100082E596E10E94FE66F801848160E08D0DF1
:103320000E9409720E948F6C6093040F7093050FC6
:103330008093060F9093070FB701FF0C880B990B32
:103340000E94C06962960FB6F894DEBF0FBECDBF73
:10335000DF91CF911F910F91FF90EF90DF90089533
:1033600060E080E00E9409720E948F6C28EE33E0DA
:1033700040E050E00E94B5B8CA01B90120E831E54B
:1033800041E050E00E94D7B8AB01BC0120E0CE0183
:1033900001960E943265BE016F5F7F4FCE01079696
:1033A0000E948A656CEE75E0CE0107960E94FF636D
:1033B000BC01CE010D960E948A65CE0107960E943F
:1033C000FA64CE0101960E94FA64BE01635F7F4FEA
:1033D00082E596E10E94DC66D98860E08D2D0E942E
:1033E0000972CE010D960E94FA648BCFCF93DF93C2
:1033F00000D000D0CDB7DEB70E94FC09CE01019607
:103400000E940D0E4AE050E06FEF7FEFCE01019673
:103410000E946019CE0101960E94FA6461E080E08A
:103420000E940972CE0101960E94359262E576E112
:10343000CE0101960E94606669E175E082E596E141
:103440000E94D4660E948F6C6093970C7093980CC6
:103450008093990C90939A0C26960FB6F894DEBF41
:103460000FBECDBFDF91CF9108950F931F93CF93E0
:10347000DF9300D000D0CDB7DEB78C01CE0101962E
:103480000E940D0E4AE050E06FEF7FEFCE010196F3
:103490000E946019CE0101960E94FA64B801CE0123
:1034A00001960E948A656AE070E0CE0101960E9452
:1034B0003672CE0101960E94FA6426960FB6F894F1
:1034C000DEBF0FBECDBFDF91CF911F910F91089549
:1034D0002F923F924F925F926F927F928F929F9224
:1034E000AF92BF92CF92DF92EF92FF920F931F9312
:1034F000CF93DF93CDB7DEB7E8970FB6F894DEBF72
:103500000FBECDBF9CA78BA71B0170E060E00E949F
:10351000B363182F66E279E0CE0149960E94936565
:1035200080915B0290915C028130910509F091C01D
:1035300088E090E090931B0280931A0289E090E06B
:10354000909319028093180280912D0C90912E0C6B
:1035500090932C0C80932B0C809114029091150267
:10356000A0911602B091170280931002909311025D
:10357000A0931202B093130280912C0290912D021D
:10358000A0912E02B0912F028093300290933102CD
:10359000A0933202B093330280912A0C8093290CBD
:1035A0008091250C9091260CA091270CB091280CAD
:1035B0008093210C9093220CA093230CB093240CA5
:1035C0008AE390E090930F0280930E028091930C17
:1035D0009091940CA091950CB091960C80936A0CEC
:1035E00090936B0CA0936C0CB0936D0C80910C02BB
:1035F00090910D0290930B0280930A028091200219
:1036000090912102A0912202B09123028093240282
:1036100090932502A0932602B0932702133509F058
:1036200089C010922C0C10922B0C8091330C8823A3
:1036300071F06DE175E0CE0101960E949365CE01B7
:1036400001960E94BE09CE0101960E94FA64E12C07
:1036500048C1029719F78AE090E090931B0280938B
:103660001A028BE090E090931902809318028091E7
:103670001F0C9091200C90932C0C80932B0C80911C
:10368000060290910702A0910802B091090280936E
:10369000100290931102A0931202B0931302809132
:1036A000280290912902A0912A02B0912B028093C6
:1036B000300290933102A0933202B0933302809192
:1036C0001E0C8093290C80911A0C90911B0CA091D8
:1036D0001C0CB0911D0C8093210C9093220CA09394
:1036E000230CB093240C8BE390E090930F02809313
:1036F0000E0280918F0C9091900CA091910CB09142
:10370000920C80936A0C90936B0CA0936C0CB0930A
:103710006D0C809104029091050290930B028093AE
:103720000A0280911C0290911D02A0911E02B0918C
:103730001F026CCFC1010197029708F0E1C181E03F
:1037400090E0A0E0B0E08093100290931102A0936B
:103750001202B0931302ABA5BCA514968D919C9157
:103760001597029750F141E050E0BD01CE0101965E
:103770000E946D07BE016F5F7F4FCE0149960E9488
:10378000C164CE0101960E94FA64CE014996B1E06F
:103790002B16310479F50E94406320E030E040E2CE
:1037A00051E40E94D1B70E94F7B960931002709360
:1037B0001102809312029093130281E090E09093A3
:1037C0002C0C80932B0C113401F58091330C882341
:1037D00009F43DCF62E275E0CE0101960E94936547
:1037E000CE0101960E94BE09CE0101960E94FA64A4
:1037F000E12C44C00E9440632091240230912502B4
:103800004091260250912702CCCF163409F044C1D2
:1038100061E080911A020E94A768E2E02E1631044E
:10382000C1F4CE0149960E9440639B01AC016091B6
:103830006A0C70916B0C80916C0C90916D0C0E94D5
:1038400018B960936A0C70936B0C80936C0C909316
:103850006D0C8091330C882371F06BE275E0CE0122
:1038600001960E949365CE0101960E94D509CE0172
:1038700001960E94FA64EE24E394F12C8091330CBB
:10388000882379F140911002509111026091120247
:10389000709113022AE0CE0101960E943265BE01AA
:1038A0006F5F7F4FCE0107960E948A656FE375E0D8
:1038B000CE0107960E94FF63BC01CE010D960E94C7
:1038C0008A65CE010D960E94BE09CE010D960E941A
:1038D000FA64CE0107960E94FA64CE0101960E9416
:1038E000FA648091100290911102A0911202B0919D
:1038F0001302181619061A061B060CF085C5163495
:1039000009F48BC4123509F48CC46E2D80911A020F
:103910000E94A76862E370E080E090E00E94C069C6
:1039200060912B0C809118020E94A76861E070E002
:1039300080E090E00E94C06960E0809118020E94DF
:10394000A76864EF71E080E090E00E94C069C12C3C
:10395000D12C7601C3948091100290911102A09114
:103960001202B0911302C816D906EA06FB060CF043
:103970005AC460912B0C809118020E94A76861E0E4
:1039800070E080E090E00E94C06960E080911802E1
:103990000E94A768609130027091310280913202DA
:1039A000909133020E94C06980913002909131025F
:1039B000A0913202B09133020297A105B1050CF437
:1039C00065C0609124027091250280912602909139
:1039D00027029B01AC010E9419B90E94F7B99B0113
:1039E000AC01C701B6010E94D7B8672B682B692BC1
:1039F00009F04CC032E0231631040CF447C065E8EE
:103A000075E081E893E10E948564C701B6010E94D8
:103A100072B72091240230912502409126025091E4
:103A200027020E9485B9AB01BC0120E0CE010796B8
:103A30000E94026561E873E1CE0101960E948A65E9
:103A4000BE01695F7F4FCE0101960E9415646DE053
:103A500075E00E94FF63BC0181E893E10E94AA64C3
:103A6000CE0101960E94FA64CE0107960E94FA6484
:103A700061E873E1CE0101960E948A65CE0101964C
:103A80000E94351ACE0101960E94FA644FEFC41AC3
:103A9000D40AE40AF40A5FCF123509F0A9CE60E037
:103AA00080911A020E94A768F2E02F163104C1F437
:103AB000CE0149960E9440639B01AC0160916A0C63
:103AC00070916B0C80916C0C90916D0C0E9419B9E7
:103AD00060936A0C70936B0C80936C0C90936D0CDC
:103AE0008091330C882309F4B2CD65E375E0CE01F3
:103AF00001960E949365CE0101960E94D50974CE6D
:103B00002114310429F023E02216310409F09FCD5D
:103B100081E090E090935C0280935B0290932C0C88
:103B200080932B0C4091AA025091AB025EA74DA747
:103B3000052F001F0027001F602F80911A020E948E
:103B4000A7688FEF9FEF90930B0280930A02412C9E
:103B5000512C32011FA218A619A61AA61BA21CA23C
:103B60001DA21EA21F8E18A219A21AA2812C912C8E
:103B700054011DAA1EAA1FAA18AE19AA1AAA1BAA86
:103B80001CAA61E0809118020E94A76861E070E0C1
:103B900080E090E00E94C06960E0809118020E947D
:103BA000A76861E070E080E090E00E94C069C30116
:103BB000B20123E030E040E050E00E94D7B8672B2C
:103BC000682B692B09F0F8C083E090E098AB8FA7D1
:103BD000C12CD12C760180910E02863308F08653D9
:103BE00020917B00982F9870277F922B90937B00D9
:103BF0008770806480937C0080917A0080648093D9
:103C00007A0080917A0086FDFCCF809178006091E7
:103C10007900762F682F072E000C880B990B0E94D5
:103C200072B79B01AC01C701B6010E9419B96B01C3
:103C30007C0162E070E080E090E00E94C069AFA586
:103C4000B8A91197B8ABAFA7AB2B29F620E030EDA0
:103C50004FE355E4C701B6010E9485B96B017C01B1
:103C60008091330C882399F12DEC3CEC4CE45EE31D
:103C7000C701B6010E942DBA87FD29C022E0B70115
:103C8000A601CE0107960E94026566E475E0CE01AA
:103C900001960E949365BE01695F7F4FCE01019638
:103CA0000E941564BC01CE010D960E948A65CE016A
:103CB0000D960E94BE09CE010D960E94FA64CE01B7
:103CC00001960E94FA64CE0107960E94FA642AE9DE
:103CD00039E949E95EE3C701B6010E942DBA87FDC3
:103CE00013C081149104A104B10411F453014201E1
:103CF0002BA13CA14DA15EA1232B242B252B21F42C
:103D00004BA25CA26DA27EA22DEC3CEC4CE45EE3E7
:103D1000C701B6010E946BB718160CF448C0811495
:103D20009104A104B10409F447C08F8D98A1A9A101
:103D3000BAA1892B8A2B8B2B69F42FA138A549A511
:103D40005AA5232B242B252B09F47EC04F8E58A275
:103D500069A27AA28F8D98A1A9A1BAA18816990605
:103D6000AA06BB064CF580910A0290910B0297FFC0
:103D700070C010920B0210920A022F8D38A149A137
:103D80005AA1820E931EA41EB51ED501C401B5957D
:103D9000A795979587958DAB9EABAFABB8AF1F8EB0
:103DA00018A219A21AA2812C912C540105C08114C9
:103DB0009104A104B10471F6E0900A02F0900B02A4
:103DC00092E0E916F1040CF060C0F7FC04C0A3E037
:103DD0002A163104B1F0BFEF4B1A5B0A6B0A7B0A5B
:103DE000E0E44E16ECE95E066104710409F0C9CE08
:103DF00033E02316310429F0E02E2114310409F0B8
:103E000070CD8BA59CA50E9440636B017C01C09284
:103E10006A0CD0926B0CE0926C0CF0926D0C20E06E
:103E200030E044EB53E4C701B6010E942DBA87FD90
:103E3000DCC020E030E044EB53E4C701B6010E944F
:103E400018B96B017C01EBCF4FA258A669A67AA6E0
:103E50007DCF2114310409F0AFCF019690930B026E
:103E600080930A022F8D38A149A15AA1820E931E78
:103E7000A41EB51ED501C401B595A7959795879544
:103E800089AB9AABABABBCAB8ACF69A97AA98BA93A
:103E90009CA92DA93EA94FA958AD621B730B840B99
:103EA000950B0E9472B74B015C01B701FF0C880BA8
:103EB000990B0E9472B79B01AC01C501B4010E942D
:103EC00085B920E030E044EB53E40E9485B96B01F2
:103ED0007C01C0922402D0922502E0922602F09248
:103EE000270220E030E040E85FE30E942DBA87FD22
:103EF00058C080915B0290915C0281309105F1F590
:103F0000C092C215D092C315E092C415F092C515A7
:103F1000C0922002D0922102E0922202F09223026B
:103F200068EA75E0CE0101960E948165CE01019696
:103F30000E94D509CE0101960E94FA6440912402A4
:103F400050912502609126027091270225E0CE0152
:103F500001960E940265CE0101960E94BE09CE0123
:103F600001960E94FA6484EF91E09093DE028093C0
:103F7000DD0264EA74E10E9451923ACF029781F621
:103F8000C092C615D092C715E092C815F092C91517
:103F9000C0921C02D0921D02E0921E02F0921F02FB
:103FA000BFCF6CE875E0CE0101960E948165CE011D
:103FB00001960E94D509CE0101960E94FA644091B3
:103FC000240250912502609126027091270225E07B
:103FD000CE0101960E940265CE0101960E94BE09A3
:103FE000CE0101960E94FA6403CF20E030E0A901DF
:103FF000C701B6010E946BB787FF0BC020E030E01D
:1040000044EB53E4C701B6010E9419B96B017C016E
:10401000ECCFC092210CD092220CE092230CF092B3
:10402000240C4FA058A469A47AA48BA19CA1ADA193
:10403000BEA1481A590A6A0A7B0A21143104D9F42C
:104040001092210C1092220C1092230C1092240C2E
:10405000ADA5BEA5812C912C54018394C12CD12CEB
:104060007601B7FF26C0C12CD12C760188248A9412
:10407000982C54011EC0EDA5FEA5812C912C540155
:104080008394F7FF04C088248A94982C5401C0902C
:10409000210CD090220CE090230CF090240C20E016
:1040A00030E044E353E4C701B6010E946BB787FFD9
:1040B00093C0C701B6019058209124023091250287
:1040C00040912602509127020E94D1B76B017C01DA
:1040D000A3019201C501B4010E94A5B80E9472B764
:1040E00020E030E040E05FE30E94D1B79B01AC01EB
:1040F000C701B6010E9418B90E94F7B96093100277
:104100007093110280931202909313028091330CEA
:10411000882309F441C02AE04FA158A569A57AA5D2
:10412000CE010D960E9432652AE04BA15CA16DA1E3
:104130007EA1CE0107960E9432656DE475E0CE0146
:1041400001960E949365BE01695F7F4FCE01019683
:104150000E9415646EE177E00E94FF63BE01635F19
:104160007F4F0E941564BC01CE0143960E948A6570
:10417000CE0143960E94BE09CE0143960E94FA6486
:10418000CE0101960E94FA64CE0107960E94FA645D
:10419000CE010D960E94FA64809110029091110256
:1041A000A0911202B0911302E12C12E5B7FF99CB56
:1041B000B095A095909581959F4FAF4FBF4F80933D
:1041C000100290931102A0931202B0931302EE24F6
:1041D000E394F12C16E485CB209124023091250242
:1041E00040912602509127022F8F38A349A35AA34A
:1041F000A701960160E070E084EB93E40E9418B997
:104200006093210C7093220C8093230C9093240CC8
:104210002F8D38A149A15AA157CFEE24E394F12C58
:1042200074CBE12C72CB52E02516310424F4211416
:10423000310409F0E1C061E080E00E94097282E08F
:104240002816310424F42114310409F09CC0C090D4
:104250006A0CD0906B0CE0906C0CF0906D0C20E030
:1042600030E044EB53E4C701B6010E942DBA87FD4C
:104270000BC020E030E044EB53E4C701B6010E94DC
:1042800018B96B017C01EBCF20E030E0A901C70138
:10429000B6010E946BB787FF0BC020E030E044EB13
:1042A00053E4C701B6010E9419B96B017C01ECCF40
:1042B000C0926A0CD0926B0CE0926C0CF0926D0C78
:1042C00080915B0290915C020197B1F463E075E02C
:1042D00081E893E10E94CE6280916A0C90916B0C10
:1042E000A0916C0CB0916D0C8093930C9093940CF6
:1042F000A093950CB093960C80915B0290915C0218
:104300000297B1F462E175E081E893E10E94CE6228
:1043100080916A0C90916B0CA0916C0CB0916D0C1B
:1043200080938F0C9093900CA093910CB093920C6F
:1043300040916A0C50916B0C60916C0C70916D0CFB
:1043400020E0CE0107960E94026561E873E1CE018C
:1043500001960E948A65BE01695F7F4FCE0101967A
:104360000E9415646EE075E00E94FF63BC0181E865
:1043700093E10E94AA64CE0101960E94FA64CE01E4
:1043800007960E94FA6491E02916310439F54091AC
:10439000100250911102609112027091130221E0FB
:1043A000CE0107960E94326565E575E0CE01019663
:1043B0000E949365BE01695F7F4FCE0101960E9406
:1043C0001564BC0181E893E10E94AA64CE010196C4
:1043D0000E94FA64CE0107960E94FA6461E873E1D4
:1043E000CE0101960E948A65CE0101960E94351A7F
:1043F000CE0101960E94FA641092100210921102EE
:10440000109212021092130280915B0290915C0252
:104410008130910509F083C080912B0C90912C0C78
:1044200090932E0C80932D0C80911002909111028C
:10443000A0911202B091130280931402909315027E
:10444000A0931602B093170280913002909131022E
:10445000A0913202B091330280932C0290932D02EE
:10446000A0932E02B0932F028091290C80932A0CE6
:104470008091210C9091220CA091230CB091240CDE
:104480008093250C9093260CA093270CB093280CB6
:1044900080916A0C90916B0CA0916C0CB0916D0C9A
:1044A0008093930C9093940CA093950CB093960CDE
:1044B00080910A0290910B0290930D0280930C025E
:1044C000232881F48091240290912502A091260254
:1044D000B09127028093200290932102A0932202A0
:1044E000B0932302CE0149960E94FA64E8960FB673
:1044F000F894DEBF0FBECDBFDF91CF911F910F911A
:10450000FF90EF90DF90CF90BF90AF909F908F90F3
:104510007F906F905F904F903F902F9008950297FB
:1045200009F780912B0C90912C0C9093200C809388
:104530001F0C8091100290911102A0911202B09173
:1045400013028093060290930702A0930802B0938F
:1045500009028091300290913102A0913202B09113
:1045600033028093280290932902A0932A02B093E9
:104570002B028091290C80931E0C8091210C90912C
:10458000220CA091230CB091240C80931A0C9093D0
:104590001B0CA0931C0CB0931D0C80916A0C909185
:1045A0006B0CA0916C0CB0916D0C80938F0C909360
:1045B000900CA093910CB093920C80910A02909170
:1045C0000B029093050280930402232809F08ACFFE
:1045D0008091240290912502A0912602B091270299
:1045E00080931C0290931D02A0931E02B0931F02A1
:1045F00079CF2F923F924F925F926F927F928F92DC
:104600009F92AF92BF92CF92DF92EF92FF920F9361
:104610001F93CF93DF9300D000D01F921F92CDB78E
:10462000DEB767E370E08091C6029091C7020E94F6
:10463000200A84E1482E512C612C712C312C212C24
:104640008FEF281A380AC301B2010E94C06967E3DC
:1046500070E08091C6029091C7020E94200A8C01EE
:1046600083E02816310434F08EE12816310444F436
:10467000012B51F084E1480E511C611C711CE0CFEC
:104680000115110509F0A6C08091C6029091C702DC
:104690008B30910509F086C08090D2159090D3158B
:1046A000A090D415B090D515C090CE15D090CF1550
:1046B000E090D015F090D11564E670E080E090E0D5
:1046C0000E94C06964E475E0CE0101960E94816594
:1046D000CE0101960E94351ACE0101960E94FA641D
:1046E00061E082E00E94097221E0B501A401CE01DF
:1046F00001960E940265BE016F5F7F4F82E596E1E1
:104700000E94DC66CE0101960E94FA646FED82E59C
:1047100096E10E9467726FE375E082E596E10E9480
:10472000FE6620E0B701A601CE0101960E94026557
:10473000BE016F5F7F4F82E596E10E94DC66CE018D
:1047400001960E94FA646CE575E082E596E10E94AC
:10475000D46689829A82AB82BC82CD82DE82EF826D
:10476000F88629813A814B815C816D817E818F81C0
:10477000988528960FB6F894DEBF0FBECDBFDF91A7
:10478000CF911F910F91FF90EF90DF90CF90BF904E
:10479000AF909F908F907F906F905F904F903F90E1
:1047A0002F9008958631910509F476CF0C9709F082
:1047B00083CF80905C0B90905D0BA0905E0BB090CF
:1047C0005F0BC090580BD090590BE0905A0BF090B3
:1047D0005B0B72CF0F3F8FEF1807CCF061E375E0F2
:1047E000CE0101960E9481654AE050E070E060E0F1
:1047F000CE0101960E946019CE0101960E94FA64D2
:104800006EE075E081E893E10E94856432C00E3F5E
:104810008FEF1807B9F160E075E0CE0101960E94B4
:1048200081654AE050E070E060E0CE0101960E94B0
:104830006019CE0101960E94FA6461EF74E081E88C
:1048400093E10E948564B801CE0101960E94D8626E
:10485000BE016F5F7F4F81E893E10E947E64CE01CD
:1048600001960E94FA646BED74E081E893E10E9486
:10487000286419821A821B821C821D821E821F825A
:1048800018866FCF60ED74E0CE0101960E948165BD
:104890004AE050E070E060E0CE0101960E946019AD
:1048A000CE0101960E94FA6460EB74E0ABCF2F92C8
:1048B0003F924F925F926F927F928F929F92AF92B0
:1048C000BF92CF92DF92EF92FF920F931F93CF93FD
:1048D000DF93CDB7DEB7AC970FB6F894DEBF0FBE4F
:1048E000CDBF8C0166E279E08AEB93E10E94CE6253
:1048F00067E370E08091C6029091C7020E94200A8F
:104900001C0160E476E0C8010E942A0D6EE575E0A6
:10491000C8010E94D4666CED75E1CE0101960E943B
:104920008A65BE016F5F7F4FC8010E94DC66CE01C1
:1049300001960E94FA6467E675E0C8010E94D46699
:104940000E948F6C28EE33E040E050E00E94B5B842
:1049500029013A01CE0109960E948E0E6DE675E09E
:10496000CE0101960E949365BE01675F7F4FCE0125
:1049700001960E941564BC01CE010F960E948A65C3
:10498000BE01615F7F4FC8010E94DC66CE010F96B9
:104990000E94FA64CE0101960E94FA64CE01099643
:1049A0000E94FA64C301B20120E13EE040E050E021
:1049B0000E94D7B84B015C01B901CE0187960E94D5
:1049C000AB0D4CE3C42ED12CE12CF12CC501B4016C
:1049D000A70196010E94D7B8B901CE0109960E949D
:1049E000AB0D62E078E0CE0101960E949365BE01B6
:1049F000675F7F4FCE0101960E941564BC01CE0116
:104A000087960E947E64CE0101960E94FA64CE01D0
:104A100009960E94FA64C301B201A70196010E949F
:104A2000D7B8CE0109960E94AB0D62E078E0CE01C6
:104A300001960E949365BE01675F7F4FCE0101968C
:104A40000E941564BC01CE0187960E947E64CE014F
:104A500001960E94FA64CE0109960E94FA6467E703
:104A600075E0CE0101960E949365BE01695D7F4F9E
:104A7000CE0101960E9415646AE775E00E94FF630B
:104A8000BC01CE0109960E948A65BE01675F7F4F17
:104A9000C8010E94DC66CE0109960E94FA64CE012C
:104AA00001960E94FA6468E875E0C8010E94D46625
:104AB000CE0101960E943592B801CE0101960E9466
:104AC000606663E875E0C8010E94C0660E94F92232
:104AD00029833A834B835C836D837E838F8398879E
:104AE00049815A816B817C8121E0CE0109960E9427
:104AF0000265BE01675F7F4FCE010F960E948A65F7
:104B000060E975E0CE010F960E94FF63BC018AEB5D
:104B100093E10E94AA64CE010F960E94FA64CE012E
:104B200009960E94FA6467E975E0CE0109960E9431
:104B300093656AEB73E1CE0109960E941564BC018E
:104B4000CE010F960E948A65BE01615F7F4FC8014A
:104B50000E94DC66CE010F960E94FA64CE0109968F
:104B60000E94FA644D815E816F81788521E0CE01DB
:104B700009960E940265BE01675F7F4F8AEB93E151
:104B80000E94C164CE0109960E94FA6469EA75E048
:104B9000CE0109960E9493656AEB73E1CE010996F6
:104BA0000E9415646AEB75E00E94FF63BC01CE01B0
:104BB0000F960E948A65BE01615F7F4FC8010E9407
:104BC000DC66CE010F960E94FA64CE0109960E941F
:104BD000FA644091930C5091940C6091950C7091F3
:104BE000960C22E0CE010F960E94026561EC75E002
:104BF000CE0109960E949365BE01615F7F4FCE0191
:104C000009960E94156463ED75E00E94FF63BC0184
:104C1000CE0145960E948A65BE016B5E7F4FC8013A
:104C20000E94DC66CE0145960E94FA64CE01099688
:104C30000E94FA64CE010F960E94FA6440918F0C94
:104C40005091900C6091910C7091920C22E0CE01E9
:104C50000F960E9402656CED75E0CE0109960E94E8
:104C60009365BE01615F7F4FCE0109960E94156476
:104C700063ED75E00E94FF63BC01CE0145960E9482
:104C80008A65BE016B5E7F4FC8010E94DC66CE0163
:104C900045960E94FA64CE0109960E94FA64CE01FC
:104CA0000F960E94FA6486EF28168FEF38062CF4D0
:104CB0006BE176E0C8010E942A0D6BEF75E0C80138
:104CC0000E942A0D23E5C22E22E0D22EEE24E39488
:104CD000F12CE2E0CE0ED11C8091590290915A0243
:104CE0008E159F050CF468C0B701CE014B960E944B
:104CF000D8626CEC78E0CE0145960E949365BE01C7
:104D0000655E7F4FCE0145960E9415646EE177E0A7
:104D10000E94FF63BC01CE0181960E948A65BE019C
:104D20006F5D7F4FC8010E94DC66B70183E0660FAC
:104D3000771F8A95E1F768547B4ECE010F960E944B
:104D40009365BE01615F7F4FC8010E94DC666AEE19
:104D500075E0C8010E94D466F60160817181660F1A
:104D6000771F660F771F60557B4ECE0109960E9414
:104D70009365BE01675F7F4FC8010E94DC666FEEDE
:104D800075E0C8010E94D466CE0109960E94FA64BB
:104D9000CE010F960E94FA64CE0181960E94FA64B9
:104DA000CE0145960E94FA64CE014B960E94FA64A9
:104DB000FFEFEF1AFF0A8DCFCE0187960E94FA64AB
:104DC000AC960FB6F894DEBF0FBECDBFDF91CF918A
:104DD0001F910F91FF90EF90DF90CF90BF90AF9019
:104DE0009F908F907F906F905F904F903F902F900B
:104DF00008952F923F924F925F926F927F928F927F
:104E00009F92AF92BF92CF92DF92EF92FF920F9359
:104E10001F93CF93DF93CDB7DEB7CA52D1400FB601
:104E2000F894DEBF0FBECDBFCB5DDE4F5983488304
:104E3000C552D14020918D0C30918E0C2F5F3F4F89
:104E400030938E0C20938D0C20918C0C21110FC36C
:104E50008B016C0181E080938C0C10928E0C10926F
:104E60008D0C66E279E0CE01875E9E4F0E949365CD
:104E700066E279E0CE01815E9E4F0E94936580914B
:104E8000590290915A028230910594F02091940237
:104E9000309195023093560220935502029741F0CB
:104EA00080919602909197029093580280935702B6
:104EB00050E040E064EF75E0C6010E94780D0130DB
:104EC000110509F0CAC266E279E08AEE93E10E9418
:104ED000CE627E0121E8E20EF11CC701880F991F06
:104EE000880F991FFC01E055FB4EC75DDE4FF9832B
:104EF000E883C952D140312C212C3AE0832E912CE9
:104F0000A12CB12C44E6442E512C612C712CCB5D8C
:104F1000DE4FE881F981C552D1408081882309F4B0
:104F200015C2A701BE016F5F7F4FCE018B5D9E4F03
:104F30000E94895D049759F3BE016F5F7F4FCE01D8
:104F40008F5F9E4F0E949365BE016F5F7E4FCE01C3
:104F5000875E9E4F0E94C164CE018F5F9E4F0E946C
:104F6000FA64B701CE018F5F9E4F0E949365BE0128
:104F70006F5F7E4FCE01815E9E4F0E94C164CE0165
:104F80008F5F9E4F0E94FA648091330C8823A1F1B9
:104F9000BE01675E7E4FCE018F5F9E4F0E948A6585
:104FA00061E277E0CE018F5F9E4F0E94FF63BC01FC
:104FB000CE01895F9E4F0E948A65CE01895F9E4F18
:104FC0000E94D509CE01895F9E4F0E94FA64CE01EE
:104FD0008F5F9E4F0E94FA64B701CE018F5F9E4F94
:104FE0000E949365CE018F5F9E4F0E94BE09CE0145
:104FF0008F5F9E4F0E94FA64C35EDE4F8881998165
:10500000CD51D140049708F0E0C070E060E0CE01DF
:10501000875E9E4F0E94B363823531F0843521F064
:105020008D7F843409F0D1C041E050E0BE01675E5D
:105030007E4FCE018F5F9E4F0E946D07CE018F5F26
:105040009E4F0E944B638B016130710521F40091EA
:10505000BE151091BF150330110521F40091C01544
:105060001091C115101611060CF0A9C080915902BB
:1050700090915A02801791070CF4A1C070E060E093
:10508000CE01875E9E4F0E94B363823509F0BFC098
:10509000C7010E94B5B2892B39F4F801EE0FFF1F4A
:1050A000ED5AFD4F11821082C7010E94B5B28130C6
:1050B0009105A1F5F801EE0FFF1FED5AFD4F918309
:1050C00080839801220F331F220F331FC95DDE4FEB
:1050D00039832883C752D140F901E95BFD4F8081B4
:1050E0009181A281B381181619061A061B0644F095
:1050F000073011050CF086C04082518262827382B3
:105100000E94A372C95DDE4FE881F981C752D14088
:10511000E256FD4F6083718382839383C75DDE4FC8
:1051200068817981C952D140CE018D5E9E4F0E9427
:105130009365B801E3E0660F771FEA95E1F76854DD
:105140007B4ECE01835F9E4F0E9493656AEE73E1B2
:10515000CE01895F9E4F0E948A65BE01635F7E4FCC
:10516000CE01895F9E4F0E9415646DE076E00E943B
:10517000FF63BE016F5F7E4F0E94156461E277E0BE
:105180000E94FF63BE016D5E7E4F0E9415646EE15A
:1051900077E00E94FF63BC018AEE93E10E94AA645B
:1051A000CE01895F9E4F0E94FA64CE01835F9E4FBD
:1051B0000E94FA64CE018D5E9E4F0E94FA64CE0179
:1051C0008F5F9E4F0E94FA64A2CEFBE02F1631043F
:1051D0000CF09DCEF6E0F29D8001F39D100D1124A0
:1051E000BE016F5F7F4FC8018E5C9B4E0E94316392
:1051F000B701C80180519C4E0E9431632FEF221AE3
:10520000320A85CE80829182A282B38279CF86349F
:1052100009F074C0C7010E94B5B2892B39F4F801B6
:10522000EE0FFF1FE856FD4F11821082C7010E944A
:10523000B5B28130910539F4F801EE0FFF1FE85641
:10524000FD4F91838083C801880F991F880F991F94
:10525000C95DDE4F99838883C752D140FC01E95B69
:10526000FD4F80819181A281B381181619061A061B
:105270001B063CF007301105E4F540825182628242
:1052800073820E94A372C95DDE4FE881F981C75223
:10529000D140E256FD4F6083718382839383C75D63
:1052A000DE4F68817981C952D140CE018D5E9E4F1B
:1052B0000E949365B80143E0660F771F4A95E1F7B6
:1052C00068547B4ECE01835F9E4F0E9493656AEEC9
:1052D00073E1CE01895F9E4F0E948A65BE01635FC4
:1052E0007E4FCE01895F9E4F0E94156460E176E09B
:1052F0003ECF80829182A282B382C3CF8434C1F434
:10530000C7010E94D3B2000F111F000F111FF80137
:10531000E95CFD4F60837183828393830E94A37253
:1053200002561D4FF801608371838283938347CFB8
:10533000843509F044CFC7010E94D3B2000F111F7A
:10534000000F111FF801E95BFD4FE4CF81E080936E
:10535000010D8091020D882319F0C6010E94572487
:105360008091020D882329F06CEB75E0C6010E9444
:105370002A0D10928C0C8091EE139091EF13892BD3
:1053800009F46BC0CE01895F9E4F0E948E0E6BE4C4
:1053900079E0CE018F5F9E4F0E949365BE01695FE9
:1053A0007E4FCE018F5F9E4F0E9415646EE177E0C5
:1053B0000E94FF636AEE73E10E941564BC018AEEED
:1053C00093E10E94AA64CE018F5F9E4F0E94FA640F
:1053D000CE01895F9E4F0E94FA646AEE73E1CE01AE
:1053E0008F5F9E4F0E948A65AE014F5F5E4F62E005
:1053F00070E089EB92E00E949614182FCE018F5F27
:105400009E4F0E94FA646AEE73E1CE018F5F9E4F59
:10541000112309F446C00E948A6564E176E0CE015A
:105420008F5F9E4F0E94FF6362ED73E10E941564DF
:10543000BC01CE01895F9E4F0E948A65CE01895FC3
:105440009E4F0E94BE09CE01895F9E4F0E94FA6462
:10545000CE018F5F9E4F0E94FA64CE01815E9E4F07
:105460000E94FA64CE01875E9E4F0E94FA64C65D78
:10547000DE4F0FB6F894DEBF0FBECDBFDF91CF91E8
:105480001F910F91FF90EF90DF90CF90BF90AF9062
:105490009F908F907F906F905F904F903F902F9054
:1054A00008950E948A6564E176E0CE018F5F9E4F89
:1054B0000E94FF636CEC73E1B9CFFF920F931F93CF
:1054C000CF93DF93EC018B0180918D0C90918E0C2A
:1054D000019690938E0C80938D0C20918C0C22233E
:1054E00039F06AE070E00E9443BA18161906F4F029
:1054F000FF24F394F0928C0C10928E0C10928D0C71
:1055000050E040E064EF75E0CE010E94780D02307B
:10551000110591F0CE010E945724F092030D6CEB1F
:1055200075E0CE010E942A0D10928C0CDF91CF9174
:105530001F910F91FF9008956BE176E0CE010E94DC
:105540002A0DEDCFAF92BF92CF92DF92EF92FF92F2
:105550000F931F93CF93DF93CDB7DEB7A0970FB60E
:10556000F894DEBF0FBECDBF66E279E084EE93E132
:105570000E94CE6266E279E088ED93E10E94CE62FD
:1055800052E9E52E52E0F52E63E5C62E62E0D62EF6
:105590007BE3A72E72E0B72E01E010E08091590264
:1055A00090915A02801791070CF482C0F501819105
:1055B0009191A191B1915F01892B8A2B8B2B19F5C8
:1055C000F60182819381F70122813381821793074B
:1055D000D1F0880F991FFC01E15DF34FD801AA0FAC
:1055E000BB1FAC5CB34F60818C910E94A768F60131
:1055F00082819381F7019383828364E670E080E087
:1056000090E00E94C069F70162817381CE014596E6
:105610000E94D862B801CE010F960E94D862B801EC
:1056200023E0660F771F2A95E1F768547B4ECE0181
:1056300009960E9493656EE177E0CE0101960E9483
:105640009365BE01675F7F4FCE0101960E9415648E
:105650006DE076E00E94FF63BE01615F7F4F0E94B4
:10566000156461E277E00E94FF63BE016B5E7F4FCD
:105670000E941564BC0184EE93E10E947E64CE0119
:1056800001960E94FA64CE0109960E94FA64CE0146
:105690000F960E94FA64CE0145960E94FA640F5F4D
:1056A0001F4FF2E0EF0EF11C82E0C80ED11C76CF46
:1056B000E091BE15F091BF15EE0FFF1FEE56FD4FA6
:1056C00060817181CE0101960E94D86246E050E06F
:1056D000BE016F5F7F4FCE0109960E94330FBE015E
:1056E000675F7F4F88ED93E10E947E64CE0109964B
:1056F0000E94FA64CE0101960E94FA64E091C015FE
:10570000F091C115EE0FFF1FEE56FD4F60817181C4
:10571000CE0101960E94D86246E050E0BE016F5F64
:105720007F4FCE0109960E94330FBE01675F7F4F06
:1057300088ED93E10E947E64CE0109960E94FA648E
:10574000CE0101960E94FA646EE177E0CE014596A3
:105750000E9493650E948F6C28EE33E040E050E099
:105760000E94B5B869017A0166E279E0CE014B96F4
:105770000E94936566E279E08AEE93E10E94CE6230
:10578000CE0101960E948E0E44E150E0BE016F5F93
:105790007F4FCE0109960E94330FBE01675F7F4F96
:1057A0008AEE93E10E94C164CE0109960E94FA64D8
:1057B000CE0101960E94FA642AE0B701A601CE014B
:1057C00009960E94326548E050E0BE01675F7F4F56
:1057D000CE010F960E94330F6AEE73E1CE0101965F
:1057E0000E948A65BE01615F7F4FCE0101960E94D3
:1057F0001564BC018EED93E10E94AA64CE0101966E
:105800000E94FA64CE010F960E94FA64CE010996B6
:105810000E94FA642AE0B701A601CE0109960E940F
:10582000326560E276E0CE0101960E949365BE018A
:10583000675F7F4FCE0101960E941564BE016B5ECB
:105840007F4F0E941564BC018AEE93E10E947E6442
:10585000CE0101960E94FA64CE0109960E94FA6474
:105860004091930C5091940C6091950C7091960C12
:1058700021E0CE0101960E940265BE016F5F7F4F5D
:10588000CE014B960E94C164CE0101960E94FA643B
:1058900067E276E0CE0101960E949365BE01655EE7
:1058A0007F4FCE0101960E941564BE016B5E7F4F53
:1058B0000E941564BC018AEE93E10E947E64CE01D1
:1058C00001960E94FA64BE01655E7F4FCE0101968B
:1058D0000E948A6546E050E0BE016F5F7F4FCE01B7
:1058E00009960E94330FBE01675F7F4F8EED93E1F3
:1058F0000E947E64CE0109960E94FA64CE01019650
:105900000E94FA6440918F0C5091900C6091910C20
:105910007091920C21E0CE0101960E940265BE01B9
:105920006F5F7F4FCE014B960E94C164CE010196FE
:105930000E94FA6465E376E0CE0101960E949365C9
:10594000BE01655E7F4FCE0101960E941564BE01C7
:105950006B5E7F4F0E941564BC018AEE93E10E944A
:105960007E64CE0101960E94FA64BE01655E7F4F9F
:10597000CE0101960E948A6546E050E0BE016F5F4D
:105980007F4FCE0109960E94330FBE01675F7F4FA4
:105990008EED93E10E947E64CE0109960E94FA6426
:1059A000CE0101960E94FA648091A2179091A317EC
:1059B000892B61F067E370E08091C6029091C70285
:1059C0000E94200A9093A3178093A2178091A21798
:1059D0009091A317892B09F0EEC00E94F922298328
:1059E0003A834B835C836D837E838F839887498161
:1059F0005A816B817C8121E0CE0109960E9402656B
:105A0000BE01675F7F4FCE014B960E94C164CE01FD
:105A100009960E94FA646FE376E0CE0109960E942F
:105A20009365BE01655E7F4FCE0109960E941564A5
:105A3000BE016B5E7F4F0E941564BC018AEE93E14C
:105A40000E947E64CE0109960E94FA64BE01655EE2
:105A50007F4FCE0109960E948A6546E050E0BE0164
:105A6000675F7F4FCE010F960E94330FBE01615FCB
:105A70007F4F8EED93E10E947E64CE010F960E94CF
:105A8000FA64CE0109960E94FA644D815E816F81AD
:105A9000788521E0CE0109960E940265BE01675F0C
:105AA0007F4FCE014B960E94C164CE0109960E94A1
:105AB000FA646AE476E0CE0109960E949365BE011D
:105AC000655E7F4FCE0109960E941564BE016B5E34
:105AD0007F4F0E941564BC018AEE93E10E947E64B0
:105AE000CE0109960E94FA64BE01655E7F4FCE0129
:105AF00009960E948A6546E050E0BE01675F7F4FCD
:105B0000CE010F960E94330FBE01615F7F4F8EED75
:105B100093E10E947E64CE010F960E94FA64CE014A
:105B200009960E94FA6464EE73E18AEE93E10E94A2
:105B30007E646EE177E0CE0101960E94936568ED88
:105B400073E1CE0101960E941564BC018EED93E1D4
:105B50000E947E64CE0101960E94FA646EED73E1AC
:105B6000CE0101960E948A65CE0101960E94BE096F
:105B7000CE0101960E94FA646AE070E080E090E055
:105B80000E94C069CE014B960E94FA64CE014596F0
:105B90000E94FA64A0960FB6F894DEBF0FBECDBF88
:105BA000DF91CF911F910F91FF90EF90DF90CF90F9
:105BB000BF90AF90089560E576E08AEE93E10E9491
:105BC00074646FE576E08EED93E10E94746466E69E
:105BD00076E08AEE93E10E9474646FE576E08EEDE4
:105BE00093E10E9474649FCFDF92EF92FF920F9334
:105BF0001F93CF93DF93CDB7DEB7C451D1400FB61B
:105C0000F894DEBF0FBECDBFCD5EDE4F5983488313
:105C1000C351D14020918D0C30918E0C2F5F3F4F9E
:105C200030938E0C20938D0C20918C0C21113FC051
:105C30008B017C01DD24D394D0928C0C10928E0CBD
:105C400010928D0C66E279E0CE01895F9E4F0E9432
:105C5000936566E279E0CE01835F9E4F0E94936573
:105C600050E040E064EF75E0C7010E94780D01301C
:105C7000110599F466E279E08AEE93E10E94CE6222
:105C8000CD5EDE4FE881F981C351D1408081811121
:105C90001DC00E94A22AD092030DCE01835F9E4FA9
:105CA0000E94FA64CE01895F9E4F0E94FA64CC5E26
:105CB000DE4F0FB6F894DEBF0FBECDBFDF91CF91A0
:105CC0001F910F91FF90EF90DF900895CD5EDE4F12
:105CD000E881F981C351D1408081882309F465C0EE
:105CE000AE014F575F4FBE016F5F7F4FCE018D5E9C
:105CF0009E4F0E94895D049749F3BE016F5F7F4FFD
:105D0000CE018F5F9E4F0E949365BE016F5F7E4FF5
:105D1000CE01895F9E4F0E94C164CE018F5F9E4F6E
:105D20000E94FA64BE016F577F4FCE018F5F9E4F76
:105D30000E949365BE016F5F7E4FCE01835F9E4FD1
:105D40000E94C164CE018F5F9E4F0E94FA64BE0123
:105D5000695F7E4F8AEE93E10E947E64CF5EDE4FE4
:105D600088819981C151D140892B09F4AFCF61E27B
:105D700077E0CE018F5F9E4F0E949365BE01635F07
:105D80007E4FCE018F5F9E4F0E9415646EE177E0DB
:105D90000E94FF63BC018AEE93E10E947E64CE0103
:105DA0008F5F9E4F0E94FA6491CF6AEE73E186EC9A
:105DB00093E10E94AA6471CF8F929F92AF92BF929B
:105DC000EF92FF920F931F93CF93DF93CDB7DEB780
:105DD0006E970FB6F894DEBF0FBECDBF0091FD0CDD
:105DE0001091FE0C0115110509F4DAC00E948F6CA8
:105DF0004B015C0178012EE3E20EF11CF70180817A
:105E00009181A281B381A5019401281B390B4A0B12
:105E10005B0BCA01B901683E33E073078105910548
:105E2000A0F128EE33E040E050E00E94B5B8861AB9
:105E3000970AA80AB90AD7018D929D92AD92BC9299
:105E40001397F80186A597A5A0A9B1A949015A0100
:105E5000880C991CAA1CBB1C88159905AA05BB05B2
:105E600008F0C4C016A617A610AA11AAF80182A9A4
:105E700093A9A4A9B5A988159905AA05BB0508F099
:105E8000BEC012AA13AA14AA15AAF80186A597A53E
:105E9000A0A9B1A9892B8A2B8B2B09F0B9C0EE5B85
:105EA000FF4F8081833009F0B3C084E08083C80154
:105EB0000E945C940196D801D2964D915D916D91AE
:105EC0007C91D597452B462B472BA1F4F801EE5B2F
:105ED000FF4F2081233011F021110CC01082F801F6
:105EE0003E9684E1DF011D928A95E9F7C8010E9480
:105EF0005C9403968230910519F0049709F050C024
:105F000080E591E00E944D5C6091FD0C7091FE0C6B
:105F1000625F7F4FCE0101960E942267CE010396F9
:105F20000E948E896091FD0C7091FE0C6A5E7F4F1D
:105F3000CE0101960E94226744E050E0BE016D5FF1
:105F40007F4F81E090E00E9430876091FD0C70915E
:105F5000FE0C6E5E7F4FCE0101960E94226744E0E8
:105F600050E0BE016D5F7F4F85E090E00E9430877A
:105F70000E9495896091FD0C7091FE0C625E7F4FCE
:105F8000CE0101960E9422678B819C81AD81BE81EA
:105F90008093441290934512A0934612B0934712F7
:105FA00060ED77E080E090E00E94C0690E947E6A28
:105FB0007C0168EE73E080E090E00E94C0690BE035
:105FC00010E0EF2841F50150110929F160ED77E06B
:105FD00080E090E00E94C0690E947E6A7C0168EEC9
:105FE00073E080E090E00E94C069EBCF821B930BCE
:105FF000A40BB50B86A797A7A0ABB1AB37CF821B7D
:10600000930BA40BB50B82AB93ABA4ABB5AB3DCF5D
:1060100090E080E050CF82EE92E10E9433910E94A6
:10602000F61966E279E0CE010D960E94936568E765
:1060300075E0CE0143960E948165CE0149960E948B
:1060400035928E8D1F928F938D8D1F928F938C8D95
:106050001F928F938B8D1F928F9384E894E09F9370
:106060008F938AE99BE09F938F930E940EBD6AE90C
:106070007BE0CE0101960E949365BE016F5F7F4F6A
:10608000CE010D960E94C164CE0101960E94FA6471
:10609000BE016D5E7F4FCE0101960E948A65BE01F2
:1060A000635F7F4FCE0101960E941564BC01CE0153
:1060B00007960E948A65CE0107960E94BE09CE010E
:1060C00007960E94FA64CE0101960E94FA64BE010E
:1060D000635F7F4FCE0101960E948A65AE014F5FDC
:1060E0005F4F63E070E088EC92E00E949614182FF6
:1060F000CE0101960E94FA640FB6F894DEBF0FBE7F
:10610000CDBF111122C060E776E0CE0101960E945A
:106110009365BE016D5E7F4FCE0101960E941564AE
:106120006CEC73E10E941564BC01CE0107960E94DD
:106130008A65CE0107960E94BE09CE0107960E948D
:10614000FA64CE0101960E94FA64CE0143960E9441
:10615000FA64CE010D960E94FA646E960FB6F8941A
:10616000DEBF0FBECDBFDF91CF911F910F91FF908A
:10617000EF90BF90AF909F908F9008957F928F92F5
:106180009F92AF92BF92CF92DF92EF92FF920F93C6
:106190001F93CF93DF93CDB7DEB762970FB6F89416
:1061A000DEBF0FBECDBF10E000E036E6C32E3BE001
:1061B000D32E40E3E42E53EEB52E66E0A62E7CEE01
:1061C000972EE1E3FE2EFEE48F2EA4E37A2E68EBF9
:1061D00072E28FE993E10E94658FF6018E2D119294
:1061E0008A95E9F7B092660BA092680B9092690BC2
:1061F000F092720B8092730BF092740B7092750B8D
:1062000060E072E0CE0101960E9422674BE750E009
:10621000BE016F5F7F4F8FE993E10E94EE8F40E3F5
:1062200050E066E67BE08FE993E10E94838F8FE97F
:1062300093E10E94BD8F68EE73E080E090E00E94E1
:10624000C0698FE993E10E94B98B892B31F50A303F
:10625000110509F05FC169E776E0CE0101960E9461
:106260009365CE0101960E94BE09CE0101960E945F
:10627000FA6462960FB6F894DEBF0FBECDBFDF9111
:10628000CF911F910F91FF90EF90DF90CF90BF9033
:10629000AF909F908F907F90089540E350E066E626
:1062A0007BE08FE993E10E94708B60918E0B70917F
:1062B0008F0B76276727762790E080E0CB01772742
:1062C0006627C090900BD090910BDC24CD24DC2469
:1062D000F12CE12C6C297D298E299F297E508A4A38
:1062E00093480E947E720E94A3726093960B7093F3
:1062F000970B8093980B9093990B0A30110509F432
:10630000AACF0E94A37260939B0C70939C0C809305
:106310009D0C90939E0C0E94A37260939F0C7093AF
:10632000A00C8093A10C9093A20CCE0101960E9428
:106330008E0ECE0101960E94BE09CE0101960E94EA
:10634000FA640E94FB72BC01CE0107960E94AB0D5D
:1063500062E574E0CE0107960E9474640E94F372B5
:10636000BC01CE0101960E94AB0DBE016F5F7F4F55
:10637000CE0107960E947E64CE0101960E94FA64C7
:1063800062E574E0CE0107960E9474640E94E9728F
:10639000BC01CE0101960E94AB0DBE016F5F7F4F25
:1063A000CE0107960E947E64CE0101960E94FA6497
:1063B00063E876E0CE0101960E949365BE01695FB5
:1063C0007F4FCE0101960E941564BC01CE010D964F
:1063D0000E948A654AE050E06FEF7FEFCE010D9694
:1063E0000E946019CE010D960E94FA64CE010196BA
:1063F0000E94FA64CE0107960E94FA6468EE73E088
:1064000080E090E00E94C0690E940B73BC01CE0145
:106410000D960E94AB0D0E940373BC01CE01019644
:106420000E94AB0D62E078E0CE0107960E94936572
:10643000BE016F5F7F4FCE0107960E941564BC01BD
:10644000CE010D960E947E64CE0107960E94FA64EA
:10645000CE0101960E94FA640E94A3720E94CB773B
:1064600060917E0C70E0CE0101960E94AB0D62E05F
:1064700078E0CE0107960E949365BE016F5F7F4F63
:10648000CE0107960E941564BC01CE010D960E94B4
:106490007E64CE0107960E94FA64CE0101960E94A6
:1064A000FA6469E876E0CE0101960E949365BE0128
:1064B000635F7F4FCE0101960E941564BC01CE013F
:1064C00007960E948A654AE050E06FEF7FEFCE01A9
:1064D00007960E946019CE0107960E94FA64CE01C9
:1064E00001960E94FA64CE010D960E94FA6468EE4D
:1064F00073E080E090E00E94C069CE0101960E94A6
:106500000D0E4AE050E06FEF7FEFCE0101960E9442
:106510006019ABCE0F5F1F4F68EE73E080E090E034
:106520000E94C0694091960B5091970B6091980B17
:106530007091990BCE0101960E940463CE010196E1
:106540000E94BE09CE0101960E94FA6440CE2F92AD
:106550003F924F925F926F927F928F929F92AF92F3
:10656000BF92CF92DF92EF92FF920F931F93CF9340
:10657000DF93CDB7DEB7C055D1090FB6F894DEBFB3
:106580000FBECDBF69E973E1CE018F5B9F4F0E94C3
:106590008A6523960EAD1FAD23970115110571F085
:1065A000D8018D918D01882349F0082E000C990B9C
:1065B0000E9485BCF80131978083F2CF6FE876E0C6
:1065C000CE0101960E949365BE016F5F7F4FCE01A1
:1065D0008F5B9F4F0E94E463182FCE0101960E94AB
:1065E000FA64112309F403C145E050E069E973E15D
:1065F000CE0101960E946D07BE016F5F7F4F8BE752
:1066000093E10E94C164CE0101960E94FA648BE777
:1066100093E10E94566360E08BE793E10E9452642D
:1066200040917F13509180136CEF74E18BE793E1FD
:106630000E94BF5F6CE774E0CE0101960E949365F3
:10664000BE016F5F7F4F8BE793E10E94E463182FD9
:10665000CE0101960E94FA6466E674E0111102C050
:106660006BE674E0CE0101960E9493656BE773E1DF
:10667000CE0101960E941564BC018AEF95E10E944B
:10668000AA64CE0101960E94FA648AEF95E10E9405
:1066900056634091FE155091FF15415051096AEF24
:1066A00075E1CE0101960E946D07BE016F5F7F4FBD
:1066B0008CED95E10E94C164CE0101960E94FA64BE
:1066C0008CED95E10E944B630E9472B79B01AC0177
:1066D0000E9432BA882309F448C06091FE15709177
:1066E000FF15625071098AEF95E10E94B363682F2C
:1066F000CE0101960E945F65BE016F5F7F4F8CEDFA
:1067000095E10E94C164CE0101960E94FA646CE793
:1067100074E0CE0101960E949365BE016F5F7F4FCA
:106720008CED95E10E94E463182FCE0101960E9442
:10673000FA641123D1F06091FE157091FF1563503A
:1067400071098AEF95E10E94B363682FCE0101962B
:106750000E945F65BE016F5F7F4F8CED95E10E94E7
:10676000C164CE0101960E94FA6484EF91E0909397
:10677000DE028093DD0264EA74E10E94519264E6D5
:1067800070E080E090E00E94C0698091340288232C
:1067900071F069E973E1CE0101960E948A65CE012C
:1067A00001960E94E10DCE0101960E94FA64CE018D
:1067B0008F5B9F4F0E94FA6481E0C05BDF4F0FB692
:1067C000F894DEBF0FBECDBFDF91CF911F910F9127
:1067D000FF90EF90DF90CF90BF90AF909F908F9001
:1067E0007F906F905F904F903F902F90089565E954
:1067F00076E0CE0101960E949365BE016F5F7F4FE8
:10680000CE018F5B9F4F0E94E463182FCE0101964B
:106810000E94FA64112309F447C045E050E069E999
:1068200073E1CE0101960E946D07BE016F5F7F4F3D
:106830008BE793E10E94C164CE0101960E94FA6445
:106840008BE793E10E94566360E08BE793E10E943F
:10685000526440917F135091801364ED74E18BE793
:1068600093E10E94BF5F64ED74E1CE014C960E94FB
:1068700093656EE774E0CE0101960E949365BE01B8
:10688000645E7F4FCE0101960E941564BC0184EFC7
:1068900095E10E94AA64CE0101960E94FA64CE019D
:1068A0004C960E94FA6461CF6BE976E0CE010196C6
:1068B0000E949365BE016F5F7F4FCE018F5B9F4F3C
:1068C0000E94E463182FCE0101960E94FA641123FE
:1068D000E1F043E050E069E973E1CE0101960E94E6
:1068E0006D07BE016F5F7F4F8BE793E10E94C1642C
:1068F000CE0101960E94FA646BE773E1CE01019626
:106900000E948A65CE010196CCCF6FE976E0CE0178
:1069100001960E949365BE016F5F7F4FCE018F5B32
:106920009F4F0E94E463182FCE0101960E94FA64E3
:10693000112301F144E050E069E973E1CE010196D1
:106940000E946D07BE016F5F7F4F8BE793E10E944E
:10695000C164CE0101960E94FA648BE793E10E9424
:106960004B6370936315609362157093C7026093D5
:10697000C602FBCE64EA76E0CE0101960E949365E2
:10698000BE016F5F7F4FCE018F5B9F4F0E94E4631C
:10699000182FCE0101960E94FA64112309F449C010
:1069A00045E050E069E973E1CE0101960E946D0770
:1069B000BE016F5F7F4F8BE793E10E94C164CE0100
:1069C00001960E94FA648BE793E10E944B637093F7
:1069D000BF156093BE1584EF91E09093DE02809323
:1069E000DD0264EA74E10E94519264E670E080E0A6
:1069F00090E00E94C0696CEC78E0CE0101960E94A4
:106A0000936569E973E1CE0101960E941564BC01AA
:106A1000CE014C960E948A65CE014C960E94BE091A
:106A2000CE014C960E94FA64CE0101960E94FA644F
:106A3000ACCE6AEA76E0CE0101960E949365BE0173
:106A40006F5F7F4FCE018F5B9F4F0E94E463182FD3
:106A5000CE0101960E94FA641123E1F044E050E077
:106A600069E973E1CE0101960E946D07BE016F5F77
:106A70007F4F8BE793E10E94C164CE0101960E9493
:106A8000FA648BE793E10E944B637093C1156093A6
:106A9000C015A1CF6FEA76E0CE0101960E94936502
:106AA000BE016F5F7F4FCE018F5B9F4F0E94E463FB
:106AB000182FCE0101960E94FA641123A1F044E040
:106AC00050E069E973E1CE0101960E946D07BE01B5
:106AD0006F5F7F4F8BE793E10E94C164CE01019607
:106AE0000E94FA6482CF64EB76E0CE0101960E94A8
:106AF0009365BE016F5F7F4FCE018F5B9F4F0E94FA
:106B0000E463182FCE0101960E94FA641123A1F0CC
:106B100047E050E069E973E1CE0101960E946D07FC
:106B2000BE016F5F7F4F8BE793E10E94C164CE018E
:106B300001960E94FA6423CE6CEB76E0CE010196BA
:106B40000E949365BE016F5F7F4FCE018F5B9F4FA9
:106B50000E94E463182FCE0101960E94FA6411117D
:106B6000D7CF64EC76E0CE0101960E949365BE011A
:106B70006F5F7F4FCE018F5B9F4F0E94E463182FA2
:106B8000CE0101960E94FA64112321F081E00E9457
:106B9000980CF5CD6EEC76E0CE0101960E949365DF
:106BA000BE016F5F7F4FCE018F5B9F4F0E94E463FA
:106BB000182FCE0101960E94FA64112319F00E9449
:106BC000DC2EDDCD65ED76E0CE0101960E94936569
:106BD000BE016F5F7F4FCE018F5B9F4F0E94E463CA
:106BE000182FCE0101960E94FA64112309F454C0B3
:106BF0004AE050E069E973E1CE0101960E946D0719
:106C0000BE016F5F7F4F8BE793E10E94C164CE01AD
:106C100001960E94FA648BE793E10E944B630E9405
:106C20007E720E94A37260939B0C70939C0C809365
:106C30009D0C90939E0C0E94A37260939F0C709386
:106C4000A00C8093A10C9093A20CCE014C960E94B4
:106C50008E0E60EE76E0CE0101960E949365BE0135
:106C6000645E7F4FCE0101960E941564BC01CE0187
:106C70008A960E948A65CE018A960E94BE09CE013C
:106C80008A960E94FA64CE0101960E94FA64CE01AF
:106C90004C960E94FA6479CD66E478E0CE010196C4
:106CA0000E949365BE016F5F7F4FCE018F5B9F4F48
:106CB0000E94E463182FCE0101960E94FA6411230A
:106CC00009F46CC045E050E069E973E1CE0101963A
:106CD0000E946D07BE016F5F7F4F8BE793E10E94BB
:106CE000C164CE0101960E94FA640E94A37260936F
:106CF0009B0C70939C0C80939D0C90939E0C8BE747
:106D000093E10E944B6360935D0270935E028093F7
:106D10005F02909360026093A4157093A515809311
:106D2000A6159093A7152091A3152093010D672B0D
:106D3000682B692B11F41092010D84EF91E0909370
:106D4000DE028093DD0264EA74E10E94519264E6FF
:106D500070E080E090E00E94C0696DE879E0CE01CB
:106D600001960E948165CE0101960E94D509CE014F
:106D700001960E94FA6440915D0250915E0260911A
:106D80005F0270916002CE0101960E940463CE0101
:106D900001960E94BE09CE0101967BCF61EF76E09D
:106DA000CE0101960E949365BE016F5F7F4FCE01B9
:106DB0008F5B9F4F0E94E463182FCE0101960E94C3
:106DC000FA641123D9F14AE050E069E973E1CE0198
:106DD00001960E946D07BE016F5F7F4F8BE793E1C5
:106DE0000E94C164CE0101960E94FA648BE793E190
:106DF0000E944B63613071058105910519F481E0B2
:106E00008093A3158BE793E10E944B63672B682B5C
:106E1000692B11F41092A3158091A3158093010D95
:106E2000882309F4D8CD0E94A37260939B0C7093C1
:106E30009C0C80939D0C90939E0CCDCD6CEF76E0D6
:106E4000CE0101960E949365BE016F5F7F4FCE0118
:106E50008F5B9F4F0E94E463182FCE0101960E9422
:106E6000FA64112359F148E050E069E973E1CE0179
:106E700001960E946D07BE016F5F7F4F8BE793E124
:106E80000E94C164CE0101960E94FA648BE793E1EF
:106E90000E944B63613071058105910519F481E011
:106EA0008093A70C8BE793E10E944B63672B682BC1
:106EB000692B09F0A0CD1092A70C9DCD65E077E07D
:106EC000CE0101960E949365BE016F5F7F4FCE0198
:106ED0008F5B9F4F0E94E463182FCE0101960E94A2
:106EE000FA64112321F145E050E069E973E1CE0134
:106EF00001960E946D07BE016F5F7F4F8BE793E1A4
:106F00000E94C164CE0101960E94FA648BE793E16E
:106F10000E944B636130710521F481E08093020D82
:106F200034CC672B09F031CC1092020D2ECC6BE0E3
:106F300077E0CE0101960E949365BE016F5F7F4F9F
:106F4000CE018F5B9F4F0E94E463182FCE01019604
:106F50000E94FA64112309F472C066E070E089E9C6
:106F600093E10E94B363682FCE0101960E945F6592
:106F7000BE016F5F7F4F8BE793E10E94C164CE013A
:106F800001960E94FA648BE793E10E94566360E0E9
:106F90008BE793E10E9452648BE793E10E944B637D
:106FA0006B01CB01181619060CF0EFCB209159029A
:106FB00030915A02261737070CF4E7CB48E050E02F
:106FC00069E973E1CE0101960E946D07BE016F5F12
:106FD0007F4F8BE793E10E94C164CE0101960E942E
:106FE000FA648BE793E10E94566380917F1390913E
:106FF00080130997A8F028E030E050E040E06BE70C
:1070000073E1CE0101960E94A865BE016F5F7F4FBC
:107010008BE793E10E94C164CE0101960E94FA645D
:10702000B601E3E0660F771FEA95E1F768547B4EFF
:1070300048E050E08BE793E10E94BF5F96CB62E1AE
:1070400077E0CE0101960E949365BE016F5F7F4F8E
:10705000CE018F5B9F4F0E94E463182FCE010196F3
:107060000E94FA64112309F402C26EE177E0CE01B6
:107070004C960E94936569E177E0CE0101960E94EB
:107080009365AE01445E5F4FBE016F5F7F4FCE01DF
:107090008F5B9F4F0E94ABA1CE0101960E94FA64C4
:1070A000CE014C960E94FA646EE177E0CE014C96D8
:1070B0000E9493656BE177E0CE0101960E94936593
:1070C000AE01445E5F4FBE016F5F7F4FCE018F5BAD
:1070D0009F4F0E94ABA1CE0101960E94FA64CE019F
:1070E0004C960E94FA646EE177E0CE014C960E94C5
:1070F00093656DE177E0CE0101960E949365AE0144
:10710000445E5F4FBE016F5F7F4FCE018F5B9F4F2D
:107110000E94ABA1CE0101960E94FA64CE014C966A
:107120000E94FA6461E277E0CE014C960E9493657A
:1071300060E277E0CE0101960E949365AE01445E65
:107140005F4FBE016F5F7F4FCE018F5B9F4F0E94ED
:10715000ABA1CE0101960E94FA64CE014C960E942A
:10716000FA6461E277E0CE014C960E94936566EA8C
:1071700075E0CE0101960E949365AE01445E5F4FBB
:10718000BE016F5F7F4FCE018F5B9F4F0E94ABA10F
:10719000CE0101960E94FA64CE014C960E94FA64D8
:1071A000CE018F5B9F4F0E9456630E94A372609333
:1071B000880C7093890C80938A0C90938B0C56E00A
:1071C000E52EF12C64E6462E512C612C712C88247E
:1071D0008394912C5701B3E0AB0EB11C27968EAD72
:1071E0009FAD27970197A816B90608F0CECAB70138
:1071F000CE018F5B9F4F0E94B363682FCE014C96E8
:107200000E945F656701E2E0CE0ED11CFFEFEF1A2E
:10721000FF0A9601A701BE016F5B7F4FCE01019669
:107220000E94A865CE0101960E944B638B01CE019E
:1072300001960E94FA640130110521F40091BE15F7
:107240001091BF150330110521F40091C015109164
:10725000C1156EE177E0CE0101960E949365A6010B
:10726000BE016F5F7F4FCE018F5B9F4F0E94A4A234
:107270006C01CE0101960E94FA6466E279E0CE01CB
:1072800001960E9493651C141D0424F59601A50126
:10729000BE016F5B7F4FCE018A960E94A865BE013A
:1072A000665D7F4FCE0101960E94C164CE018A9631
:1072B0000E94FA64101611061CF176012FEFE21AF3
:1072C000F20ACE0101960E94FA64CE014C960E9409
:1072D000FA6480CFA501BE016F5B7F4FCE018A9615
:1072E0000E946D07BE01665D7F4FCE0101960E9430
:1072F000C164CE018A960E94FA64101611060CF73A
:107300008091590290915A02801791070CF446C05F
:1073100070E060E0CE014C960E94B363823509F0C4
:1073200042C0CE0101960E944B63672B682B692BEC
:1073300039F4F801EE0FFF1FED5AFD4F1182108254
:10734000CE0101960E944B63613071058105910564
:1073500029F5F801EE0FFF1FED5AFD4F9182808253
:10736000000F111F000F111FF801E95BFD4F808115
:107370009181A281B381181619061A061B0624F002
:1073800040825182628273820E94A37202561D4F14
:10739000D8016D937D938D939C9313971C141D04BA
:1073A0000CF48BCF8ECF8634E9F5CE0101960E9486
:1073B0004B63672B682B692B39F4F801EE0FFF1F25
:1073C000E856FD4F11821082CE0101960E944B6358
:1073D000613071058105910539F4F801EE0FFF1F49
:1073E000E856FD4F91828082000F111F000F111F80
:1073F000F801E95BFD4F80819181A281B38118166C
:1074000019061A061B0624F040825182628273829A
:107410000E94A37202561D4FF8016083718382831C
:107420009383BCCF843481F4CE0101960E944B63D8
:10743000000F111F000F111FF801E95CFD4F608361
:10744000718382839383A0CF843509F0A7CFCE01C7
:1074500001960E944B63000F111F000F111FF801CE
:10746000E95BFD4F6083718382839383D1CF68E8AA
:1074700079E0CE0101960E948165BE016F5F7F4F6A
:10748000CE018F5B9F4F0E94E463182FCE010196BF
:107490000E94FA64112309F41CC144E050E069E938
:1074A00073E1CE0101960E946D07BE016F5F7F4FB1
:1074B0008BE793E10E94C164CE0101960E94FA64B9
:1074C0008BE793E10E94566360E08BE793E10E94B3
:1074D000526440917F13509180136EE67CE08BE7FD
:1074E00093E10E94BF5F61E07AE0CE01CB960E94FB
:1074F00093656BE773E1CE01C3960E948A658FA9FD
:1075000098AD10E0892BE1F066E279E0CE018A9631
:107510000E94936521968EAD9FAD21979E01295BB8
:107520003F4F7901892B09F05DC0CE01C3960E94BF
:107530004B63D7016C93CE018A960E94FA6411E0E6
:10754000CE01C3960E94FA64CE01CB960E94FA64E3
:10755000112309F41AC98E01095B1F4FE0EDEE2ECD
:10756000E4E1FE2E6801B4E0CB0ED11CF80181915C
:107570008F01D7018D937D011D8E1C8E1F8E1E8E57
:1075800019A218A24AE0BE016F5F7F4F90E00E94EF
:1075900077B3BE016F5F7F4FCE014C960E94CE62E3
:1075A000CE014C960E94BE09CE014C960E94FA6410
:1075B000C016D106D9F684EF91E09093DE02809355
:1075C000DD0264EA74E10E94519264E670E080E0BA
:1075D00090E00E94C0696DE779E0CE0101960E94BB
:1075E0008165D5CB50E040E0BE01655C7F4FCE01A8
:1075F000C3960E94A4A28C01892B11F40FA918AD87
:107600004E01BCE18B0E911C66E279E0C4010E9440
:1076100093655701D12CC12C782C692C45018E180B
:107620009F081016110684F59801A601BE016D5C35
:107630007F4FCE0101960E94A865BE016F5F7F4F0C
:10764000872D962D0E94C164CE0101960E94FA6496
:10765000872D962D0E944B63F50161935F016801B0
:10766000FFEFCF1ADF0AA601BE01655C7F4FCE0196
:10767000C3960E94A4A28C018FA998ADC816D90602
:1076800068F210E000E0CACF8FA998ADC816D906FD
:10769000D8F4A601BE016D5C7F4FCE0101960E9419
:1076A0006D07BE016F5F7F4FCE014C960E94C16493
:1076B000CE0101960E94FA64CE014C960E944B6363
:1076C000E80CF91CD7016C93CE014C960E94FA6429
:1076D00032CF66E779E0CE0101960E948165BE0156
:1076E0006F5F7F4FCE018F5B9F4F0E94E463182F27
:1076F000CE0101960E94FA641123E9F146E050E0C0
:1077000069E973E1CE0101960E946D07BE016F5FCA
:107710007F4F8BE793E10E94C164CE0101960E94E6
:10772000FA648BE793E10E94566380917F139091F6
:107730008013892B09F429C88BE793E10E944B63DE
:107740007093CD156093CC1570933602609335021B
:1077500084EF91E09093DE028093DD0264EA74E1AD
:107760000E94519264E670E080E090E00E94C0695F
:1077700062E679E032CF63E277E0CE0101960E94C3
:107780009365BE016F5F7F4FCE018F5B9F4F0E945D
:10779000E463182FCE0101960E94FA641123A9F028
:1077A00065E579E0CE0101960E94816564E670E0AE
:1077B000CE0101960E943672CE0101960E94FA64B3
:1077C000F0E0E0E019950C94C5336AE277E0CE0171
:1077D0004C960E949365BE01645E7F4F89E993E1F8
:1077E0000E94E46311E0811115C062E377E0CE01ED
:1077F00001960E949365BE016F5F7F4F89E993E117
:107800000E94E46311E0811101C010E0CE010196F5
:107810000E94FA64CE014C960E94FA64112389F109
:107820006AE377E0CE0101960E94936562EE75E10E
:10783000CE0101960E941564BC0181E893E10E948B
:10784000AA64CE0101960E94FA646CEC78E0CE0145
:1078500001960E94936561E873E1CE0101960E9452
:107860001564BC01CE014C960E948A65CE014C96EF
:107870000E94BE09CE014C960E94FA64CE01019688
:107880006CC564E477E0CE014C960E949365BE011E
:10789000645E7F4F89E993E10E94E46311E0811106
:1078A00015C06BE477E0CE0101960E949365BE019E
:1078B0006F5F7F4F89E993E10E94E46311E08111DA
:1078C00001C010E0CE0101960E94FA64CE014C96F0
:1078D0000E94FA64112369F067E479E081E893E19A
:1078E0000E94856468EE75E181E893E10E947E6400
:1078F000ACCF62E577E0CE0101960E949365BE01B0
:107900006F5F7F4FCE018F5B9F4F0E94E463182F04
:10791000CE0101960E94FA64112331F00E94BE301C
:10792000109234020C94C5336BE577E0CE014C968F
:107930000E949365BE01645E7F4F89E993E10E94D6
:10794000E46311E0811115C060E677E0CE01019695
:107950000E949365BE016F5F7F4F89E993E10E94AA
:10796000E46311E0811101C010E0CE0101960E9494
:10797000FA64CE014C960E94FA64112309F441C0C6
:1079800061E277E0CE0101960E94936540919D13DC
:1079900050919E138D819E81481B590BBE016F5FD4
:1079A0007F4F89E993E10E945DA1AC014F5F5F4F7A
:1079B00069E973E1CE014C960E946D07BE01645ED9
:1079C0007F4F8BE793E10E94C164CE014C960E94E9
:1079D000FA64CE0101960E94FA648BE793E10E945B
:1079E0004B636115710531F481E0809391020E942F
:1079F000B69F96CF6130710509F092CF1092910237
:107A0000F6CF65E677E0CE0101960E949365BE0150
:107A10006F5F7F4FCE018F5B9F4F0E94E463182FF3
:107A2000CE0101960E94FA64112309F43BC143E0A0
:107A300050E069E973E1CE0101960E946D07BE0135
:107A40006F5F7F4F8BE793E10E94C164CE01019687
:107A50000E94FA646BE773E1CE0101960E948A6589
:107A6000CE0101960E94E10DCE0101960E94FA64BA
:107A700084EF91E09093DE028093DD026BE773E187
:107A8000CE0101960E948A6560E0CE0101960E94B7
:107A90006664BC018EEE95E10E94AA64CE01019657
:107AA0000E94FA646BE773E1CE0101960E948A6539
:107AB00060E0CE0101960E946664BC0188EE95E10B
:107AC0000E94AA64CE0101960E94FA644091F215C8
:107AD0005091F31564E675E18EEE95E10E94BF5F6B
:107AE0004091EC155091ED156FE675E188EE95E14A
:107AF0000E94BF5F64EA74E18091DD029091DE0232
:107B00000E94519269E677E0CE0101960E9493654A
:107B10006BE773E1CE0101960E941564BC01CE01B2
:107B20008A960E948A65CE0101960E94FA6480912D
:107B3000601590916115892B39F4BE01665D7F4F08
:107B400089E79FE00E94DC6668EB7BE080E090E0E4
:107B50000E94C0698091601590916115029709F0AB
:107B600087C06BE773E1CE01C3960E948A6561E727
:107B700077E0CE0101960E949365CE0101960E94A6
:107B8000E29FCE0101960E94FA6464EF71E080E00A
:107B900090E00E94C06964E777E0CE0101960E9400
:107BA0009365CE0101960E94E29FCE0101960E944C
:107BB000FA646CED75E080E090E00E94C0696DE7CA
:107BC00077E0CE0101960E949365CE0101960E9456
:107BD000E29FCE0101960E94FA6464EF71E080E0BA
:107BE00090E00E94C0696BE877E0CE0101960E94A8
:107BF0009365CE0101960E94E29FCE0101960E94FC
:107C0000FA6464EF71E080E090E00E94C06969E688
:107C100077E0CE0101960E949365BE016D5C7F4FB7
:107C2000CE0101960E941564BC01CE014C960E94C3
:107C30008A65CE0101960E94FA64CE014C960E949C
:107C40005663BE01645E7F4FCE0101960E948A6535
:107C5000CE0101960E94E29FCE0101960E94FA6435
:107C6000CE014C960E94FA64CE01C3960E94FA643B
:107C700068EB7BE080E090E00E94C06964E675E11B
:107C8000CE0101960E949365CE0101960E94E10DFE
:107C9000CE0101960E94FA6410923402CE018A96B7
:107CA0000C94493669E977E0CE0101960E9493650C
:107CB000BE016F5F7F4FCE018F5B9F4F0E94E463D9
:107CC000182FCE0101960E94FA64112309F486C090
:107CD00044E050E069E973E1CE0101960E946D072E
:107CE000BE016F5F7F4F8BE793E10E94C164CE01BD
:107CF00001960E94FA646EE977E0CE0101960E9437
:107D000093656BE773E1CE0101960E941564BC0197
:107D1000CE014C960E948A65CE0101960E94FA64BB
:107D20008091601590916115892B39F4BE01645ED4
:107D30007F4F89E79FE00E94DC6668E873E180E09E
:107D400090E00E94C0698091601590916115029742
:107D500059F565EA77E0CE0101960E94936580911E
:107D60007F1390918013892B19F56EEA77E0CE018D
:107D700001960E94CE62BE01645E7F4FCE018A965C
:107D80000E948A65CE018A960E94E29FCE018A9661
:107D90000E94FA6468E873E180E090E00E94C069A4
:107DA000CE0101960E94FA64109234020C94473678
:107DB000BE016F5F7F4FCE018A960E948A65CE0119
:107DC0008A960E94E29FCE018A960E94FA6460E73A
:107DD00077E180E090E00E94C069CDCF67EB77E06B
:107DE000CE0101960E949365BE016F5F7F4FCE0169
:107DF0008F5B9F4F0E94E463182FCE0101960E9473
:107E0000FA64112309F45CC069E973E18BE793E13B
:107E10000E94AA6481E08093340269E973E1CE0193
:107E200001960E948A65CE0101960E94E10DCE0165
:107E300001960E94FA6480916015909161150297F5
:107E400009F16BE773E189E79FE00E94DC6668EB6C
:107E50007BE080E090E00E94C069CE0101960E9424
:107E60007BA0BE016F5F7F4F89E993E10E94C164EF
:107E7000CE0101960E94FA6460ED77E080E090E028
:107E80000E94C0698091601590916115029771F40C
:107E90006BE773E1CE0101960E948A65CE010196DF
:107EA0000E94E29FCE0101960E94FA6480919D1388
:107EB00090919E13892B09F433CD6CEC78E0BCC60D
:107EC0006BEB77E0CE0101960E949365BE016F5F78
:107ED0007F4FCE018F5B9F4F0E94E463182FCE012E
:107EE00001960E94FA64112309F492C180916015F1
:107EF00090916115019709F013CD61EC77E0CE0107
:107F0000C3960E949365BE016D5C7F4F89E79FE039
:107F10000E94DC666CE271E080E090E00E94C06943
:107F2000CE018A960E947BA064E670E080E090E03B
:107F30000E94C06910E000E065E0C62ED12C7AE016
:107F4000A72EB12C6CEC77E0CE0101960E949365D0
:107F500050E040E0BE016F5F7F4FCE018A960E94E5
:107F6000A4A27C01CE0101960E94FA64A7014F5F92
:107F70005F4FBE01665D7F4FCE0101960E946D0787
:107F8000BE016F5F7F4FCE01C3960E94C164CE01D8
:107F900001960E94FA648FA998AD892B09F170E0CF
:107FA00060E0CE01C3960E94B363082E000C990BCB
:107FB000C0970A97A8F46EEC77E0CE0101960E9474
:107FC0009365BE016F5F7F4FCE01C3960E94E4634D
:107FD000E82ECE0101960E94FA64FF24F394E1108A
:107FE000F12C60E178E0CE0101960E94816564E1A8
:107FF00070E0CE0101960E9438A5CE0101960E9444
:10800000FA640F5F1F4F62E370E080E090E00E942F
:10801000C069C801B6010E9443BA0197C1F4CE01FC
:1080200001960E947A0F8D819E81892B09F4BBC035
:10803000BE016F5F7F4F89E993E10E94AA640E94AD
:10804000A732FF24F394CE0101960E94FA64CE0178
:1080500001960E947BA0BE016F5F7F4FCE018A9682
:108060000E94C164CE0101960E94FA6462E370E04E
:1080700080E090E00E94C0690436110519F0FF20ED
:1080800009F460CF8091330C8823F1F06CEC78E038
:10809000CE014C960E949365BE016D5C7F4FCE0170
:1080A0004C960E941564BC01CE0101960E948A651F
:1080B000CE0101960E94BE09CE0101960E94FA648B
:1080C000CE014C960E94FA648FA998AD892B69F075
:1080D00070E060E0CE01C3960E94B363082E000CEE
:1080E000990BC0970A9708F477C066ED77E0CE0148
:1080F00001960E949365CE018A960E94FA64CE0191
:10810000C3960E94FA648D819E81009709F446C04F
:10811000E981FA812081222309F440C00797F0F118
:108120006EE379E0CE014C960E94816568EC70E0C8
:10813000CE014C960E9438A5CE014C960E94FA645E
:10814000BE016F5F7F4FCE014C960E948A6560ED45
:1081500077E0CE014C960E943672CE014C960E947A
:10816000FA6462EE77E0CE014C960E94936569E96D
:1081700073E1CE014C960E941564BC01CE018A9633
:108180000E948A65CE018A960E94BE09CE018A9617
:108190000E94FA64CE014C960E94FA64CE010196C8
:1081A0000E94FA64BDCB043111050CF44CCFC80118
:1081B000B5010E9443BA892B09F045CFBE016D5C21
:1081C0007F4F89E79FE00E94DC6668EC70E080E00A
:1081D00090E00E94C06937CF6EEC77E0CE01019647
:1081E0000E949365BE016F5F7F4FCE01C3960E94D0
:1081F000E463182FCE0101960E94FA64111175CF25
:10820000BE016D5C7F4FCE0101960E94786573CFF1
:1082100060EF77E0CE0101960E949365BE016F5F2B
:108220007F4FCE018F5B9F4F0E94E463182FCE01DA
:1082300001960E94FA64112309F4E8C025E030E0B9
:1082400044E050E069E973E1CE0101960E94A8651F
:10825000BE016F5F7F4F8BE793E10E94C164CE0147
:1082600001960E94FA6469E973E1CE0101960E94C9
:108270008A65CE0101960E94E10DCE0101960E9411
:10828000FA648BE793E10E944B636130710509F05A
:1082900067C070936115609360156FE378E0CE015D
:1082A00001960E948165CE0101960E94E10DCE01EA
:1082B00001960E94FA6465EF77E0CE014C960E9429
:1082C000936568EE75E1CE014C960E941564BC0181
:1082D000CE0101960E948A6548EC50E06FEF7FEF77
:1082E000CE0101960E946019CE0101960E94FA64A7
:1082F000CE014C960E94FA640E9440A140E052ECEC
:1083000061E070E089E79FE00E94455D84EF91E0C5
:108310009093DE028093DD0264EA74E10E94519240
:1083200064E078E0CE014C960E94936562EE75E1C0
:10833000CE014C960E941564BC01CE0101960E94AC
:108340008A6560ED77E0CE0101960E943672CE011B
:1083500001960E94FA64CE014C960E94FA64E0CA2B
:1083600061157105D1F5109261151092601561E3E8
:1083700078E0CE0101960E948165CE0101960E94AF
:10838000E10DCE0101960E94FA646BEF77E0CE0119
:108390004C960E94936568EE75E1CE014C960E9462
:1083A0001564BC01CE0101960E948A6548EC50E03C
:1083B0006FEF7FEFCE0101960E946019CE0101960A
:1083C0000E94FA64CE014C960E94FA640E9440A179
:1083D00040E855E260E070E095CF6230710509F049
:1083E0009FCA709361156093601560E278E0CE01DA
:1083F00001960E948165CE0101960E94E10DCE0199
:1084000001960E94FA646FEF77E0C1CF69E078E0EF
:10841000CE0101960E949365BE016F5F7F4FCE0132
:108420008F5B9F4F0E94E463182FCE0101960E943C
:10843000FA64112309F441C047E050E069E973E1AF
:10844000CE0101960E946D07BE016F5F7F4F8BE7E3
:1084500093E10E94C164CE0101960E94FA6464ED2A
:1084600077E0CE0101960E949365BE016F5F7F4F5A
:108470008BE793E10E94E463182FCE0101960E94DE
:10848000FA6411111092000D68ED74E0CE010196AE
:108490000E949365BE016F5F7F4F8BE793E10E945F
:1084A000E463182FCE0101960E94FA64112309F4A7
:1084B00004CD81E08093000D00CD61E178E0CE0134
:1084C00001960E949365BE016F5F7F4FCE018F5B67
:1084D0009F4F0E94E463182FCE0101960E94FA6418
:1084E000112381F146E050E069E973E1CE01019684
:1084F0000E946D07BE016F5F7F4F8BE793E10E9483
:10850000C164CE0101960E94FA648BE793E10E9458
:1085100040636093A8157093A9158093AA15909352
:10852000AB1584EF91E09093DE028093DD0264EA64
:1085300074E10E94519264E670E080E090E00E9455
:10854000C069BBCC68E178E0CE0101960E949365DA
:10855000BE016F5F7F4FCE018F5B9F4F0E94E46330
:10856000182FCE0101960E94FA64112301F148E010
:1085700050E069E973E1CE0101960E946D07BE01EA
:108580006F5F7F4F8BE793E10E94C164CE0101963C
:108590000E94FA648BE793E10E9440636093AE15FA
:1085A0007093AF158093B0159093B115BACF61E277
:1085B00078E0CE0101960E949365BE016F5F7F4F08
:1085C000CE018F5B9F4F0E94E463182FCE0101966E
:1085D0000E94FA64112301F149E050E069E973E176
:1085E000CE0101960E946D07BE016F5F7F4F8BE742
:1085F00093E10E94C164CE0101960E94FA648BE768
:1086000093E10E9440636093B2157093B315809319
:10861000B4159093B51585CF6BE278E0CE01019645
:108620000E949365BE016F5F7F4FCE018F5B9F4FAE
:108630000E94E463182FCE0101960E94FA64112370
:10864000F1F049E050E069E973E1CE0101960E9442
:108650006D07BE016F5F7F4F8BE793E10E94C1649E
:10866000CE0101960E94FA648BE793E10E94406379
:108670000E94F7B97093B9156093B81552CF65E3AE
:1086800078E0CE0101960E949365BE016F5F7F4F37
:10869000CE018F5B9F4F0E94E463182FCE0101969D
:1086A0000E94FA641123F1F04AE050E069E973E1B5
:1086B000CE0101960E946D07BE016F5F7F4F8BE771
:1086C00093E10E94C164CE0101960E94FA648BE797
:1086D00093E10E9440630E94F7B97093B7156093CD
:1086E000B6151FCF60E478E0CE0101960E94936535
:1086F000BE016F5F7F4FCE018F5B9F4F0E94E4638F
:10870000182FCE0101960E94FA64112311F14BE05B
:1087100050E069E973E1CE0101960E946D07BE0148
:108720006F5F7F4F8BE793E10E94C164CE0101969A
:108730000E94FA648BE793E10E9440630E94F7B9BC
:108740006093BA157093BB158093BC159093BD15BB
:10875000E8CE6CE478E0CE0101960E949365BE01FC
:108760006F5F7F4FCE018F5B9F4F0E94E463182F96
:10877000CE0101960E94FA641123E1F045E050E039
:1087800069E973E1CE0101960E946D07BE016F5F3A
:108790007F4F8BE793E10E94C164CE0101960E9456
:1087A000FA648BE793E10E944B637093AD1560937D
:1087B000AC15B7CE62E578E0CE0101960E949365D4
:1087C000BE016F5F7F4FCE018F5B9F4F0E94E463BE
:1087D000182FCE0101960E94FA64112309F45BC29E
:1087E0000E94A3726093880C7093890C80938A0C0A
:1087F00090938B0C26E030E045E050E069E973E1AE
:10880000CE0101960E94A865BE016F5F7F4F8BE786
:1088100093E10E94C164CE0101960E94FA648BE745
:1088200093E10E944B634B016B0181E08093A315A0
:108830008093010D0E94A37260939B0C70939C0C1B
:1088400080939D0C90939E0C8114910491F58091DE
:10885000BE159091BF15FC01EE0FFF1FED5AFD4FA5
:1088600011821082880F991F880F991FFC01E95C03
:10887000FD4F10821182128213828091C015909157
:10888000C115FC01EE0FFF1FED5AFD4F1182108242
:10889000880F991F880F991FFC01E95CFD4F10821A
:1088A00011821282138258E7E52EF12C04EB10E0BE
:1088B00029C1F1E08F16910409F06BC080919D13DE
:1088C00090919E130897C0F047E050E069E973E18A
:1088D000CE0101960E946D07CE0101960E94406371
:1088E0006093A8157093A9158093AA159093AB1562
:1088F000CE0101960E94FA648091BE159091BF1539
:10890000FC01EE0FFF1FED5AFD4F21E030E03183F7
:108910002083880F991F880F991FFC01E95BFD4F89
:1089200084E893E0A0E0B0E080839183A283B383E6
:108930000E94A372E091BE15F091BF15EE0FFF1FCC
:10894000EE0FFF1FE256FD4F608371838283938396
:108950008091C0159091C115FC01EE0FFF1FED5ADB
:10896000FD4F11821082880F991F880F991FFC01FB
:10897000E256FD4F1082118212821382895C9D4F54
:10898000DC011D921D921D921C921397F12CE12C7B
:108990008DCFB2E08B16910409F056C180919D13E2
:1089A00090919E130897C0F047E050E069E973E1A9
:1089B000CE0101960E946D07CE0101960E94406390
:1089C0006093AE157093AF158093B0159093B11569
:1089D000CE0101960E94FA644090AE155090AF15FA
:1089E0006090B0157090B115A30192016091B2151D
:1089F0007091B3158091B4159091B5150E946BB725
:108A000087FF10C020E030E040EA50E4C301B2012B
:108A10000E9419B96093B2157093B3158093B41581
:108A20009093B5158091AC159091AD15019797FD78
:108A300022C0880F991F880F991F8C01035E1C4F5D
:108A400020E030E040E251E46091A8157091A91552
:108A50008091AA159091AB150E9419B99B01AC01A8
:108A6000F80160817181828193810E942DBA10E0AA
:108A700000E0181614F004EB10E08091BE15909100
:108A8000BF15FC01EE0FFF1FED5AFD4F1182108242
:108A9000880F991F880F991FFC01E95CFD4F108218
:108AA0001182128213828091C0159091C115FC0130
:108AB000EE0FFF1FED5AFD4F21E030E031832083A0
:108AC000880F991F880F991FFC01E95BFD4F80EB10
:108AD00094E0A0E0B0E080839183A283B3830E94FE
:108AE000A372E091C015F091C115EE0FFF1FEE0FBC
:108AF000FF1FE256FD4F608371838283938338E7C3
:108B0000E32EF12C28E0821A910832E083169104BA
:108B100008F062C080914302909144028A35910529
:108B200014F410E000E08091BE159091BF15FC0197
:108B3000EE0FFF1FED5AFD4F11821082880F991F13
:108B4000880F991FFC01E95CFD4F1082118212828F
:108B500013828091C0159091C115FC01EE0FFF1F8B
:108B6000ED5AFD4F21E030E031832083880F991FBB
:108B7000880F991FFC01E95CFD4F4CE251E060E079
:108B800070E04083518362837383895B9D4F48E526
:108B900052E060E070E0DC014D935D936D937C9357
:108BA00013970E94A372E091C015F091C115EE0FCA
:108BB000FF1FEE0FFF1FE256FD4F6083718382831C
:108BC0009383B8E0CB16D10421F41092A315109230
:108BD000010D58E7E52EF12CC8010E940B08909377
:108BE000440280934302801B910B97FF03C0919531
:108BF0008195910903973CF0C8010E940B0890935E
:108C0000440280934302C7010E947F07909346026B
:108C1000809345028E199F0997FF03C09195819516
:108C2000910903973CF0C7010E947F079093460289
:108C30008093450268E578E0CE0101960E94936535
:108C400069E973E10C942D3CF3E08F16910409F06F
:108C50009DCE809143029091440204EB10E08A354E
:108C6000910514F410E000E08091BE159091BF15BD
:108C7000FC01EE0FFF1FED5AFD4F11821082880F8D
:108C8000991F880F991FFC01E95CFD4F108211822A
:108C90001282138234CF60E678E0CE0101960E9402
:108CA0009365BE016F5F7F4FCE018F5B9F4F0E9428
:108CB000E463182FCE0101960E94FA64112389F112
:108CC00043E050E0BE016F5B7F4FCE0101960E94F2
:108CD0006D07BE016F5F7F4F8BE793E10E94C16418
:108CE000CE0101960E94FA6480917F1390918013C7
:108CF000892B41F08BE793E10E944B6370935C02F8
:108D000060935B0280915B0290915C0201970297F5
:108D100008F4D3C881E090E090935C0280935B02FA
:108D2000CCC869E378E0CE014C960E949365BE0101
:108D3000645E7F4FCE018F5B9F4F0E94E46311E022
:108D4000811116C061EA78E0CE0101960E94936518
:108D5000BE016F5F7F4FCE018F5B9F4F0E94E46328
:108D600011E0811101C010E0CE0101960E94FA6469
:108D7000CE014C960E94FA64112309F46AC069E39B
:108D800078E0CE0101960E949365BE016F5F7F4F30
:108D9000CE018F5B9F4F0E94E463182FCE01019696
:108DA0000E94FA641123A1F046E050E0BE016F5B1F
:108DB0007F4FCE0101960E946D07BE016F5F7F4F0E
:108DC0008BE793E10E94C164CE0101960E94FA6490
:108DD00061EA78E0CE0101960E949365BE016F5F63
:108DE0007F4FCE018F5B9F4F0E94E463182FCE010F
:108DF00001960E94FA641123A1F042E050E0BE0106
:108E00006F5B7F4FCE0101960E946D07BE016F5FC1
:108E10007F4F8BE793E10E94C164CE0101960E94CF
:108E2000FA6480917F1390918013892B09F445C8CF
:108E30006BE773E1CE0101960E948A6561E070E004
:108E4000CE0101960E94681ACE0101960E94FA6432
:108E500034C86DE678E0CE018A960E949365BE0123
:108E6000665D7F4FCE018F5B9F4F0E94E46311E0F0
:108E700081112BC064E678E0CE014C960E94936588
:108E8000BE01645E7F4FCE018F5B9F4F0E94E46303
:108E900011E0811116C06CE678E0CE0101960E94C7
:108EA0009365BE016F5F7F4FCE018F5B9F4F0E9426
:108EB000E46311E0811101C010E0CE0101960E942F
:108EC000FA64CE014C960E94FA64CE018A960E9402
:108ED000FA64112309F4ECC06DE678E0CE01019646
:108EE0000E949365BE016F5F7F4FCE018F5B9F4FE6
:108EF0000E94E463182FCE0101960E94FA641123A8
:108F000009F467C046E050E0BE016F5B7F4FCE01C1
:108F100001960E946D07BE016F5F7F4F8BE793E163
:108F20000E94C164CE0101960E94FA648BE793E12E
:108F30000E9440636B017C0120E030E0A9010E94A7
:108F40002DBA18160CF091C0A701960160E070E0F0
:108F50008AE794E40E9485B90E94F7B960933002D1
:108F600070933102809332029093330280913002E9
:108F700090913102A0913202B09133021816190675
:108F80001A061B0664F081E090E0A0E0B0E0809358
:108F9000300290933102A0933202B0933302809159
:108FA0005B0290915C028130910509F06BC0809169
:108FB000300290913102A0913202B091330280933D
:108FC0002C0290932D02A0932E02B0932F020C94AA
:108FD0005D3F47E050E0BE016F5B7F4FCE010196E1
:108FE0000E946D07BE016F5F7F4F8BE793E10E9488
:108FF000C164CE0101960E94FA646BE175E0CE0176
:1090000001960E949365BE016F5F7F4FCE018F5B1B
:109010009F4F0E94E463182FCE0101960E94FA64CC
:10902000112331F081E090E090935C0280935B0229
:1090300062E777E0CE0101960E949365BE016F5F03
:109040007F4FCE018F5B9F4F0E94E463182FCE01AC
:1090500001960E94FA64112309F468CF82E090E03F
:1090600090935C0280935B0261CF81E090E0A0E08E
:10907000B0E08093300290933102A0933202B0931B
:10908000330274CF029711F00C945D3F809130024F
:1090900090913102A0913202B09133028093280264
:1090A00090932902A0932A02B0932B020C945D3F67
:1090B00064E778E0CE014C960E949365BE01645E41
:1090C0007F4FCE018F5B9F4F0E94C463FF24F394B8
:1090D000811117C069E778E0CE0101960E9493657F
:1090E000BE016F5F7F4FCE018F5B9F4F0E94E46395
:1090F000FF24F394811101C0F12CCE0101960E944E
:10910000FA64CE014C960E94FA648E01045E1F4FF1
:10911000FF2009F45CC164E778E0CE0101960E946B
:109120009365BE016F5F7F4FCE018F5B9F4F0E94A3
:10913000E463F82ECE0101960E94FA64F11036C065
:109140006BE175E0CE0101960E949365BE016F5FF1
:109150007F4FCE018F5B9F4F0E94E463F82ECE01BC
:1091600001960E94FA64FF2031F081E090E0909334
:109170005C0280935B0262E777E0CE0101960E9479
:109180009365BE016F5F7F4FCE018F5B9F4F0E9443
:10919000E463F82ECE0101960E94FA64FF2031F0BC
:1091A00082E090E090935C0280935B0281E090E02B
:1091B000A0E0B0E08093300290933102A09332029D
:1091C000B093330280915B0290915C0281309105F3
:1091D00009F07AC09093AB028093AA0260E878E02D
:1091E0008BE793E10E94CE6269E778E0CE010196B9
:1091F0000E949365BE016F5F7F4FCE018F5B9F4FD3
:109200000E94E463F82ECE0101960E94FA64FF20CA
:10921000F9F046E050E0BE016F5B7F4FC8010E944D
:109220006D0762E176E0CE0101960E949365B80178
:10923000CE0101960E941564BC018BE793E10E9468
:10924000AA64CE0101960E94FA64C8010E94FA64E1
:109250008091300290913102A0913202B09133029C
:1092600080932C0290932D02A0932E02B0932F0294
:109270006DE279E0CE0101960E948165CE010196F2
:109280000E94BE09CE0101960E94FA646BE773E169
:10929000CE0101960E948A6562E070E0CE010196DF
:1092A0000E94681ACE0101960E94FA646DE179E08D
:1092B000CE0101960E948165CE0101960E94351A69
:1092C000CE0101960E94FA64E0905B02F0905C028D
:1092D000E2E0EE16F10409F064C064ED77E08BE79C
:1092E00093E10E94CE626CE079E0CE0101960E948B
:1092F0008165CE0101960E94BE09CE0101960E94B1
:10930000FA646BE773E1CE0101960E948A6563E01F
:1093100070E0CE0101960E94681ACE0101960E946B
:10932000FA64F0925C02E0925B028091CA1590911F
:10933000CB159093AB028093AA0260E079E0CE0156
:1093400001960E948165CE0101960E94351ACE01D8
:1093500001960E94FA648091CA159091CB1591955F
:10936000819591099093CB158093CA15EE24E394CF
:10937000F12CF092AB02E092AA0284EF91E090937C
:10938000DE028093DD0264EA74E10E94519264E699
:1093900070E080E090E00E94C069F0925C02E09290
:1093A0005B026CEC78E0CE0101960E94936569E95E
:1093B00073E1CE0101960E941564BC01C8010E94B0
:1093C0008A65C8010E94BE09C8010C943C3C64E84F
:1093D00078E0CE01C3960E949365BE016D5C7F4F1D
:1093E000CE018F5B9F4F0E94E463EE24E3948111D2
:1093F00042C061ED78E0CE018A960E949365BE017D
:10940000665D7F4FCE018F5B9F4F0E94E463EE2429
:10941000E39481112CC060ED78E0CE014C960E945F
:109420009365BE01645E7F4FCE018F5B9F4F0E94AC
:10943000E463EE24E394811117C06BE878E0CE0179
:1094400001960E949365BE016F5F7F4FCE018F5BD7
:109450009F4F0E94E463EE24E394811101C0E12C4C
:10946000CE0101960E94FA64C8010E94FA64CE01FE
:109470008A960E94FA64CE01C3960E94FA64EE2096
:1094800009F468C164E878E0CE0101960E94936512
:10949000BE016F5F7F4FCE018F5B9F4F0E94E463E1
:1094A000E82ECE0101960E94FA6446E050E0E110F9
:1094B00018C061ED78E0CE0101960E949365BE016F
:1094C0006F5F7F4FCE018F5B9F4F0E94E463E82E5A
:1094D000CE0101960E94FA64EE2009F463C042E0D6
:1094E00050E0BE016F5B7F4FCE0101960E946D0779
:1094F000BE016F5F7F4F8BE793E10E94C164CE0195
:1095000001960E94FA6480917F1390918013892BB9
:1095100009F447CF62E176E0C8010E949365B80183
:109520008BE793E10E94E463811115C06BE87AE058
:10953000CE0101960E949365BE016F5F7F4F8BE75E
:1095400093E10E94E463FF24F3948111F12CCE0196
:1095500001960E94FA64C8010E94FA64FF2009F48F
:10956000E0C08BE793E10E94406320916A0C309148
:109570006B0C40916C0C50916D0C0E9419B96B01F1
:109580007C0120E030E044EB53E40E942DBA87FDDB
:1095900055C020E030E044EB53E4C701B6010E941F
:1095A00018B9EDCF43E050E0BE016F5B7F4FCE01B5
:1095B00001960E946D07BE016F5F7F4F8BE793E1BD
:1095C0000E94C164CE0101960E94FA646BE175E0CD
:1095D000CE0101960E949365BE016F5F7F4FCE0161
:1095E0008F5B9F4F0E94E463E82ECE0101960E949C
:1095F000FA64EE2031F081E090E090935C02809379
:109600005B0262E777E0CE0101960E949365BE019E
:109610006F5F7F4FCE018F5B9F4F0E94E463E82E08
:10962000CE0101960E94FA64EE2009F46CCF82E02C
:1096300090E090935C0280935B0265CF20E030E085
:10964000A901C701B6010E946BB787FF0BC020E0DC
:1096500030E044EB53E4C701B6010E9419B96B0135
:109660007C01ECCFC0926A0CD0926B0CE0926C0C37
:10967000F0926D0C8BE793E10E94406320E030E0B4
:10968000A9010E942DBA87FD15C06BE87AE0CE01D2
:1096900001960E9493656BE773E1CE0101960E94EB
:1096A0001564BC018BE793E10E94AA64CE01019688
:1096B0000E94FA648BE793E10E94406320E030E06F
:1096C000A9010E946BB787FF2CC08BE793E10E9432
:1096D000406320E030E0A9010E942DBA181694F5ED
:1096E0008BE793E10E944063AB01BC0122E0C8011B
:1096F0000E94026562E176E0CE0101960E949365C8
:10970000B801CE0101960E941564BC018BE793E17C
:109710000E94AA64CE0101960E94FA64C8010E94C8
:10972000FA646BE773E1CE0101960E948A6562E0FC
:1097300070E0CE0101960E94681ACE0101960E9447
:10974000FA642FCE8BE793E10E944063AB01BC012A
:109750007058CCCF60E978E0CE018A960E9493657C
:10976000BE01665D7F4FCE018F5B9F4F0E94E46319
:10977000FF24F394811129C06FE878E0C8010E94AA
:109780009365B801CE018F5B9F4F0E94E463FF2475
:10979000F394811117C066E978E0CE0101960E942A
:1097A0009365BE016F5F7F4FCE018F5B9F4F0E941D
:1097B000E463FF24F394811101C0F12CCE010196E2
:1097C0000E94FA64C8010E94FA64CE018A960E943F
:1097D000FA64FF2009F48AC0CE018F5B9F4F0E947C
:1097E000566360E978E0CE0101960E949365BE0160
:1097F0006F5F7F4FCE018F5B9F4F0E94E463F82E17
:10980000CE0101960E94FA64FF2021F145E050E06C
:10981000BE016F5B7F4FCE0101960E946D07BE01B6
:109820006F5F7F4F8BE793E10E94C164CE01019689
:109830000E94FA6480917F1390918013892B09F420
:10984000B0CD6BE773E1CE0101960E948A6563E0BB
:1098500070E06FCF46E050E0BE016F5B7F4FCE01FE
:1098600001960E946D07BE016F5F7F4F8BE793E10A
:109870000E94C164CE0101960E94FA646BE175E01A
:10988000CE0101960E949365BE016F5F7F4FCE01AE
:109890008F5B9F4F0E94E463F82ECE0101960E94D9
:1098A000FA64FF2031F081E090E090935C028093B5
:1098B0005B0262E777E0CE0101960E949365BE01EC
:1098C0006F5F7F4FCE018F5B9F4F0E94E463F82E46
:1098D000CE0101960E94FA64FF2009F4ABCF82E02A
:1098E00090E090935C0280935B02A4CF6EE978E0F5
:1098F000CE018A960E949365BE01665D7F4FCE01C0
:109900008F5B9F4F0E94E463FF24F394811129C071
:109910006DE978E0C8010E949365B801CE018F5BC4
:109920009F4F0E94E463FF24F394811117C064EAFF
:1099300078E0CE0101960E949365BE016F5F7F4F74
:10994000CE018F5B9F4F0E94E463FF24F39481114B
:1099500001C0F12CCE0101960E94FA64C8010E9458
:10996000FA64CE018A960E94FA64FF2009F424C1A9
:109970006EE978E0CE0101960E949365BE016F5FAB
:109980007F4FCE018F5B9F4F0E94E463F82ECE0184
:1099900001960E94FA64FF2009F443C045E050E0BC
:1099A000BE016F5B7F4FCE0101960E946D07BE0125
:1099B0006F5F7F4F8BE793E10E94C164CE010196F8
:1099C0000E94FA6480917F1390918013892B61F03B
:1099D0008BE793E10E94406360936A0C70936B0C79
:1099E00080936C0C90936D0CC0906A0CD0906B0CB3
:1099F000E0906C0CF0906D0C20E030E044EB53E410
:109A0000C701B6010E942DBA87FD57C020E030E0A3
:109A100044EB53E4C701B6010E9418B96B017C0105
:109A2000EBCF46E050E0BE016F5B7F4FCE01019669
:109A30000E946D07BE016F5F7F4F8BE793E10E942D
:109A4000C164CE0101960E94FA646BE175E0CE011B
:109A500001960E949365BE016F5F7F4FCE018F5BC1
:109A60009F4F0E94E463F82ECE0101960E94FA6493
:109A7000FF2031F081E090E090935C0280935B02E4
:109A800062E777E0CE0101960E949365BE016F5FA9
:109A90007F4FCE018F5B9F4F0E94E463F82ECE0173
:109AA00001960E94FA64FF2009F48CCF82E090E0D6
:109AB00090935C0280935B0285CF20E030E0A901A7
:109AC000C701B6010E946BB787FF0BC020E030E0F2
:109AD00044EB53E4C701B6010E9419B96B017C0144
:109AE000ECCFC0926A0CD0926B0CE0926C0CF092AE
:109AF0006D0C80915B0290915C02019771F4C092B1
:109B0000930CD092940CE092950CF092960C63E03A
:109B100075E081E893E10E94CE6280916A0C909199
:109B20006B0CA0916C0CB0916D0C20915B0230918C
:109B30005C022230310571F480938F0C9093900C6D
:109B4000A093910CB093920C62E175E081E893E1EF
:109B50000E94CE6240916A0C50916B0C60916C0C2B
:109B600070916D0C21E0C8010E94026561E873E10B
:109B7000CE0101960E948A65B801CE0101960E942D
:109B800015646DE075E00E94FF63BC0181E893E11C
:109B90000E94AA64CE0101960E94FA64C8010E9444
:109BA000FA6461E873E1CE0101960E948A65CE01F4
:109BB00001960E94351AC1CD6CEA78E0CE018A96F2
:109BC0000E949365BE01665D7F4FCE018F5B9F4F04
:109BD0000E94E463FF24F394811129C06BEA78E0CA
:109BE000C8010E949365B801CE018F5B9F4F0E9410
:109BF000E463FF24F394811117C061EB78E0CE0198
:109C000001960E949365BE016F5F7F4FCE018F5B0F
:109C10009F4F0E94E463FF24F394811101C0F12C53
:109C2000CE0101960E94FA64C8010E94FA64CE0136
:109C30008A960E94FA64FF2009F410C2C090300294
:109C4000D0903102E0903202F090330267EB78E07E
:109C5000CE0101960E949365BE016F5F7F4FCE01DA
:109C60008F5B9F4F0E94E463B82ECE0101960E9445
:109C7000FA64BB2009F464C044E050E0BE016F5BAD
:109C80007F4FCE0101960E946D07BE016F5F7F4F2F
:109C90008BE793E10E94C164CE0101960E94FA64B1
:109CA00080915B0290915C028130910509F094C033
:109CB000C0902C02D0902D02E0902E02F0902F0246
:109CC00081E090E0A0E0B0E080932C0290932D0220
:109CD000A0932E02B0932F0280917F139091801356
:109CE000892B09F091C06CEB78E08BE793E10E943F
:109CF000CE6280917F1390918013892B81F06BE766
:109D000073E1CE0101960E948A6570E060E0CE01A9
:109D100001960E94681ACE0101960E94FA64809111
:109D20005B0290915C028130910509F08BC1C09279
:109D30002C02D0922D02E0922E02F0922F0231CB13
:109D400045E050E0BE016F5B7F4FCE0101960E945F
:109D50006D07BE016F5F7F4F8BE793E10E94C16487
:109D6000CE0101960E94FA646BE175E0CE01019686
:109D70000E949365BE016F5F7F4FCE018F5B9F4F47
:109D80000E94E463B82ECE0101960E94FA64BB20C3
:109D900031F081E090E090935C0280935B0262E797
:109DA00077E0CE0101960E949365BE016F5F7F4F01
:109DB000CE018F5B9F4F0E94E463B82ECE010196C7
:109DC0000E94FA64BB2009F46BCF82E090E090938C
:109DD0005C0280935B0264CF029709F07DCFC09054
:109DE0002802D0902902E0902A02F0902B0281E014
:109DF00090E0A0E0B0E08093280290932902A09325
:109E00002A02B0932B0268CF62EC78E0CE01019673
:109E10000E949365BE016F5F7F4F8BE793E10E94C5
:109E2000C463B82ECE0101960E94FA64BB2009F4E7
:109E300076CF8BE793E10E94406320E030E0A901F8
:109E40000E946BB7811128C080915B0290915C02E7
:109E5000019731F465EC78E08BE793E10E94CE62E4
:109E600080915B0290915C02029731F46CEB78E098
:109E70008BE793E10E94CE6280917F1390918013D3
:109E8000892B09F44CCF6BE773E1CE0101960E9458
:109E90008A6561E070E03BCF61E277E0CE01019638
:109EA0000E949365BE016F5F7F4F8BE793E10E9435
:109EB000C463B82ECE0101960E94FA64BB2009F457
:109EC0002ECF41E050E06BE773E1CE0101960E9496
:109ED0006D07CE0101960E9440632B013C01CE012B
:109EE00001960E94FA6420E030E0A901C301B201AA
:109EF0000E946BB7181634F0412C512C30E8632EB9
:109F00003FE3732EA0905B02B0905C02F1E0AF16CD
:109F1000B10409F071C0A301920160E070E48CE922
:109F200095E40E9485B96093240270932502809382
:109F30002602909327026093C2157093C3158093F5
:109F4000C4159093C51560932002709321028093ED
:109F5000220290932302B501C8010E94D8626AECE4
:109F600078E0CE0101960E949365B801CE0101967A
:109F70000E941564BC01CE018A960E948A65CE01BA
:109F80008A960E94D509CE018A960E94FA64CE0173
:109F900001960E94FA64C8010E94FA646EEE78E0AD
:109FA000CE0101960E948165CE0101960E94D509DD
:109FB000CE0101960E94FA6440912402509125023C
:109FC000609126027091270225E0CE0101960E9441
:109FD0000265CE0101960E94BE09CE0101960E9443
:109FE000FA6484EF91E09093DE028093DD0264EAEC
:109FF00074E10E94519293CE22E0A216B10409F0BE
:10A00000AACFA301920160E070E48CE196E40E9483
:10A0100085B9609324027093250280932602909361
:10A0200027026093C6157093C7158093C815909347
:10A03000C91560931C0270931D0280931E029093B9
:10A040001F0289CF029709F0ACC9C0922802D092B2
:10A050002902E0922A02F0922B02A3C96FEC78E069
:10A06000CE018A960E949365BE01665D7F4FCE0148
:10A070008F5B9F4F0E94E463FF24F394811129C0FA
:10A080006EEC78E0C8010E949365B801CE018F5B49
:10A090009F4F0E94E463FF24F394811117C064ED85
:10A0A00078E0CE0101960E949365BE016F5F7F4FFD
:10A0B000CE018F5B9F4F0E94E463FF24F3948111D4
:10A0C00001C0F12CCE0101960E94FA64C8010E94E1
:10A0D000FA64CE018A960E94FA64FF2009F427C12F
:10A0E00027968EAD9FAD2797059708F45AC944E08F
:10A0F00050E0BE016F5B7F4FCE0101960E946D075D
:10A10000BE016F5F7F4F8BE793E10E94C164CE0178
:10A1100001960E94FA646FEC78E0CE0101960E94ED
:10A120009365BE016F5F7F4FCE018F5B9F4F0E9493
:10A13000E463F82ECE0101960E94FA64FF2009F430
:10A1400095C044E050E0BE016F5B7F4FCE010196A9
:10A150000E946D07BE016F5F7F4F8BE793E10E9406
:10A16000C164CE0101960E94FA648BE793E10E94DC
:10A17000406320E030E0A9010E942DBA18160CF0CF
:10A1800010C98BE793E10E944063609324027093AF
:10A190002502809326029093270220915B02309142
:10A1A0005C022130310509F0ADC06093C215709397
:10A1B000C3158093C4159093C515609320027093C6
:10A1C00021028093220290932302B901C8010E94C8
:10A1D000D8626AEC78E0CE0101960E949365B801DE
:10A1E000CE0101960E941564BC01CE018A960E94A0
:10A1F0008A65CE018A960E94D509CE018A960E9470
:10A20000FA64CE0101960E94FA64C8010E94FA64C1
:10A210006CED78E0CE0101960E948165CE01019639
:10A220000E94D509CE0101960E94FA644091240251
:10A2300050912502609126027091270225E0CE01FF
:10A2400001960E940265CE0101960E94BE09CE01D0
:10A2500001960E94FA6484EF91E09093DE0280936D
:10A26000DD0264EA74E10E9451929BC845E050E02F
:10A27000BE016F5B7F4FCE0101960E946D07BE014C
:10A280006F5F7F4F8BE793E10E94C164CE0101961F
:10A290000E94FA646BE175E0CE0101960E9493651D
:10A2A000BE016F5F7F4FCE018F5B9F4F0E94E463C3
:10A2B000F82ECE0101960E94FA64FF2031F081E071
:10A2C00090E090935C0280935B0262E777E0CE01BE
:10A2D00001960E949365BE016F5F7F4FCE018F5B39
:10A2E0009F4F0E94E463F82ECE0101960E94FA640B
:10A2F000FF2009F43ACF82E090E090935C028093D3
:10A300005B0233CF2230310509F05FCF6093C61571
:10A310007093C7158093C8159093C91560931C025C
:10A3200070931D0280931E0290931F024ECF6CEA21
:10A3300076E0C8010E949365B801CE018F5B9F4F04
:10A340000E94E463FF24F394811117C06AED78E062
:10A35000CE0101960E949365BE016F5F7F4FCE01D3
:10A360008F5B9F4F0E94E463FF24F394811101C02F
:10A37000F12CCE0101960E94FA64C8010E94FA6491
:10A38000FF2009F46BC06CEA76E0CE0101960E94D2
:10A390009365BE016F5F7F4FCE018F5B9F4F0E9421
:10A3A000E463F82ECE0101960E94FA64FF2099F032
:10A3B00042E050E069E973E1CE0101960E946D0729
:10A3C000BE016F5F7F4F8BE793E10E94C164CE01B6
:10A3D00001960E94FA646AED78E0CE0101960E942F
:10A3E0009365BE016F5F7F4FCE018F5B9F4F0E94D1
:10A3F000E463F82ECE0101960E94FA64FF2099F0E2
:10A4000043E050E069E973E1CE0101960E946D07D7
:10A41000BE016F5F7F4F8BE793E10E94C164CE0165
:10A4200001960E94FA648BE793E10E944B63653BBF
:10A43000710548F4CB010E940B089093440280936D
:10A4400043020C94D14969EC78E0CE0101960E9458
:10A450008165CE0101960E94D5096FC96EED78E045
:10A46000CE0101960E949365BE016F5F7F4FCE01C2
:10A470008F5B9F4F0E94E463F82ECE0101960E94ED
:10A48000FA64FF2009F4F2C226E030E044E050E034
:10A4900069E973E1CE0101960E94A865BE016F5F74
:10A4A0007F4F8BE793E10E94C164CE0101960E9429
:10A4B000FA648BE793E10E944B636B011B0161E23D
:10A4C00077E0CE0101960E94936540919D135091D3
:10A4D0009E138D819E81481B590BBE016F5F7F4F7C
:10A4E00089E993E10E945DA1AC014F5F5F4F69E98B
:10A4F00073E1C8010E946D07B8018BE793E10E94E8
:10A50000C164C8010E94FA64CE0101960E94FA64F7
:10A510008BE793E10E9440634B015C01A60141502F
:10A5200051092D965FAF4EAF2D978091330C882344
:10A53000C1F168E478E0CE0101960E948165CE0108
:10A5400001960E94D509CE0101960E94FA64B601D7
:10A55000CE0101960E94D862CE0101960E94D509D3
:10A56000CE0101960E94FA646EE177E0CE01019679
:10A570000E949365CE0101960E94D509CE010196F5
:10A580000E94FA6422E0B501A401CE0101960E9466
:10A590000265CE0101960E94BE09CE0101960E947D
:10A5A000FA6460E088E30E948F69E2EBFBE0E491EB
:10A5B000EC8FE8EFFBE0E491F0E0EE0FFF1FE454D6
:10A5C000F64F859194919E8F8D8F1FA219A618A684
:10A5D00018870F831D821E82198289E08A8381E099
:10A5E0008B838C831C8A1B8A1EA21DA21CA21BA209
:10A5F0001AA219A218A21F8E11E0BE01665D7F4F3C
:10A600008F8198850E9486A3882309F45BC067E048
:10A61000CE018A960E94C0A299A98913EECF8981A2
:10A6200081111DC08F8198850E944EA3BE01665D79
:10A630007F4F8F8198850E940BA340E064EB8F8150
:10A6400098850E94D7A28F8198850E942AA3082FFF
:10A650008F8198850E944EA3011101C019830A8140
:10A660008AA5803109F420C5BE01665D7F4FCE0109
:10A6700001960E94A2A4801790F48A818A838D811A
:10A680008F5F8D838AA5883231F0B0F4803119F064
:10A69000823209F0B2CF8E818F5F8E83AECF8AA5D2
:10A6A000803111F48CE0EACFBE01665D7F4FCE01B0
:10A6B00001960E94A2A4E2CF8B3369F3823409F0A1
:10A6C0009CCFE9CF8F8198850E944EA340E06CEC2F
:10A6D0008F8198850E94D7A2498164E48F819885F3
:10A6E0000E94D7A28B818823C9F1EA81E9500EEE3E
:10A6F00012E0E33038F4F0E0EE0FFF1FE95EFC4FAC
:10A70000008111818C81882309F470C089818111B5
:10A710006DC00E948F6C2B013C01C801110FAA0B68
:10A72000BB0B61968CAF9DAFAEAFBFAF61978F8112
:10A7300098850E942AA3813089F00E948F6C6196CF
:10A740002CAD3DAD4EAD5FAD6197621B730B840BBD
:10A75000950B641575058605970548F38CE08A838B
:10A7600010E000E0AFE74A2EBFE15B2E8FE3682EDA
:10A770008D818017110609F00CF49FC0402FBE0197
:10A780006D5C7F4FCE0101960E9406A47A803CE06A
:10A79000371598F5FCE07F2E8BA98031A1F1BE0121
:10A7A0006D5C7F4FCE0101960E94A2A4871509F42B
:10A7B0007CC0AE01465D5F4FBE016D5C7F4FCE0138
:10A7C00001960E9442A4882309F46FC08BA98031AE
:10A7D00009F46BC05BE0751609F46AC08CE078166A
:10A7E000A1F09AE0791267C06EA610C0B801110FEF
:10A7F000880B990B0E94C069B1CF49E0741660F6CE
:10A80000E9E07E2EC9CF8CE0D1CF4EA68F8198850E
:10A810000E944EA3BE016D5C7F4F8F8198850E9480
:10A820000BA340E06EE48F8198850E94D7A240E0A0
:10A830006CA58F8198850E94D7A240E06DA58F817D
:10A8400098850E94D7A28BA9803131F040E06EA597
:10A850008F8198850E94D7A28F8198850E944EA3F0
:10A86000BE016D5C7F4F8F8198850E940BA349814B
:10A8700068E48F8198850E94D7A264E170E080E04F
:10A8800090E00E94C0698981882331F06AE070E01D
:10A8900080E090E00E94C0698F8198850E944EA35D
:10A8A0008A81871508F4872D8A830F5F1F4F60CF39
:10A8B000AFE5AEA7ABCF5EA6A9CF0E8110E00B30FF
:10A8C000110514F00AE010E0BBE5CB16D10408F442
:10A8D0004AC072E4C72E7CE0D72E5601412C512C81
:10A8E0003201F12CE12C0E151F05B9F06E2DCE01B1
:10A8F00001960E94CCA49B01AC01F50121933193F8
:10A90000419351935F01C301B2010E9419B92B0118
:10A910003C01FFEFEF1AFF0AE6CFB7010F2C000C46
:10A92000880B990B0E9472B79B01AC01C301B20165
:10A930000E9485B94B015C0110E000E0E016F106D1
:10A94000E9F1D6012D913D914D915C91C501B40184
:10A950000E9418B9F60161937193819391936F01ED
:10A960000F5F1F4FEBCF121413040CF05FC00215E2
:10A9700013053CF49801215031092D963FAF2EAFBD
:10A980002D972C966FAD2C97CE0101960E94CCA4EA
:10A990009B01AC012D960EAD1FAD2D97000F111F21
:10A9A000000F111F0E5B134FC501B4010E9418B9AF
:10A9B000D8016D937D938D939C93139788E2E2E485
:10A9C000FCE0ABE7B5E101900D928A95E1F784EFE9
:10A9D00091E09093DE028093DD0264EA74E10E94CC
:10A9E000519268EA78E081E893E10E94856444E04E
:10A9F00050E069E973E1CE0101960E946D07BE0146
:10AA00006F5F7F4F81E893E10E947E64CE010196E3
:10AA10000E94FA6461E873E1CE0101960E948A65A2
:10AA2000CE0101960E94BE090C94CE40211431043F
:10AA300029F622E4E22E2CE0F22E0215130509F489
:10AA4000BDCF622DCE0101960E94CCA49B01AC012A
:10AA5000C501B4010E9418B9F70161937193819304
:10AA600091937F01FFEF2F1A3F0AE7CF62EE78E064
:10AA7000CE0101960E949365BE016F5F7F4FCE01AC
:10AA80008F5B9F4F0E94E463F82ECE0101960E94D7
:10AA9000FA64FF2009F443C047E050E069E973E13C
:10AAA000CE0101960E946D07BE016F5F7F4F8BE75D
:10AAB00093E10E94C164CE0101960E94FA6464EDA4
:10AAC00077E0CE0101960E949365BE016F5F7F4FD4
:10AAD0008BE793E10E94E463F82ECE0101960E9479
:10AAE000FA64F1101092000D68ED74E0CE01019649
:10AAF0000E949365BE016F5F7F4F8BE793E10E94D9
:10AB0000E463F82ECE0101960E94FA64FF2011F44E
:10AB10000C94D14981E08093000D0C94D1496AEEE8
:10AB200078E0CE0101960E949365BE016F5F7F4F72
:10AB3000CE018F5B9F4F0E94E463F82ECE010196F9
:10AB40000E94FA64FF2071F141E069E672E0CE01F3
:10AB500001960E941373BE016F5F7F4F80E096E104
:10AB60000E94670C80E096E10E942B86811104C050
:10AB70006CE578E00C94ED3A80E096E10E94737603
:10AB8000892B51F080E096E10E94A081682F80E53A
:10AB900091E10E94A65AF0CF80E096E10E943786AC
:10ABA0000C94C53361EF78E0CE0101960E94936565
:10ABB000BE016F5F7F4FCE018F5B9F4F0E94E463AA
:10ABC000F82ECE0101960E94FA64FF20E9F02DB71D
:10ABD0003EB72A5231400FB6F8943EBF0FBE2DBF8C
:10ABE000ADB7BEB711968AE291E0E4EAF4E10190D4
:10ABF0000D920197E1F70E9436160FB6F894DEBF6A
:10AC00000FBECDBF0C94C5336AEF78E0CE0101963C
:10AC10000E949365BE016F5F7F4FCE018F5B9F4F98
:10AC20000E94E463F82ECE0101960E94FA64FF2090
:10AC300009F459C08DB79EB78A5291400FB6F89467
:10AC40009EBF0FBE8DBFADB7BEB711968AE291E031
:10AC5000E4EAF4E101900D920197E1F70E94F3120A
:10AC60000FB6F894DEBF0FBECDBF67E978E0CE0126
:10AC700001960E948165EDB7FEB7EA52F1400FB62A
:10AC8000F894FEBF0FBEEDBFADB7BEB711968AE216
:10AC900091E0E4EAF4E101900D920197E1F70E945E
:10ACA000CD100FB6F894DEBF0FBECDBF4DB75EB767
:10ACB0004A5251400FB6F8945EBF0FBE4DBFADB7BC
:10ACC000BEB711968AE291E0E4EAF4E101900D92B8
:10ACD0000197E1F70E9436160FB6F894DEBF0FBE5B
:10ACE000CDBF0C94CB366CEF78E0CE0101960E947C
:10ACF0009365BE016F5F7F4FCE018F5B9F4F0E94B8
:10AD0000E463F82ECE0101960E94FA64FF20E1F080
:10AD100065E878E0CE0101960E948165BE016F5F13
:10AD20007F4FC8010E948A65C8010E94BE09C80100
:10AD30000E94FA64ADB7BEB7AA52B1400FB6F894FC
:10AD4000BEBF0FBEADBFBDCF60E079E0CE010196C2
:10AD50000E949365BE016F5F7F4FCE018F5B9F4F57
:10AD60000E94E463F82ECE0101960E94FA64FF204F
:10AD700009F4ECC069E678E0CE018A960E9481650C
:10AD8000BE01665D7F4FCE0101960E948A65AE01CD
:10AD90004F5F5F4F62E070E089EB92E00E94961493
:10ADA000F82ECE0101960E94FA64F1101FC0BE0178
:10ADB000665D7F4FC8010E948A6564E079E0C80142
:10ADC0000E94FF636CEC73E10E941564BC01CE012C
:10ADD00001960E948A65CE0101960E94BE09CE01AD
:10ADE00001960E94FA64C8010E94FA6468EE73E05A
:10ADF00080E090E00E94C069BE01665D7F4FCE0199
:10AE000001960E948A65AE014F5F5F4F63E070E07C
:10AE10008CEA92E00E949614F82ECE0101960E94D0
:10AE2000FA64F1101FC0BE01665D7F4FC8010E9429
:10AE30008A6564E176E0C8010E94FF636CEC73E10F
:10AE40000E941564BC01CE0101960E948A65CE0164
:10AE500001960E94BE09CE0101960E94FA64C801C3
:10AE60000E94FA6468EE73E080E090E00E94C0699E
:10AE700060EC73E1CE0101960E948A65AE014F5FDE
:10AE80005F4F61E070E083E892E00E949614F82E34
:10AE9000CE0101960E94FA64F1101EC060EC73E1CD
:10AEA000C8010E948A6564E176E0C8010E94FF63E0
:10AEB0006CEC73E10E941564BC01CE0101960E9406
:10AEC0008A65CE0101960E94BE09CE0101960E94BC
:10AED000FA64C8010E94FA6468EE73E080E090E0D2
:10AEE0000E94C0698091000D882311F40C944E3E9D
:10AEF00043E163E872E0CE0101960E941373BE0144
:10AF00006F5F7F4F86E396E10E94670C86E396E1D0
:10AF10000E942B86882311F40C944E3E60EC73E162
:10AF200086E396E10E94EA6666E970E080E090E0E0
:10AF30000E94C06986E396E10E94378662E370E072
:10AF400080E090E00E94C0690C944E3E64E179E09C
:10AF5000CE0101960E949365BE016F5F7F4FCE01C7
:10AF60008F5B9F4F0E94E463182FCE0101960E94D1
:10AF7000FA64112301F194E3E92E9CE0F92E01E03B
:10AF800010E0F2E0EF0EF11C8091590290915A020C
:10AF90008017910714F40C94C53360E0D7018C91AD
:10AFA0000E94A7686CE271E080E090E00E94C069B6
:10AFB0000F5F1F4FE6CF68E179E0CE0101960E9456
:10AFC0009365BE016F5F7F4FCE018F5B9F4F0E94E5
:10AFD000E463182FCE0101960E94FA64112301F157
:10AFE00084E3E82E8CE0F82E01E010E0B2E0EB0EF6
:10AFF000F11C8091590290915A028017910714F424
:10B000000C94C53361E0F70180810E94A7686CE26F
:10B0100071E080E090E00E94C0690F5F1F4FE6CFB3
:10B020006DE179E0CE0101960E949365BE016F5FEC
:10B030007F4FCE018F5B9F4F0E94E463182FCE019C
:10B0400001960E94FA64112311F40C94C53327E091
:10B0500030E046E050E069E973E1CE0101960E94DC
:10B06000A865BE016F5F7F4F8BE793E10E94C164CB
:10B07000CE0101960E94FA648BE793E10E944B6334
:10B08000672B71F41092330C69E973E1CE010196DC
:10B090000E948A65CE0101960E94E10D0C94CE407B
:10B0A00081E08093330CF0CF0D3008F0E6CAFACA85
:10B0B0002F923F924F925F926F927F928F929F92C8
:10B0C000AF92BF92CF92DF92EF92FF920F931F93B6
:10B0D000CF93DF93CDB7DEB7C258D1090FB6F8943E
:10B0E000DEBF0FBECDBF6C015B0188EE482E83E052
:10B0F000582E612C712C02E014E09BE5892E912CD6
:10B100008C0E9D1E8CE0880E911C1B019FEF291A4E
:10B11000390AD6015996ED90FC90F701858182306D
:10B1200008F493C082859385A485B5858F7199278E
:10B13000AA27BB27892B8A2B8B2B09F086C040E2DC
:10B1400050E0BE016F5F7F4FC7010E948280803256
:10B1500009F07BC08981882309F477C0853E79F3A3
:10B160008E3269F38C8583FDEACF22961FAE1EAE28
:10B17000229780E893E09FAF8EAF24961FAE24976E
:10B18000BE016F5F7F4FE0E080E04EE2DB019D910A
:10B19000BD019032A1F0883049F426E730E02C0F51
:10B1A0003D1F2E0F311DD9014C93EF5F26E730E094
:10B1B0002C0F3D1F2E0F311DD9019C93EF5F8F5F28
:10B1C0008B3021F786E790E08C0F9D1F8E0F911D2D
:10B1D000FC011082D60159966D917C9121E0AE015F
:10B1E0004A585F4FCE01CE960E941182882369F1A2
:10B1F000BE01625C7F4FCE0181960E94DB85AE016D
:10B200004A585F4FBE016F5D7F4FCE01855A9F4FF9
:10B210000E944986CE01855A9F4F0E942B86882323
:10B2200009F4ACC0F12CFA141B042CF569E0CE0132
:10B2300001960E945F65CE0101960E94D509CE015C
:10B2400001960E94FA64F394EECF6F961FAE1EAE85
:10B250006F97A3964CAE5DAE6EAE7FAEA3976D9624
:10B260001FAF0EAF6D97E6961FAE1EAEE697A8967F
:10B270001FAEA897CFCFB401CE0101960E9493656F
:10B28000CE0101960E94D509CE0101960E94FA6472
:10B29000E696EEADFFADE697309709F447C085819D
:10B2A000823008F443C06CE774E0CE0101960E943E
:10B2B0009365CE0101960E94BE09CE0101960E94BF
:10B2C000FA646F968EAD9FAD6F979C838B83A39628
:10B2D0008CAD9DADAEADBFADA3978D839E83AF8387
:10B2E000B887A7968CAD9DADAEADBFADA79789874A
:10B2F0009A87AB87BC871A8309838DE0F401DE014E
:10B300001D9601900D928A95E1F7E6968EAD9FAD60
:10B31000E6979B8F8A8FB101CE0101960E94585803
:10B32000CE01855A9F4F0E943786F3CE64E279E0C2
:10B33000CE0101960E949365CE0101960E94D50927
:10B34000CE0101960E94FA64E696EEADFFADE69757
:10B3500040E050E0BA01309721F043895489658973
:10B360007689CE0101960E940463CE0101960E9467
:10B37000BE09CE0101960E94FA64D2CFCE57DF4FAC
:10B380000FB6F894DEBF0FBECDBFDF91CF911F91F6
:10B390000F91FF90EF90DF90CF90BF90AF909F9074
:10B3A0008F907F906F905F904F903F902F90089577
:10B3B0000895AF92BF92CF92DF92EF92FF920F93D8
:10B3C0001F93CF93DF936C017B018B01040F151F3B
:10B3D000EB015E01AE18BF08C017D10759F06991A3
:10B3E000D601ED91FC910190F081E02DC6011995F7
:10B3F000892B79F7C501DF91CF911F910F91FF90B4
:10B40000EF90DF90CF90BF90AF900895FC01A0899E
:10B41000B1898C91A689B78982FD0FC09C91818DDD
:10B420008F5F8F73228D821749F0A18DAE0FBF2FD2
:10B43000B11D5D969C93818F08958C910895FC01B8
:10B44000538D448D252F30E0842F90E0821B930B89
:10B45000541710F0CF96089501970895FC01918D2F
:10B46000828D981761F0A28DAE0FBF2FB11D5D9632
:10B470008C91928D9F5F9F73928F90E008958FEFD4
:10B480009FEF0895FC01918D828D981731F0828D88
:10B49000E80FF11D858D90E008958FEF9FEF0895DF
:10B4A000FC01918D228D892F90E0805C9F4F821B43
:10B4B00091098F739927089589E79FE00E94505A58
:10B4C00021E0892B09F420E0822F089586E190E1A4
:10B4D0000E94505A21E0892B09F420E0822F089520
:10B4E00083EB90E10E94505A21E0892B09F420E07F
:10B4F000822F089580E591E10E94505A21E0892B26
:10B5000009F420E0822F0895FC01A48DA80FB92F23
:10B51000B11DA35ABF4F2C91848D90E001968F737B
:10B520009927848FA689B7892C93A089B1898C919A
:10B53000837080648C93938D848D981306C00288E9
:10B54000F389E02D80818F7D80830895EF92FF92B3
:10B550000F931F93CF93DF93EC0181E0888F9B8D36
:10B560008C8D98131AC0E889F989808185FF15C0F0
:10B570009FB7F894EE89FF896083E889F989808113
:10B580008370806480839FBF81E090E0DF91CF91E2
:10B590001F910F91FF90EF900895F62E0B8D10E004
:10B5A0000F5F1F4F0F731127E02E8C8D8E110CC073
:10B5B0000FB607FCFACFE889F989808185FFF5CFBE
:10B5C000CE010E94845AF1CFEB8DEC0FFD2FF11DBF
:10B5D000E35AFF4FF0829FB7F8940B8FEA89FB89FB
:10B5E00080818062CFCFCF93DF93EC01888D882359
:10B5F000B9F0AA89BB89E889F9898C9185FD03C0D6
:10B60000808186FD0DC00FB607FCF7CF8C9185FFBA
:10B61000F2CF808185FFEDCFCE010E94845AE9CF21
:10B62000DF91CF91089580E090E0892B29F00E946E
:10B630007A5A81110E94000080E090E0892B29F065
:10B640000E94705A81110E94000080E090E0892BD6
:10B6500029F00E94665A81110E94000080E090E06B
:10B66000892B29F00E945C5A81110C9400000895E6
:10B670008150823108F05AC0E82FF0E08827EC5B57
:10B68000F44A8F4F0C9457BA645B685B565B5C5B03
:10B69000605B965B6B5B715B755B7B5B7F5B835B0E
:10B6A000895B8D5B965B915B975B9B5B8091800078
:10B6B0008F77809380000895809180008F7DF9CFEF
:10B6C00080918000877FF5CF84B58F7784BD089502
:10B6D00084B58F7DFBCF8091B0008F778093B000D1
:10B6E00008958091B0008F7DF9CF809190008F7781
:10B6F000809390000895809190008F7DF9CF809184
:10B700009000877FF5CF8091A0008F778093A00075
:10B7100008958091A0008F7DF9CF8091A000877F50
:10B72000F5CF809120018F7780932001089580913B
:10B7300020018F7DF9CF80912001877FF5CF3FB722
:10B74000F89480917B1690917C16A0917D16B09113
:10B750007E1626B5A89B05C02F3F19F00196A11DA6
:10B76000B11D3FBFBA2FA92F982F8827BC01CD014B
:10B77000620F711D811D911D42E0660F771F881FAA
:10B78000991F4A95D1F708950E9480BC0F931F938B
:10B79000CF93DF93EC0188819981009759F02A813A
:10B7A0003B812617370730F081E0DF91CF911F9161
:10B7B0000F9108958B016F5F7F4F0E949FBB009791
:10B7C00059F0998388831B830A832C813D81232B25
:10B7D00059F7FC011082E8CF80E0E7CFEF92FF92AB
:10B7E0000F931F93CF93DF936115710541F480E0B0
:10B7F000DF91CF911F910F91FF90EF900895411528
:10B800005105B1F07B01EC010C811D81040F151F66
:10B81000B8010E94C65B882351F3288139818C814D
:10B820009D81B701820F931F0E94D0BC1D830C83A2
:10B8300081E0DECFCF93DF93EC018881998100977F
:10B8400011F00E9416BB198218821D821C821B8275
:10B850001A82DF91CF910895EF92FF920F931F9379
:10B86000CF93DF93EC017B018A01BA010E94C65B92
:10B8700081110BC0CE010E941A5CCE01DF91CF91E5
:10B880001F910F91FF90EF9008951D830C83B701D6
:10B89000888199810E94D0BCF0CF8CBD9DBD089558
:10B8A0008F929F92AF92BF92CF92DF92EF92FF92D0
:10B8B0000F931F93CF93DF93D091770FD13208F07E
:10B8C000D7C0182FC091760F0E949F5B6B017C013F
:10B8D00080914E0F81116BC082E080934E0F1093C8
:10B8E0004D0F8FEF80934C0F10924B0FD0934A0F58
:10B8F000A6E5BFE0EAE2FFE080E0D81391C0109235
:10B90000290F8091290FCC0FC82BC093290F80914C
:10B91000280F813009F088C01092280F0E949F5B89
:10B920006B017C018091290F8093BB008091500FA7
:10B930009091510FA091520FB091530F892B8A2BE8
:10B940008B2BA1F00E949F5B0091500F1091510F23
:10B950002091520F3091530F6C197D098E099F0968
:10B96000061717072807390708F442C08091BC0062
:10B9700083FDD8CF85EC8093BC000E949F5B6B0158
:10B980007C0180914E0F823009F450C080914C0FA1
:10B990008F3F09F46FC080914C0F803209F46CC066
:10B9A00080914C0F803309F469C084E026C08091F7
:10B9B000500F9091510FA091520FB091530F892BBE
:10B9C0008A2B8B2B09F484CF0E949F5B8090500FB1
:10B9D0009090510FA090520FB090530F6C197D09A9
:10B9E0008E099F0986169706A806B90608F070CF3B
:10B9F00080914F0F0E948E7985E01092550F109222
:10BA0000770F1092540FDF91CF911F910F91FF90FC
:10BA1000EF90DF90CF90BF90AF909F908F90089560
:10BA20009D9191938F5F69CF85EEA5CF8091500F47
:10BA30009091510FA091520FB091530F892B8A2BE7
:10BA40008B2B09F49ECF0E949F5B0091500F1091A9
:10BA5000510F2091520F3091530F6C197D098E09AF
:10BA60009F09061717072807390708F08ACFC0CFA4
:10BA700081E0C3CF80E0C1CF82E0BFCF83E0BDCF04
:10BA8000682F8DEE91E10C943F76CF93DF93EC011C
:10BA90009A01AB01E889F98982E08083211581EE62
:10BAA00038074105510581F160E079E08DE390E0D0
:10BAB0000E94B5B821503109410951095695479561
:10BAC00037952795EC85FD851082EE85FF852083CF
:10BAD000188EEC89FD8986E08083EA89FB89808164
:10BAE00080618083EA89FB89808188608083EA891C
:10BAF000FB89808180688083EA89FB8980818F7DD2
:10BB00008083DF91CF910895E889F989108220E13F
:10BB1000D9CF8F929F92AF92BF92CF92DF92EF9246
:10BB2000FF920F931F93CF93DF9300D0CDB7DEB773
:10BB30004C017B016A01DC01ED91FC9180E8DB01A5
:10BB4000982F1D929A95E9F7DA011D928A95E9F7E7
:10BB5000808190E8A92EB12C811119C084E090E079
:10BB600006C08F0181E090E0D4010D931C930F90EB
:10BB70000F900F90DF91CF911F910F91FF90EF9059
:10BB8000DF90CF90BF90AF909F908F9008958F01DE
:10BB90000F5F1F4F6081663229F394F4662309F327
:10BBA0006532D1F0B2E0AB16B10444F0F701608326
:10BBB000F1E0AF1AB108C70101967C01F801E7CFA7
:10BBC0006B3209F45EC06D3369F78181882351F2CD
:10BBD00080E8A82EB12C45C081818983882311F289
:10BBE00082818A838F01811103C00E5F1F4FBACFFC
:10BBF0000D5F1F4F1B8240E150E070E060E0CE011E
:10BC000001960E94AEB1CECF663281F06B32A1F5C3
:10BC100060E232C0F801818189838823A1F18281A9
:10BC20008A83811107C00E5F1F4F7801870183E06F
:10BC300090E09ACF7801F3E0EF0EF11C1B8240E117
:10BC400050E070E060E0CE0101960E94AEB114C0F9
:10BC5000D6016C93B1E0AB1AB108F60131966F01D1
:10BC6000870178019FEFE91AF90AD8016C916532D2
:10BC700089F254F66623C9F2E2E0AE16B10444F745
:10BC8000EFCF60E28FCF8701D0CFCF92DF92EF92DC
:10BC9000FF920F931F93CF93DF93D82FC62F61325C
:10BCA00008F098C00E949F5B6B017C0180914E0F51
:10BCB00081116BC081E080934E0F80934D0F9FEFF9
:10BCC00090934C0F10924B0F9C0F90934A0F8093C0
:10BCD000290F8091290FDD0FD82BD093290F809148
:10BCE000280F813009F078C01092280F0E949F5BC6
:10BCF0006B017C018091290F8093BB008091500FD4
:10BD00009091510FA091520FB091530F892B8A2B14
:10BD10008B2BA1F00E949F5B0091500F1091510F4F
:10BD20002091520F3091530F6C197D098E099F0994
:10BD3000061717072807390708F448C08091BC0088
:10BD400083FDD8CF85EC8093BC000E949F5B6B0184
:10BD50007C0180914E0F813009F440C080914B0FDF
:10BD60008C1710F4C0914B0FEAE2FFE0A8E0BFE0AF
:10BD700080E08C1355C08C2FDF91CF911F910F91D4
:10BD8000FF90EF90DF90CF9008958091500F9091A9
:10BD9000510FA091520FB091530F892B8A2B8B2BEF
:10BDA00009F484CF0E949F5B0091500F1091510FB6
:10BDB0002091520F3091530F6C197D098E099F0904
:10BDC000061717072807390708F070CF80914F0F23
:10BDD0000E948E79C0E0CFCF85EEB5CF8091500F15
:10BDE0009091510FA091520FB091530F892B8A2B34
:10BDF0008B2B09F4AECF0E949F5B0091500F1091E6
:10BE0000510F2091520F3091530F6C197D098E09FB
:10BE10009F09061717072807390708F09ACFD6CFCA
:10BE200091919D938F5FA5CFCF93DF93EC016E85AA
:10BE30007F858889998941E00E94B17C882351F0EF
:10BE40008A8920E2829FC00111248C5F924FDF918A
:10BE5000CF91089590E080E0FACF8F929F92AF92B9
:10BE6000BF92CF92DF92EF92FF920F931F93CF93E7
:10BE7000DF9300D01F92CDB7DEB7FC018581813002
:10BE800091F080E00F900F900F900F90DF91CF9185
:10BE90001F910F91FF90EF90DF90CF90BF90AF90E8
:10BEA0009F908F900895848181FFEBCF838994893F
:10BEB000A589B689892B8A2B8B2B09F45EC07F015B
:10BEC00040E050E0BA01CF010E94F47E8823C9F21D
:10BED000F701C38CD48C8788908CA18CB28C82E0C3
:10BEE00090E0A0E0B0E0F60180839183A283B38369
:10BEF0009E012F5F3F4FB501A401C6010E949C7DAA
:10BF0000882309F4BECF00E010E09801B501A40138
:10BF1000C6010E94FA7C882309F4B3CF89809A80F5
:10BF2000AB80BC80F6018789803111F188EF9FEFEB
:10BF3000AFEFBFE088169906AA06BB06C8F2F70164
:10BF4000178A108E118E128E138A148A158A168AF9
:10BF5000848180688483C7010E94CE81882309F48C
:10BF600090CF40E050E0BA01C7010E94F47E8ACF32
:10BF700088EF9FEFA0E0B0E0DDCF81E083CF0F93AB
:10BF80001F93CF93DF934115510541F0FC010481CC
:10BF900015810115110539F4FB011082DF91CF9154
:10BFA0001F910F910895415051094017510708F40E
:10BFB0008A01EB01FC0160817181A801CE010E9420
:10BFC000E5BCC00FD11F1882E9CF20E3FC0120831C
:10BFD0003296862F82958F706F706A3030F4605D74
:10BFE0006293682F8111F5CF0895695CF9CF5F9254
:10BFF0006F927F928F929F92AF92BF92CF92DF9279
:10C00000EF92FF920F931F93CF93DF93CDB7DEB7DD
:10C01000C754D1090FB6F894DEBF0FBECDBF5C0187
:10C020003B0119A218A280E893E09F8F8E8F1BA27C
:10C030001C821B829A8389831E8210E000E06E01BD
:10C040008EE1C80ED11C83E2E82E82E1F82EF501C4
:10C05000E00FF11F80818F3211F40F5F1F4FD50168
:10C06000A00FB11FFE01FB9690E080E04F012D91E3
:10C070002F3249F0222339F00F5F1F4F0196219391
:10C080008C309105A1F7880D991DFC011082F501F6
:10C09000E00FF11F80818F3211F40F5F1F4FF50108
:10C0A000E00FF11F508041E0511040E030E020E00F
:10C0B000B401C701F3011995811121C0F3E2EF1614
:10C0C000F2E1FF06C1F480E0C95BDF4F0FB6F894E0
:10C0D000DEBF0FBECDBFDF91CF911F910F91FF90BB
:10C0E000EF90DF90CF90BF90AF909F908F907F9018
:10C0F0006F905F900895C7010E94FD81E4CF5520A5
:10C1000091F021E0A401B701C6010E941182982E8E
:10C1100083E2E81682E1F80681F0C7010E94FD8102
:10C12000911010C0D0CF93E2E91692E1F90619F010
:10C13000C7010E94FD8181E0C7CF992021F2FE0155
:10C1400031967F019E2D8F2D7601C92ED82E7FCF5F
:10C150008F929F92AF92BF92CF92DF92EF92FF9217
:10C16000CF9329EF31E13093F70C2093F60C88231D
:10C1700009F46DC040E060E070E0CB010E94B17C4A
:10C1800081110BC080E0CF91FF90EF90DF90CF90B6
:10C19000BF90AF909F908F9008958091C20E8F773F
:10C1A00089F78091CE0E9091CF0EA091D00EB091D4
:10C1B000D10E84369105A105B10520F3C090CA0EB9
:10C1C000D090CB0EE090CC0EF090CD0EC114D104E7
:10C1D000E104F104B9F240E0C701B6010E94B17C6C
:10C1E000882381F280910F0D9091100D811592405E
:10C1F00049F6A091140DAA2329F26091120D7091B5
:10C20000130D6115710509F4BDCF2091110D222385
:10C2100009F4B8CFA09317122093091290E080E0A0
:10C2200030E0E1E0F0E0C82FAF01082E02C0440F7B
:10C23000551F0A94E2F72417350769F041E0480FCB
:10C2400001968930910579F7409312129BCFC12C4A
:10C25000D12C7601C0CF8093121220911A0D30910B
:10C260001B0D50E040E02115310541F42091280DCF
:10C270003091290D40912A0D50912B0D20930A12D7
:10C2800030930B1240930C1250930D12460157013C
:10C29000860E971EA11CB11C809218129092191242
:10C2A000A0921A12B0921B12E091150DF091160D8A
:10C2B000F0931E12E0931D12B0E00E94F6B8DC016C
:10C2C000CB01880D991DAA1DBB1D80931F12909351
:10C2D0002012A0932112B093221225E0EE0FFF1F2F
:10C2E0002A95E1F7E150FE4FEF2FFF27E6958E0FDD
:10C2F0009F1FA11DB11D8093131290931412A09340
:10C300001512B09316128090170D9090180DB12C45
:10C31000A12C8114910441F48090240D9090250D5E
:10C32000A090260DB090270DC81AD90AEA0AFB0A78
:10C33000C80CD91CEA1CFB1C04C0F694E794D794E3
:10C34000C794CA95D2F7C0920E12D0920F12E09203
:10C350001012F092111285EFC8168FE0D806E10492
:10C36000F10428F48CE080931C1281E00CCF80E172
:10C3700025EFC2162FEFD206E104F104A0F380915D
:10C38000300D9091310DA091320DB091330D80930D
:10C390001F1290932012A0932112B093221280E2D8
:10C3A000E2CF1092F50C1092F40C1092550F1092EF
:10C3B000770F0E94707986EE95E79093F30C809347
:10C3C000F20C87EE95E79093F10C8093F00C0895B2
:10C3D0008F929F92AF92BF92CF92DF92EF92FF9295
:10C3E0000F931F93CF93DF93CDB7DEB760970FB650
:10C3F000F894DEBF0FBECDBF7C019091FB0C99235A
:10C4000051F108E0933309F404E06B0180E591E019
:10C410000E944D5C9E012F5F3F4F5901490110E082
:10C42000812F0E941A88F40181934F018823D9F04B
:10C430001F5F0113F5CF00E0F50181915F018D31A0
:10C4400061F0883151F08A51823038F00F5F10135B
:10C45000F3CF0E94958918E08AC060E170E0802FD8
:10C460000E947888102FA12EB12CF501EE0FFF1F2E
:10C47000E052F34F1182108283EE93E00197F1F7BF
:10C4800042E870E060E0812F0E945B884FEF62E03D
:10C4900070E0812F0E945B88B601C114D10491F431
:10C4A000809161029091620201968115F0EC9F07E4
:10C4B00008F471C0909362028093610260916102FE
:10C4C00070916202812F0E94458886E0E5E4F3E0E6
:10C4D000DE01199601900D928A95E1F7F7018381AB
:10C4E0008F778C8784818D8785818E87A7014E5FAA
:10C4F0005F4F24E030E06CE070E0812F0E941E88E6
:10C50000B601812F0E942F8826E030E0AE01475F00
:10C510005F4F66E070E0812F0E941E8861E070E04E
:10C52000812F0E94788827E02A9DC0012B9D900DC5
:10C5300011249C012855334F7901F9011182108291
:10C5400022E030E0AE01415F5F4F68E270E0812F92
:10C550000E9488888F859889982789279827F701CE
:10C56000938382831682158214820E949589812F7B
:10C5700060960FB6F894DEBF0FBECDBFDF91CF91AE
:10C580001F910F91FF90EF90DF90CF90BF90AF90F1
:10C590009F908F90089580E090EC8CCFFB010190EC
:10C5A0000020E9F73197AF01461B570B0C942C5C28
:10C5B0000F931F93CF93DF93CDB7DEB762970FB67C
:10C5C000F894DEBF0FBECDBF8C01CB01F801118204
:10C5D000108213821282158214824AE0BE016F5FBC
:10C5E0007F4F0E9413B3BE016F5F7F4FC8010E944F
:10C5F000CE6262960FB6F894DEBF0FBECDBFDF915C
:10C60000CF911F910F9108950F931F93CF93DF93B5
:10C61000CDB7DEB7A1970FB6F894DEBF0FBECDBF82
:10C620008C01CB01BA01F8011182108213821282AF
:10C63000158214822AE0AE014F5F5F4F0E9455B30E
:10C64000BE016F5F7F4FC8010E94CE62A1960FB6F8
:10C65000F894DEBF0FBECDBFDF91CF911F910F9138
:10C660000895CF93DF93EC016115710531F00E94BD
:10C67000CE62CE01DF91CF9108950E941A5CF9CF6E
:10C68000FC0180819181009711F00C94B1B260E0BF
:10C6900070E0CB010895FC0180819181009711F039
:10C6A0000C94D3B260E070E0CB010895AF92BF92DA
:10C6B000CF92DF92EF92FF920F931F93CF93DF936E
:10C6C000DC01CD90DC901197C114D10439F014969F
:10C6D000CD91DC918C017601209761F4DF91CF91AF
:10C6E0001F910F91FF90EF90DF90CF90BF90AF9090
:10C6F000089575015701BFEFAB1ABB0AF70180819E
:10C70000082E000C990B0E94FAB2892B91F7219701
:10C71000CC0DDD1D8881082E000C990B0E94FAB209
:10C72000892B29F0CE15DF0510F02197F3CFAE014C
:10C730004F5F5F4F4E195F09D80115965C934E937A
:10C740001497CE14DF0420F4B701C6010E949ABCEE
:10C75000D801ED91FC91119714968D919C91E80F61
:10C76000F91F1082BBCFFC0124813581621773074A
:10C7700048F480819181009729F0860F971FFC0172
:10C780008081089580E00895FC0124813581FB01BA
:10C790004481558124173507A0F0FC0180819181E7
:10C7A000009779F0FB01608171816115710549F095
:10C7B000241B350B820F931F0E94C7BC21E0892BDD
:10C7C00009F020E0822F0895FB0144815581FC018E
:10C7D000248135812417350778F080819181009775
:10C7E00059F0FB01608171816115710529F00E948A
:10C7F000D7BC21E0892B09F020E0822F0895CF9348
:10C80000DF93EC01FB0101900020E9F73197AF01C4
:10C81000461B570B0E94EE5B811103C0CE010E94A4
:10C820001A5CCE01DF91CF910895CF93DF93EC0195
:10C83000FB0144815581608171810E94EE5B811111
:10C8400003C0CE010E941A5CCE01DF91CF91089502
:10C85000EF92FF920F931F93CF93DF93EC017B0135
:10C86000CB010E940AB30097A9F00C811D81080F2B
:10C87000191FB801CE010E94C65B882361F0288190
:10C8800039818C819D81B701820F931F0E9403B370
:10C890001D830C8381E0DF91CF911F910F91FF9059
:10C8A000EF900895CF93DF931F921F92CDB7DEB71D
:10C8B00069831A8241E050E0BE016F5F7F4F0E94A2
:10C8C000EE5B0F900F90DF91CF910895CF93DF93A0
:10C8D000EC010E945264811103C0CE010E941A5CD7
:10C8E000CE01DF91CF910895FB0101900020E9F77F
:10C8F0003197AF01461B570B0C94EE5BFB01448153
:10C900005581608171810C94EE5BEF92FF920F93E1
:10C910001F93CF93DF93EC018B01CB010E940AB3ED
:10C920007C01BC01CE010E94C65B81110BC0CE010F
:10C930000E941A5CCE01DF91CF911F910F91FF9061
:10C94000EF900895FD82EC82B801888199810E9460
:10C9500003B3F0CFCF93DF93EC01FB01861797076A
:10C9600049F0608171816115710541F04481558103
:10C970000E942C5CCE01DF91CF9108950E941A5C39
:10C98000F9CF0F931F93CF93DF938C01EB01FC0141
:10C99000808191810097E1F068817981611571054D
:10C9A000A9F0428153812C813D814217530770F0D9
:10C9B0000E94D0BC8C819D81F801958384831D8267
:10C9C0001C82DF91CF911F910F9108950E9416BB99
:10C9D00088819981F801918380838A819B819383E7
:10C9E00082838C819D8195838483198218821B8226
:10C9F0001A82E5CFFC0180819181009711F00C949F
:10CA000016BB0895EF92FF920F931F93CF93DF937E
:10CA1000CDB7DEB7A1970FB6F894DEBF0FBECDBF7E
:10CA20007C01CB01BA01F7011182108213821282BC
:10CA30001582148242E0420F8E010F5F1F4F0E9449
:10CA4000ECB0BC01C7010E943163A1960FB6F89407
:10CA5000DEBF0FBECDBFDF91CF911F910F91FF9031
:10CA6000EF9008950F931F93CF93DF93CDB7DEB769
:10CA7000A2970FB6F894DEBF0FBECDBF8C01CB01DD
:10CA8000BA01F80111821082138212821582148277
:10CA900030E0AE014F5F5F4F0E941EB3BE016F5F7B
:10CAA0007F4FC8010E94CE62A2960FB6F894DEBFF7
:10CAB0000FBECDBFDF91CF911F910F910895CF93FE
:10CAC000DF931F921F92CDB7DEB7FC011182108257
:10CAD000138212821582148269831A82BE016F5FEB
:10CAE0007F4F0E94CE620F900F90DF91CF910895FB
:10CAF000FC011182108213821282158214820C941E
:10CB0000C164FC0111821082138212821582148288
:10CB10000C948564FC0111821082138212821582AA
:10CB200014820C94AA64FC01118210821382128276
:10CB3000158214826115710551F0FB0101900020EE
:10CB4000E9F73197AF01461B570B0C942C5C089505
:10CB5000AF92BF92CF92DF92EF92FF920F931F930B
:10CB6000CF93DF935C016B017A01890124173507AC
:10CB700020F48F2D7901042F182F66E279E0C5018A
:10CB80000E949365D6011496CD91DC91EC16FD06BA
:10CB9000C8F40C171D0708F4E801D601ED91FC91CB
:10CBA0001197EC0FFD1F108110826D917C916E0D1D
:10CBB0007F1DC5010E943163F60180819181C80FFC
:10CBC000D91F1883C501DF91CF911F910F91FF905D
:10CBD000EF90DF90CF90BF90AF900895FB01019050
:10CBE0000020E9F73197AF01461B570BDC01ED91AF
:10CBF000FC910280F381E02D19948F929F92AF9265
:10CC0000BF92EF92FF920F931F93CF93DF93CDB715
:10CC1000DEB7A1970FB6F894DEBF0FBECDBF7C0183
:10CC2000FA01CB0119A2223008F42AE08E010F5D2F
:10CC30001F4F822E912CB12CA12CBF01A501940174
:10CC40000E94B5B8F901CA016A300CF5605DD801DF
:10CC50006E938D01232B242B252B79F790E080E018
:10CC6000109721F0BD01C7010E94EE65A1960FB695
:10CC7000F894DEBF0FBECDBFDF91CF911F910F9112
:10CC8000FF90EF90BF90AF909F908F900895695C58
:10CC9000DECFCF93DF93482F50E070E060E020E1DB
:10CCA00080E591E10E94FD65EC016AE979E080E5AB
:10CCB00091E10E94EE658C0F9D1FDF91CF91089549
:10CCC0008F929F92AF92BF92CF92DF92EF92FF929C
:10CCD0000F931F93CF93DF937C01EB016C0182E0F4
:10CCE000C80ED11C4701E5E08E0E911C10E000E05B
:10CCF000F60141916F0150E070E060E02AE0CE0162
:10CD00000E94FD655C01E881F9810190F081E02DD0
:10CD10006EE2CE0119958A0D9B1D080F191FC814CC
:10CD2000D90431F7F701458150E070E060E02AE076
:10CD3000CE010E94FD65800F911FDF91CF911F9161
:10CD40000F91FF90EF90DF90CF90BF90AF909F90AA
:10CD50008F9008950F931F93CF93DF93EC01CB0136
:10CD6000BE010E9460668C016AE979E0CE010E94F2
:10CD7000EE65800F911FDF91CF911F910F91089564
:10CD80000F931F93CF93DF93EC010E94EE658C010C
:10CD90006AE979E0CE010E94EE65800F911FDF9174
:10CDA000CF911F910F9108956115710511F00C94A9
:10CDB000EE6590E080E00895DB0114964D915C9162
:10CDC00015976D917C91DC01ED91FC910280F381CE
:10CDD000E02D19940F931F93CF93DF93EC010E94E2
:10CDE000DC668C016AE979E0CE010E94EE65800F75
:10CDF000911FDF91CF911F910F910895EF92FF92B4
:10CE00000F931F93CF93DF938C017B01D0E0C0E0A1
:10CE1000F701EC0FFD1F6491662361F0D801ED91DD
:10CE2000FC910190F081E02DC8011995892B11F03A
:10CE30002196EECFCE01DF91CF911F910F91FF9000
:10CE4000EF900895DC0180E294E08D939D9384E05F
:10CE5000FB0101900D928A95E1F708951F920F92C0
:10CE60000FB60F9211240BB60F922F933F934F934F
:10CE70005F936F937F938F939F93AF93BF93EF9342
:10CE8000FF9389E79FE00E94845AFF91EF91BF9141
:10CE9000AF919F918F917F916F915F914F913F9152
:10CEA0002F910F900BBE0F900FBE0F901F901895F3
:10CEB0001F920F920FB60F9211240BB60F922F9361
:10CEC0003F934F935F936F937F938F939F93AF9312
:10CED000BF93EF93FF9389E79FE00E94065AFF916B
:10CEE000EF91BF91AF919F918F917F916F915F91E2
:10CEF0004F913F912F910F900BBE0F900FBE0F904F
:10CF00001F9018951F920F920FB60F9211240BB617
:10CF10000F922F933F934F935F936F937F938F93D2
:10CF20009F93AF93BF93EF93FF9386E190E10E94AD
:10CF3000845AFF91EF91BF91AF919F918F917F9113
:10CF40006F915F914F913F912F910F900BBE0F907A
:10CF50000FBE0F901F9018951F920F920FB60F9251
:10CF600011240BB60F922F933F934F935F936F93C0
:10CF70007F938F939F93AF93BF93EF93FF9386E13C
:10CF800090E10E94065AFF91EF91BF91AF919F915E
:10CF90008F917F916F915F914F913F912F910F9062
:10CFA0000BBE0F900FBE0F901F9018951F920F92FF
:10CFB0000FB60F9211240BB60F922F933F934F93FE
:10CFC0005F936F937F938F939F93AF93BF93EF93F1
:10CFD000FF9383EB90E10E94845AFF91EF91BF9100
:10CFE000AF919F918F917F916F915F914F913F9101
:10CFF0002F910F900BBE0F900FBE0F901F901895A2
:10D000001F920F920FB60F9211240BB60F922F930F
:10D010003F934F935F936F937F938F939F93AF93C0
:10D02000BF93EF93FF9383EB90E10E94065AFF9129
:10D03000EF91BF91AF919F918F917F916F915F9190
:10D040004F913F912F910F900BBE0F900FBE0F90FD
:10D050001F9018951F920F920FB60F9211240BB6C6
:10D060000F922F933F934F935F936F937F938F9381
:10D070009F93AF93BF93EF93FF9380E591E10E945D
:10D08000845AFF91EF91BF91AF919F918F917F91C2
:10D090006F915F914F913F912F910F900BBE0F9029
:10D0A0000FBE0F901F9018951F920F920FB60F9200
:10D0B00011240BB60F922F933F934F935F936F936F
:10D0C0007F938F939F93AF93BF93EF93FF9380E5ED
:10D0D00091E10E94065AFF91EF91BF91AF919F910C
:10D0E0008F917F916F915F914F913F912F910F9011
:10D0F0000BBE0F900FBE0F901F901895CF93DF932C
:10D10000282F30E0F901EA52F64F8491F901E658F0
:10D11000F44FD491F901E054F44FC491CC23A1F021
:10D1200081110E94385BEC2FF0E0EE0FFF1FE454FA
:10D13000F64FA591B491EC91ED2381E090E009F4D4
:10D1400080E0DF91CF91089580E090E0FACF1F93C7
:10D15000CF93DF93282F30E0F901EA52F64F849104
:10D16000F901E658F44FD491F901E054F44FC49119
:10D17000CC23A9F0162F81110E94385BEC2FF0E030
:10D18000EE0FFF1FEA5BF44FA591B4918FB7F894AF
:10D19000EC91111108C0D095DE23DC938FBFDF9195
:10D1A000CF911F910895DE2BF8CFAF92BF92CF920F
:10D1B000DF92EF92FF920F931F93CF93DF936B0158
:10D1C0007A01EC01CE58D94E28813CE0389F80018D
:10D1D000399F100D1124A090A117B12C27FF1FC05B
:10D1E000FB011182108288818F5F8883888198017A
:10D1F000280F311D87FD3A95F6012A153B051CF4D1
:10D2000088818C30C4F180819181049680349C495E
:10D2100008F473C0F60180819181049670C0888102
:10D220009801280F311D87FD3A952A153B05DCF63C
:10D230008881A801480F511D87FD5A95FA01EE0F0C
:10D24000FF1FE40FF51FE85BFD4E808186FFCBCF0B
:10D250008881F801E80FF11D87FDFA95CF01EE0FE7
:10D26000FF1FE80FF91FE85BFD4E808160E08F73C0
:10D270000E94A768B8CF808191812881A801420FC0
:10D28000511D27FD5A959A01FA01EE0FFF1FE20F7B
:10D29000F31FE85BFD4E21813281820F931FF7015E
:10D2A0009183808388819801280F311D87FD3A95ED
:10D2B000F901EE0FFF1FE20FF31FE85BFD4E8081C7
:10D2C00086FF22C08881080F111D87FD1A95F8017D
:10D2D000EE0FFF1FE00FF11FE85BFD4E808161E064
:10D2E0008F73DF91CF911F910F91FF90EF90DF909F
:10D2F000CF90BF90AF900C94A76880E49CE9F701B1
:10D30000918380838FEF8883DF91CF911F910F915D
:10D31000FF90EF90DF90CF90BF90AF900895CF93A4
:10D32000DF9390E0FC01E658F44F24918054944F31
:10D33000FC0184918823D1F090E0880F991FFC01B3
:10D34000E05AF44FA591B491FC01EA5BF44FC5910A
:10D35000D49161110EC09FB7F8948C91E22FE095A3
:10D360008E238C932881E223E8839FBFDF91CF91A6
:10D3700008958FB7F894EC91E22BEC938FBFF6CF22
:10D380008F929F92AF92BF92CF92DF92EF92FF92D5
:10D390006B017C010E949F5B4B015C01C114D104B5
:10D3A000E104F104B9F00E949F5B681979098A09C8
:10D3B0009B09683E73408105910580F321E0C21A04
:10D3C000D108E108F10888EE880E83E0981EA11CC0
:10D3D000B11CE4CFFF90EF90DF90CF90BF90AF9063
:10D3E0009F908F900895AF92BF92CF92DF92EF926D
:10D3F000FF920F931F93CF93DF93C82FD62F1092D6
:10D40000D6151092D7151092D8151092D9151092E2
:10D41000DA1561E00E948F6960E08C2F0E94A76896
:10D420006D2F70E090E080E00E94C06960E08C2F7A
:10D430000E948F698BE990E00197F1F700E911E014
:10D440008C2F0E947E68892B81F401501109C1F74D
:10D450008EEF9FEFDF91CF911F910F91FF90EF9093
:10D46000DF90CF90BF90AF90089500E911E08C2F2E
:10D470000E947E68019721F401501109C1F7E8CF9D
:10D4800018E2D0E800E090E9E92EFF24F3948C2F15
:10D490000E947E68892B29F481E0E81AF108B9F727
:10D4A000D7CF0E949F5B6B017C0180E9A82EBB2433
:10D4B000B3948C2F0E947E68019729F481E0A81A0A
:10D4C000B108B9F7C5CF0E949F5B6C197D098E0921
:10D4D0009F09693271058105910538F0E02FF0E070
:10D4E000E253FA4E80858D2B8087D69511F40F5F1D
:10D4F000D0E8115041F690E080E0ACCF0F931F933D
:10D50000CF93DF9300D000D01F921F92CDB7DEB72C
:10D510008091671781112AC010924F1710924E17F1
:10D5200088EE93E0A0E0B0E08093501790935117FD
:10D53000A0935217B09353178AEA93E090934D1734
:10D5400080934C1780E294E090935B1780935A1776
:10D5500010925C1710925D1710925E1710925F1771
:10D5600088E08093641781E08093671789E097E1F2
:10D570009093FE0C8093FD0C8091081781119DC043
:10D5800060E372E080E090E00E94C0691FB7F89409
:10D5900080910717811127C0E5EFFBE08491EFEA46
:10D5A000FBE09491E82FF0E0EE0FFF1FE05AF44FFC
:10D5B000A591B491EC91E92321F461E085E30E9407
:10D5C000A76861E085E30E948F698CB580618CBD9E
:10D5D0008CB580648CBD61E084E30E948F6961E05A
:10D5E00083E30E948F69809107178F5F80930717ED
:10D5F0001FBFEAECFBE0E491F0E0EE0FFF1FEA5BF7
:10D60000F44F859194919093FA0C8093F90CE4E88F
:10D61000FBE0E491E093F80C61E08AE00E948F69FE
:10D620000E947E8680E591E00E944D5C84E38093B9
:10D63000FB0C80E80E9407880E94F187882309F488
:10D64000F5C088E00E9407880E94DE87883009F0D4
:10D65000EDC080E10E9407880E94DE87803109F0DA
:10D66000E5C080E00E9407880E94DE87182F8111A4
:10D67000DDC041E050E0BE016F5F7F4F8FE190E081
:10D680000E9488868981833009F0D0C080E480932D
:10D69000FC0C42E06EE170E0812F0E945B8842E06A
:10D6A0006FE170E0812F0E945B881F5F183089F75F
:10D6B0000E94958981E08093081780E591E00E949F
:10D6C0004D5C46E050E063E672E089E090E00E9445
:10D6D000308780E294E09A8389831B821C821D82BA
:10D6E0001E82CE0103960E948E890E9495898091A8
:10D6F000FD0C9091FE0CDC0192961D921D921D92E4
:10D700001C929597FC0116A217A210A611A69A9634
:10D710001D921D921D921C929D9740E65AEE60E06C
:10D7200070E046AB57AB60AF71AF40EA5FE060E0DE
:10D7300070E0DA964D935D936D937C93DD973E9602
:10D7400024E1DF011D922A95E9F726E0E3E6F2E005
:10D75000DC01189601900D922A95E1F7FC01EE5B31
:10D76000FF4F10820E945C948C01019709F0CBC09E
:10D7700080E591E00E944D5C6091FD0C7091FE0C83
:10D78000625F7F4FCE0101960E942267CE01039611
:10D790000E948E896091FD0C7091FE0C6A5E7F4F35
:10D7A000CE0101960E94226744E050E0BE016D5F09
:10D7B0007F4F81E090E00E9430876091FD0C709176
:10D7C000FE0C6E5E7F4FCE0101960E94226744E000
:10D7D00050E0BE016D5F7F4F85E090E00E94308792
:10D7E0000E9495896091FD0C7091FE0C625E7F4FE6
:10D7F000CE0101960E9422678B819C81AD81BE8102
:10D800008093441290934512A0934612B09347120E
:10D810000E949F5B7F7380916102909162026827F2
:10D82000792770936202609361026DC087E38093F1
:10D83000FB0C80E80E9407880E94F187882329F169
:10D8400088E00E9407880E94DE878830F1F480E13A
:10D850000E9407880E94DE87182F8031B1F480E093
:10D860000E9407880E94DE8781110FC041E050E0CE
:10D87000BE016F5F7F4F89E390E00E9488868981B7
:10D88000843019F41093FC0C13CF83E38093FB0CCA
:10D8900080E80E9407880E94F187882371F180E167
:10D8A0000E9407880E94DE87803139F582E10E945C
:10D8B00007880E94DE87823101F580E00E94078898
:10D8C0000E94DE87811119C084E08093FC0C15E56D
:10D8D000188741E050E0BE01685F7F4F8BE190E028
:10D8E0000E9430871F8341E050E0BE01695F7F4F97
:10D8F0008AE190E00E943087DBCE1092FB0C0E9400
:10D90000958910E000E0C80128960FB6F894DEBFB4
:10D910000FBECDBFDF91CF911F910F9108952FB70B
:10D92000F89460917716709178168091791690919D
:10D930007A162FBF0895CF92DF92EF92FF92CF9386
:10D94000DF938091F412883050F0CFEFDFEFCE01FB
:10D95000DF91CF91FF90EF90DF90CF900895E0910D
:10D960001913E11142C00E948F6C6B017C0128EEFB
:10D97000C20E23E0D21EE11CF11C88EE92E10E944F
:10D98000B28D882311F380914F13882331F0809159
:10D990001A1390911B13892BC1F288EE92E10E9419
:10D9A000158CEC01CF3FDC0771F080914F13882379
:10D9B00071F280911A1390911B13019790931B138E
:10D9C00080931A13C4CF0E948F6CC616D706E80640
:10D9D000F90698F61092191388EE92E10E940D8EC6
:10D9E00088EE92E10E94D48DB2CFE150E0931913FA
:10D9F0000E2E000CFF0BE252FD4EC38DD0E0A7CFE0
:10DA00000F931F93CF93DF93EC018C01F801819169
:10DA10008F018823C1F10E949B6CF8012291022E94
:10DA2000000C330B8217930789F38F3F980791F00F
:10DA3000A091191391E09A0F909319130A2E000CDC
:10DA4000BB0BA252BD4E5B968C93903219F48FE1C2
:10DA5000809319132FE1EC17FD07D9F092919F3FA6
:10DA6000D1F3A091191381E08A0F809319130A2E24
:10DA7000000CBB0BA252BD4E5B969C93803259F7B3
:10DA800020931913E8CF81E0DF91CF911F910F917F
:10DA9000089580E0F9CF0F931F93CF93DF93EC01AC
:10DAA0000E948F6C8B010E940B7B8F3F69F00E945C
:10DAB0008F6C601B710B6C177D07A8F380E0DF9102
:10DAC000CF911F910F91089581E0F9CF4F925F920E
:10DAD0006F927F928F929F92AF92BF92CF92DF927E
:10DAE000EF92FF920F931F93CF93DF93CDB7DEB7E3
:10DAF00063970FB6F894DEBF0FBECDBF7C016B01FC
:10DB00003A01FB0120E090E080E06AE031913323AC
:10DB100009F461C040ED430F4A3008F04DC0689FE2
:10DB2000A001699F500D1124CA01C097830F911D58
:10DB300037FD9A958F3F910549F340F3F7014281F4
:10DB40005381648175818091971790919817A09166
:10DB50009917B0919A17481759076A077B0709F474
:10DB60000DC28701085F1F4F0E948F6C6F7077276F
:10DB70007C5FC8010E94658F813009F004C280E299
:10DB800094E09A838983F70182819381A481B5818E
:10DB90008B839C83AD83BE8345E350E0BE016F5F02
:10DBA0007F4FC8010E94EE8F892BA9F5D12CC12C83
:10DBB000C8010E94918C17C03E3209F0BFCF2330BC
:10DBC00009F4BCCFD301A20FB11D12968C932F5F25
:10DBD00090E080E09BCF233009F0B0CFF301858344
:10DBE000CC24C394D12CC60163960FB6F894DEBF43
:10DBF0000FBECDBFDF91CF911F910F91FF90EF909E
:10DC0000DF90CF90BF90AF909F908F907F906F905C
:10DC10005F904F9008950E948F6CF7017783668321
:10DC200042E050E0B7016A5F7F4FC8010E94838FD6
:10DC300081E090E09A83898342E050E0BE016F5F0B
:10DC40007F4FC8010E94838F80E091E09A8389838F
:10DC500042E050E0BE016F5F7F4FC8010E94838F9A
:10DC60001A82198242E050E0BE016F5F7F4FC80107
:10DC70000E94838F42E050E0BE016F5F7F4FC8017A
:10DC80000E94838F42E050E0BE016F5F7F4FC8016A
:10DC90000E94838F5601F6018081882301F165017E
:10DCA000F60181912F01882311F08E32B1F44601E3
:10DCB0008A189B081814190474F48D8641E050E00A
:10DCC000BE01635F7F4FC8010E94838FA401B5012D
:10DCD000C8010E94838F5201DECF6201E1CF1D8611
:10DCE00041E050E0BE01635F7F4FC8010E94838F17
:10DCF000C12CDD24D394DA82C98242E050E0BE0117
:10DD00006F5F7F4FC8010E94838FDA82C98242E031
:10DD100050E0BE016F5F7F4FC8010E94838FC80132
:10DD20000E94BD8F892B09F441CFF3E0AF2EB12CB7
:10DD3000230122E0420E511CD4C0F70142815381DD
:10DD400064817581808D918DA28DB38D481759079F
:10DD50006A077B0709F008C1848D958DC59709F086
:10DD600003C181A192A15DEFC52EDD24DA940C9749
:10DD70000CF4ADC04CE050E0BE016F5F7F4FC801B6
:10DD80000E94708B8B819C819827892798279A8B7A
:10DD9000898BF7014681578129813A8142175307C0
:10DDA00009F0E7C097FFE5C08F7092703BEFC32E7C
:10DDB000DD24DA94892B09F08AC06F807884762478
:10DDC000672476242AEFC22EDD24DA9461147104CC
:10DDD00009F47DC0D12CC12C8D819E819827892783
:10DDE0009827C816D906F8F441E050E0BE01635FF9
:10DDF0007F4FC8010E94708B4D85442331F050E065
:10DE000070E060E0C8010E94708B8D858111ECCFBD
:10DE100044E050E070E060E0C8010E94708BFFEFCA
:10DE2000CF1ADF0AD9CF912C812C41E050E0BE01FE
:10DE30006D5E7F4FC8010E94708B4B89842F807C60
:10DE400009F06CC0442331F050E070E060E0C8019C
:10DE50000E94708B8B898111E8CF42E050E0BE01B7
:10DE6000615F7F4FC8010E94708B42E050E0BE01AD
:10DE7000635F7F4FC8010E94708B44E050E070E008
:10DE800060E0C8010E94708B42E050E0BE016F5E0E
:10DE90007F4FC8010E94708B8F85988949895A8964
:10DEA0008115914009F043C0CD84DE84DC24CD246B
:10DEB000DC2481E0C816D104D1F54115544009F0A5
:10DEC0004AC044E050E0B201C8010E94708B21E0DA
:10DED000A21AB10809F46CCEFFEFCF16DF0609F0E5
:10DEE00067CE0E948F6C3B014C01C8010E94B98B28
:10DEF000181619060CF421CF0E948F6C6619770949
:10DF000088099909693873418105910548F562E3EB
:10DF100070E080E090E00E94C069E7CF41E050E00F
:10DF200070E060E0C8010E94708B1B8A93CF542779
:10DF30004527542770E060E0C8010E94708BFFEF16
:10DF40008F1A9F0A6814790409F06FCF96EFC92ED3
:10DF5000DD24DA94BCCFE7EFCE2EDD24DA94B7CF00
:10DF6000CC24CA94DC2CB3CF6EEFC62EDD24DA9419
:10DF7000AECF4CEFC42EDD24DA94A9CF8EEFC82E9D
:10DF8000DD24DA9430CED12CC12C2DCE1F920F92ED
:10DF90000FB60F9211242F933F938F939F93AF93BC
:10DFA000BF938091771690917816A0917916B091D1
:10DFB0007A163091761623E0230F2D3758F5019607
:10DFC000A11DB11D20937616809377169093781635
:10DFD000A0937916B0937A1680917B1690917C1657
:10DFE000A0917D16B0917E160196A11DB11D809362
:10DFF0007B1690937C16A0937D16B0937E16BF91EE
:10E00000AF919F918F913F912F910F900FBE0F90E5
:10E010001F90189526E8230F0296A11DB11DD2CF9F
:10E02000CF92DF92EF92FF92CF93DF93EC016032B9
:10E0300082E07807CCF5653B710514F064EB70E085
:10E04000898128E830E0281B310987FD3395220FAC
:10E05000331F220F331F6901330FEE08FF088A8137
:10E0600028E532E0281B310987FD3395220F331F45
:10E07000220F331F032E000C440B550B2C193D09A6
:10E080004E095F09DB0177FF02C0B0E0A0E00E940B
:10E0900001B924EB30E040E050E00E94D7B8C20E56
:10E0A000D31EE41EF51EB601E881E03370F5298128
:10E0B00088E890E0821B910927FD9395880F991FAE
:10E0C000880F991F681779077CF02A8188E592E00C
:10E0D000821B910927FD9395880F991F880F991F1F
:10E0E000681779070CF4CB010297880F991F4FB777
:10E0F000F8942E2F30E0F901EE0FFF1FE20FF31F0F
:10E10000E85BFD4E928381834FBFDF91CF91FF90FB
:10E11000EF90DF90CF9008951F93CF93DF93EC01A2
:10E12000162F8881803308F04EC061E0812F0E9455
:10E130008F698881282F30E0F901EE0FFF1FE20F71
:10E14000F31FE85BFD4E1F736081607C612B608371
:10E1500019821A822CE0622F0E9437BA829FB00186
:10E16000112430E020E0AB01420F531FFA01EE0F03
:10E17000FF1FE40FF51FE85BFD4E908196FD16C072
:10E180002F5F3F4F2C30310571F7813009F5109228
:10E19000800082E0809381001092850010928400BC
:10E1A000B19A80916F00826080936F00E8818E2F1A
:10E1B00090E0FC01EE0FFF1FE80FF91FE85BFD4E3A
:10E1C0008081806480838881DF91CF911F91089541
:10E1D000823061F41092900080939100109295002B
:10E1E0001092940088BB80937100E0CF833069F473
:10E1F0001092A00082E08093A1001092A5001092DE
:10E20000A40089BB80937200D1CF8111CFCF10922F
:10E21000200182E0809321011092250110922401B7
:10E220008ABB80937300C2CF1F920F920FB60F92DA
:10E2300011240BB60F922F933F934F935F936F93DD
:10E240007F938F939F93AF93BF93EF93FF9348E296
:10E2500051E064E271E090E080E00E94D568FF91B7
:10E26000EF91BF91AF919F918F917F916F915F914E
:10E270004F913F912F910F900BBE0F900FBE0F90BB
:10E280001F9018951F920F920FB60F9211240BB684
:10E290000F922F933F934F935F936F937F938F933F
:10E2A0009F93AF93BF93EF93FF9348EA50E064EAE4
:10E2B00070E083E090E00E94D568FF91EF91BF91FC
:10E2C000AF919F918F917F916F915F914F913F910E
:10E2D0002F910F900BBE0F900FBE0F901F901895AF
:10E2E0001F920F920FB60F9211240BB60F922F931D
:10E2F0003F934F935F936F937F938F939F93AF93CE
:10E30000BF93EF93FF9348E950E064E970E082E047
:10E3100090E00E94D568FF91EF91BF91AF919F91DE
:10E320008F917F916F915F914F913F912F910F90BE
:10E330000BBE0F900FBE0F901F9018951F920F925B
:10E340000FB60F9211240BB60F922F933F934F935A
:10E350005F936F937F938F939F93AF93BF93EF934D
:10E36000FF9348E850E064E870E081E090E00E94AC
:10E37000D568FF91EF91BF91AF919F918F917F9160
:10E380006F915F914F913F912F910F900BBE0F9026
:10E390000FBE0F901F901895FC01248131E030933F
:10E3A000540F2093760F1092550F1092770F83859C
:10E3B000862B90E00E94405D81E00C94505C0F93AE
:10E3C0001F93CF938C01C62F0E94CC716C2F646079
:10E3D000C8010E94CC716C2F6B7FC8010E94CC7168
:10E3E00083EC90E00197F1F7CF911F910F91089581
:10E3F000CF93C82F682F607F82E596E10E94DF717E
:10E4000080E1C89FB001112482E596E1CF910C9480
:10E41000DF71CF93DF9300D000D01F921F92CDB752
:10E42000DEB798E0EBE4F3E0DE01119601900D9287
:10E430009A95E1F790915B16961708F46FEF70E0EC
:10E44000660F771F21E030E02C0F3D1F620F731F16
:10E45000FB019081890F806828960FB6F894DEBF83
:10E460000FBECDBFDF91CF910C94F8710F931F9326
:10E47000CF93DF9320919102222321F120919002EA
:10E48000222301F1EB018C0161E080E00E9409721E
:10E49000B80182E596E10E94DC6663E37CE082E5F8
:10E4A00096E10E94FE6661E0F80184810E94097293
:10E4B000BE01DD0F880B990BDF91CF911F910F915A
:10E4C0000C94C069DF91CF911F910F9108950F9324
:10E4D0001F93CF938C01C62F607F61600E94DF7114
:10E4E00080E1C89FB00111246160C8010E94DF7102
:10E4F00081E090E0CF911F910F91089560936E1687
:10E5000070936F168093701690937116645D7E4FB2
:10E510008F4F9F4F60936A1670936B1680936C16A3
:10E5200090936D1682E090E0909369168093681640
:10E530000E948F6C609364167093651680936616C4
:10E54000909367160895CF92DF92EF92FF920F9308
:10E550001F930E948F6C8B019C01C0906416D09019
:10E560006516E0906616F090671660916E167091D1
:10E570006F1680917016909171160C191D092E0955
:10E580003F09083E134021053105E0F0DC01CB01D5
:10E590000196A11DB11D80936E1690936F16A093E6
:10E5A0007016B0937116B701A60148515C4F6F4FBA
:10E5B0007F4F409364165093651660936616709370
:10E5C0006716C7CF1F910F91FF90EF90DF90CF900C
:10E5D00008950E94A3720E94CB778091840C90E0F2
:10E5E0008E54984F08950E94A3720E94CB77809119
:10E5F000830C90E008950E94A3720E94CB778091D3
:10E60000820C90E008950E94A3720E94CB778091C3
:10E610007F0C90E008950E94A3720E94CB778091B6
:10E62000800C90E008952F923F924F925F926F92EC
:10E630007F928F929F92AF92BF92CF92DF92EF9292
:10E64000FF920F931F93CF93DF93CDB7DEB7C756DB
:10E65000D1090FB6F894DEBF0FBECDBF5C013B0100
:10E66000A6964FAFA6974E018EE1880E911C63E2ED
:10E6700072E1C4010E94DB851C821B8280E893E06A
:10E680009A8389831E8263018E010F5F1F4F2401CD
:10E6900018016FE270E0C6010E94BCBC009709F44B
:10E6A00059C0F60120812F3271F4FFEFCF1ADF0A33
:10E6B000902F812F8201492E582E942D852D2801CF
:10E6C000092F182FE6CF8C198D3008F08CE0E82E3A
:10E6D000F12CA701B601CE01885A9F4F0E94E5BCDC
:10E6E000E8E5F0E0EC0FFD1FEE0DFF1D1082C80104
:10E6F0000E94FD8121E0AE01485A5F4FB201C8017E
:10E700000E941182811120C01EAE1DAE80E893E0F0
:10E710009CAF8BAF21961FAE2197A896EEADFFADB3
:10E72000A8976E0E7F1EF3018081811120C0BE016B
:10E73000655C7F4FC1010E94DB854CE754E0B1016D
:10E74000C5010E94498631C0CE0CDF1CC2010E9467
:10E75000FD81B3CFC60186199709A8969FAF8EAFEA
:10E76000A897B201CE01CB960E94DB85D6CF19A225
:10E7700018A280E893E09F8F8E8F1BA221968FAD09
:10E78000219781112DC0F5011382128288EE93E04A
:10E79000A0E0B0E084839583A683B78382E094E011
:10E7A00091838083128E118E1486C501C959DF4F63
:10E7B0000FB6F894DEBF0FBECDBFDF91CF911F9192
:10E7C0000F91FF90EF90DF90CF90BF90AF909F9010
:10E7D0008F907F906F905F904F903F902F90089513
:10E7E0008250A6962FADA697A3018230C8F463E2AB
:10E7F00072E1C4010E941182882329F2A6968FAD8E
:10E80000A697867039F049A95AA96BA97CA9C401B9
:10E810000E94F47EB401C1010E94DB85A3018FCF69
:10E82000BE01655C7F4FC4010E941182882309F4F8
:10E83000AACFCE01CB960E94FD81E0CF0F931F930C
:10E84000CF93DF93CDB7DEB7AD970FB6F894DEBFA9
:10E850000FBECDBF8091030D882331F08091EE1360
:10E860009091EF13892B11F40E94A22A66E279E0BD
:10E87000CE0188960E9493658091020D8823E1F075
:10E8800062E27CE0CE0101960E948165CE01019694
:10E890000E94D509CE0101960E94FA6469E672E0F1
:10E8A000CE0101960E949365CE0101960E94BE0999
:10E8B000CE0101960E94FA648091030D81111BC064
:10E8C0008091010D81117BC08091000D882309F496
:10E8D00049C10FE110E08091FF0C882309F4BAC010
:10E8E0000150110909F45CC064E170E080E090E03F
:10E8F0000E94C069F0CF8091EE139091EF13892BA5
:10E90000F9F264E170E080E090E00E94C06964E1A7
:10E910007CE0CE0188960E9485646AEE73E1CE01A8
:10E9200001960E948A65AE014F5F5F4F63E070E021
:10E9300089E692E00E949614182FCE0101960E945B
:10E94000FA64111127C0BE01685D7F4FCE014C965D
:10E950000E948A656CEC73E1CE014C960E941564AE
:10E96000BC01CE0101960E948A65CE0101960E94EB
:10E97000BE09CE0101960E94FA64CE014C960E9417
:10E98000FA6480916F1790917017019690937017A9
:10E9900080936F171092030D8091010D811190CF1C
:10E9A000CE0188960E94FA64AD960FB6F894DEBF49
:10E9B0000FBECDBFDF91CF911F910F910895809130
:10E9C000E2139091E313892B09F47ECF66E07CE09B
:10E9D000CE0188960E9485646EED73E1CE010196AA
:10E9E0000E948A65AE014F5F5F4F62E070E083E88E
:10E9F00092E00E949614182FCE0101960E94FA64AC
:10EA0000111162CFBE01685D7F4FCE014C960E940E
:10EA10008A656CEC73E1CE014C960E941564BC01D2
:10EA2000CE0101960E948A65CE0101960E94BE0920
:10EA3000CE0101960E94FA64CE014C960E94FA64BF
:10EA400080916F1790917017019690937017809333
:10EA50006F173ACF43E166E772E0CE0101960E945C
:10EA60001373BE016F5F7F4F86E396E10E94670CD0
:10EA700081E08093FF0C86E396E10E942B86882339
:10EA8000E1F16AEE73E186E396E10E94EA6686E3CD
:10EA900096E10E94378662E370E080E090E00E9499
:10EAA000C0691092FF0C8091020D882331F1CE01D4
:10EAB0004C960E948E0E6BE379E0CE0182960E9406
:10EAC0009365BE01645E7F4FCE0182960E941564FD
:10EAD000BC01CE0101960E948A65CE0101960E947A
:10EAE000BE09CE0101960E94FA64CE0182960E9470
:10EAF000FA64CE014C960E94FA6486E396E10E9485
:10EB0000378662E370E080E090E00E94C069109276
:10EB1000FF0C43E163E872E0CE0101960E9413739B
:10EB2000BE016F5F7F4F86E396E10E94670C81E034
:10EB30008093FF0C86E396E10E942B86882331F0B8
:10EB40006EED73E186E396E10E94EA6686E396E164
:10EB50000E94378662E370E080E090E00E94C06926
:10EB60001092FF0C66E279E08EED93E10E94CE6296
:10EB700066E279E08AEE93E10E94CE6211CF2091A5
:10EB8000CA17260F3327331F21323105ECF42091A9
:10EB90004E0FFC0190E080E0243069F082E008959F
:10EBA000A091CA172191AC014655584EA40FB52F1C
:10EBB000B11D2C930196861798F38091CA17680FA0
:10EBC0006093CA1780E0089581E00895089508953C
:10EBD0000895E091F50C8091F40CE81730F4F0E022
:10EBE000E85FF04F808190E008958FEF9FEF0895E8
:10EBF0009091F50C8091F40C2FEF3FEF981748F4AB
:10EC0000E92FF0E0E85FF04F208130E09F5F9093C4
:10EC1000F50CC90108958091F40C9091F50C891BB5
:10EC2000990B0895CF92DF92EF92FF920F931F936B
:10EC3000CF93DF937C01CB018A012091540F2223D3
:10EC400089F0EB016B01C40ED51ECC15DD0569F012
:10EC50006991D701ED91FC910190F081E02DC70100
:10EC60001995F3CF642F0E94BF75C801DF91CF9132
:10EC70001F910F91FF90EF90DF90CF900895CF9369
:10EC8000DF931F92CDB7DEB769832091540F222303
:10EC9000F9F02091770F203258F021E030E0FC01AC
:10ECA0003383228390E080E00F90DF91CF9108952D
:10ECB0008091550FE82FF0E0EA5AF04F9981908348
:10ECC0008F5F8093550F8093770F81E090E0ECCFBA
:10ECD00061E0CE0101960E94BF75F7CF8EBD0DB4E5
:10ECE00007FEFDCF0895DC015996ED91FC91309718
:10ECF000B9F083899489A589B6894285538564854D
:10ED00007585841B950BA60BB70B811520E8920720
:10ED1000A105B10538F08FEF9FE7A0E0B0E00895BE
:10ED200090E080E00895CF93DF931F92CDB7DEB7D8
:10ED30006983DC01ED91FC910280F381E02D41E0DB
:10ED400050E0BE016F5F7F4F19950F90DF91CF911B
:10ED50000895FC0120812EBD9B012150310941F015
:10ED600051810DB407FEFDCF4EB55EBD4193F5CF89
:10ED700061507109860F971F0DB407FEFDCF2EB5A8
:10ED8000FC0120830895E091F90CF091FA0C908138
:10ED90008091F80C80958923808308958EBD0000B2
:10EDA0000DB407FEFDCF8EB5089590E02091FB0CC9
:10EDB000233339F40C96982F990F990F990F80E00F
:10EDC00008954896F8CFCF93DF931F92CDB7DEB763
:10EDD0006983DC01ED91FC910280F381E02D41E03B
:10EDE00050E0BE016F5F7F4F19950F90DF91CF917B
:10EDF0000895FC01818D928D0895CF93DF931F922A
:10EE0000CDB7DEB76983DC01ED91FC910280F3811F
:10EE1000E02D41E050E0BE016F5F7F4F19950F90EC
:10EE2000DF91CF910895FC019485FB0184859813AF
:10EE300003C081E0983008F080E00895CF93DF931D
:10EE40001F92CDB7DEB76983DC01ED91FC910280A2
:10EE5000F381E02D41E050E0BE016F5F7F4F1995D7
:10EE60000F90DF91CF91089561E0FC0184810C94B3
:10EE7000A768CF93DF93EC018FEF8EBD2FEF8F81CB
:10EE80009885AC014F5F5F4F58874F838130924028
:10EE900028F40DB407FEFDCF2EBDF1CF0DB407FE53
:10EEA000FDCFCE010E9434771E82DF91CF9108956D
:10EEB000CF92DF92EF92FF920F931F93CF93DF9346
:10EEC000CDB7DEB7AF970FB6F894DEBF0FBECDBF9C
:10EED0007C016A0100E214E01A8309831C861B8608
:10EEE00088EE93E0A0E0B0E08D879E87AF87B88B77
:10EEF0008AEA93E09A878987188F0F8B198E1A8E6A
:10EF00001B8E1C8E88E089A31BA70AA71CA61DA622
:10EF10001EA61FA68091441290914512A091461200
:10EF2000B09147128EA39FA3A8A7B9A78B839C83F8
:10EF3000AD83BE8318861F82AE01465D5F4FCE0152
:10EF400001960E94666D81309105B1F4D701ED9173
:10EF5000FC910488F589E02D1DA30CA38CA59DA52B
:10EF6000AEA5BFA58EA39FA3A8A7B9A7A601BE0162
:10EF70006C5D7F4FC7011995AF960FB6F894DEBF51
:10EF80000FBECDBFDF91CF911F910F91FF90EF90FA
:10EF9000DF90CF9008954F925F926F927F928F9201
:10EFA0009F92AF92BF92CF92DF92EF92FF920F9318
:10EFB0001F93CF93DF934B015C018091BE1890911A
:10EFC000BF18A091C018B091C11888159905AA055D
:10EFD000BB0509F4C6C08CE3C82ED12CE12CF12C62
:10EFE000C501A70196010E94B5B860937E0CCA01C5
:10EFF000B901A70196010E94B5B860937F0CC501C5
:10F00000B40120E13EE040E050E00E94B5B8CA0102
:10F01000B90128E130E040E050E00E94B5B86093CB
:10F02000800CC501B40120E831E541E050E00E94C8
:10F03000B5B869017A01CA01B9016C5F7F4F8F4F82
:10F040009F4F27E030E040E050E00E94B5B86F5F8E
:10F050006093810C412C512C320140E004E610E019
:10F06000C0E9D1E0242F30E02E54384FF901E3708D
:10F07000FF273097F9F4C901B8010E9443BA892BE0
:10F0800031F4C901BE010E9443BA892B99F48EE67E
:10F0900091E0A0E0B0E0480E591E6A1E7B1ED3012D
:10F0A000C201AA27BB27C816D906EA06FB0638F014
:10F0B0004F5FD8CF8DE691E0A0E0B0E0ECCF409379
:10F0C000840CC90164E670E00E9443BAEC01C901F6
:10F0D00060E971E00E9443BA309721F42097D9F497
:10F0E0000097C9F04DE651E060E070E0441A550A1F
:10F0F000660A770AC418D508E608F708A6E4B4E05B
:10F1000020E0213069F43097E9F5209711F4009759
:10F11000C9F54DE106C04EE651E060E070E0E6CF93
:10F120004C9150E070E060E031E0320FC416D5063B
:10F13000E606F70640F0C41AD50AE60AF70A119661
:10F14000232F3C30F1F62F5F2093830CC394C092A1
:10F15000820C8092BE189092BF18A092C018B092F4
:10F16000C118DF91CF911F910F91FF90EF90DF9029
:10F17000CF90BF90AF909F908F907F906F905F9057
:10F180004F9008954CE1CDCF1F920F920FB60F9282
:10F1900011240BB60F922F933F934F935F936F936E
:10F1A0007F938F939F93AF93BF93EF93FF93809140
:10F1B000EE170E947E682091F1173091F2172F5FB1
:10F1C0003F4F3093F2172093F1179091F017953637
:10F1D00018F096E09093ED179091ED17943009F4A4
:10F1E0006EC0F8F4923031F1933009F44CC0909134
:10F1F000EF17992319F0811171C02F9AFF91EF91A8
:10F20000BF91AF919F918F917F916F915F914F913E
:10F210003F912F910F900BBE0F900FBE0F901F903C
:10F220001895953009F457C0963009F791E09093FE
:10F23000BD184FC08111DBCF2091F1173091F2172B
:10F240002436310528F41092F2171092F117CFCF1F
:10F250001092BD181092F017E091F01791E09E0FF8
:10F260009093F017F0E02091F1173091F217EE0F24
:10F27000FF1FED50F84E318320831092F217109249
:10F28000F11793E019C0813009F0B1CFE091F01788
:10F2900091E09E0F9093F017F0E02091F1173091DC
:10F2A000F217EE0FFF1FED50F84E318320831092BE
:10F2B000F2171092F11794E09093ED1798CF8823EE
:10F2C00059F22091F1173091F2172536310508F4E3
:10F2D0008ECF95E0F1CF81118ACFB5CF2F988ECF09
:10F2E00010924E0F81E080934D0F1092280F61E035
:10F2F00084E10E94A76861E085E10E94A768E9EBCC
:10F30000F0E080818E7F808380818D7F808388E4A0
:10F310008093B80085E48093BC000895CF93DF9379
:10F3200091E09093A9178823B9F0C091B800D091CB
:10F33000BA008091BC008A7B8093BC0060E084E1CD
:10F340000E94A76860E085E10E94A7680E9470792A
:10F35000D093BA00C093B800DF91CF91089585EDA6
:10F360008093BC008091500F9091510FA091520F4B
:10F37000B091530F0796A11DB11D23E0B695A79537
:10F38000979587952A95D1F72091BC0024FD03C05D
:10F3900010924E0F08954091500F5091510F60916F
:10F3A000520F7091530F452B462B472B69F3009753
:10F3B000A105B10541F025E32A95F1F70000019779
:10F3C000A109B109E1CF80914F0F0C948E791F9262
:10F3D0000F920FB60F9211240BB60F922F933F93FB
:10F3E0004F935F936F937F938F939F93AF93BF934D
:10F3F000EF93FF938091B900887F803609F44DC068
:10F4000008F040C0883209F4A9C028F5803109F419
:10F410009DC0C8F4882309F4FBC0883009F496C065
:10F42000FF91EF91BF91AF919F918F917F916F91DC
:10F430005F914F913F912F910F900BBE0F900FBE98
:10F440000F901F901895883109F488C0803241F7D9
:10F4500080934C0F14C0803409F49DC040F4803375
:10F46000B9F38833E9F680934C0F85ECB0C0803552
:10F4700009F485C0883509F496C0883489F60E945D
:10F48000AF79CECF883909F48CC038F5883729F0A8
:10F4900050F4883611F0803719F683E080934E0FD0
:10F4A0001092EC1757C0883809F47BC0803919F0E6
:10F4B000803809F0B5CF8091EC17803208F071C028
:10F4C000E091EC1781E08E0F8093EC178091BB00E8
:10F4D000F0E0E453F84E80833DC0803B39F0E0F427
:10F4E000803A09F479C0883A09F09ACF84E0809391
:10F4F0004E0F1092CB171092CA17E091F20CF091B8
:10F50000F30C19958091CA1781110FC081E0809387
:10F51000CA171092AA1709C0803C09F4A6CF883CEC
:10F5200009F4A3CF883B09F07BCFE091CB1781E0B2
:10F530008E0F8093CB17F0E0E655F84E80818093D4
:10F54000BB009091CB178091CA1729C08091290FD9
:10F550008093BB0085EC8093BC0062CF90914B0FF1
:10F5600080914A0F981758F5E0914B0F81E08E0F6C
:10F5700080934B0FF0E0E65DF04F8081E9CFE091A2
:10F580004B0F81E08E0F80934B0F8091BB00F0E01A
:10F59000E65DF04F808390914B0F80914A0F981752
:10F5A000C8F285E8D8CFE0914B0F81E08E0F8093B1
:10F5B0004B0F8091BB00F0E0E65DF04F80838091BF
:10F5C0004D0F81115CCF81E08093280F84EA8093F6
:10F5D000BC0010924E0F24CF85EC8093BC0010929B
:10F5E0004E0F8091EC17803230F4E091EC17F0E090
:10F5F000E453F84E10826091EC1770E0E091F00C4B
:10F60000F091F10C8CEC97E119951092EC1708CF62
:10F6100010924C0F34CF8FEF0E946E768EB5089506
:10F620008F929F92AF92BF92FF920F931F93CF93AF
:10F63000DF93EC01F62E49015A018E81882319F0DF
:10F64000CE010E94397760E08C810E94A7688CE22D
:10F6500091E00E944B6D8F2D80640E946E7608E1D0
:10F6600010E0D501C401002E04C0B695A79597956A
:10F6700087950A94D2F70E946E7608501109083FC8
:10F680008FEF180771F785E9FF2021F088E0F81265
:10F690000DC087E80E946E7610E00E940B7B8A877F
:10F6A00087FF06C01F3F21F01F5FF7CF8FEFF2CF1C
:10F6B000DF91CF911F910F91FF90BF90AF909F90DE
:10F6C0008F900895AF92BF92CF92DF92EF92FF9208
:10F6D0000F931F93CF93DF93EC016901C801820F51
:10F6E000931F8130924050F58E81882379F0888174
:10F6F0009981AA81BB8184179507A607B70731F4C2
:10F700008F819885C816D90608F042C0488359836E
:10F710006A837B838B85833039F089E0440F551FE2
:10F72000661F771F8A95D1F79A01AB0161E1CE017F
:10F730000E94107B882389F083E08D83CE010E9494
:10F74000347780E0DF91CF911F910F91FF90EF9080
:10F75000DF90CF90BF90AF9008950E948F6C5B01B7
:10F760000E940B7B8A878F3F69F40E948F6C6A1915
:10F770007B096D327140A0F38FE08D83CE010E9432
:10F780003477DCCF8E3FB1F418861F8281E08E8300
:10F790008FEF8EBD2FEF8F8198858C159D0560F4BE
:10F7A0000DB407FEFDCF2EBD8F81988501969887F9
:10F7B0008F83F1CF8DE0E1CFC8010197F7012FEFE3
:10F7C000AF014E195F094817590738F40DB407FE09
:10F7D000FDCF3EB531932EBDF3CF0DB407FEFDCF67
:10F7E0002EB5E80EF91EF70120838F819885080F4A
:10F7F000191F18870F838985882319F00115124076
:10F8000030F08E81882319F0CE010E94397781E093
:10F8100099CF0F931F93CF93DF93EC01890182E17E
:10F82000411551056105710599F08B85833039F0DB
:10F8300089E0440F551F661F771F8A95D1F79A01FB
:10F84000AB0168E1CE010E94107B882319F084E0AF
:10F850008D8338C08EEF8EBDF801C8019E5F0DB458
:10F8600007FEFDCF20812EBD0DB407FEFDCF218107
:10F870002EBD3296E817F90791F70DB407FEFDCFBC
:10F880008FEF0E946E768FEF0E946E760E940B7B48
:10F890008A878F71853089F488E592E00E944B6DEC
:10F8A0008823A9F020E030E0A9016DE0CE010E949C
:10F8B000107B882371F084E1CBCF81E18D83CE0171
:10F8C0000E943477CE010E94347780E00AC085E13F
:10F8D000BFCF0E940B7B8111EECFCE010E94347707
:10F8E00081E0DF91CF911F910F9108958091A4172E
:10F8F0008823A9F14091DF025091E0026091E1027A
:10F900007091E20224E03DE08091F60C9091F70CBA
:10F910000E94097C811102C080E008954091A517E2
:10F920005091A6176091A7177091A817411551051E
:10F930006105710591F024E03DE08091F60C909115
:10F94000F70C0E94097C882339F31092A5171092B6
:10F95000A6171092A7171092A8171092A41781E06B
:10F9600008958F929F92AF92BF92EF92FF920F9362
:10F970001F93CF934B015C01C42F8091DF029091C4
:10F98000E002A091E102B091E20288159905AA0572
:10F99000BB0549F10E94767C81110BC080E0CF91BC
:10F9A0001F910F91FF90EF90BF90AF909F908F901D
:10F9B000089584E0E82E8DE0F82E00E012E030E0BB
:10F9C00020E0B501A4018091F60C9091F70C0E9403
:10F9D000627B882319F38092DF029092E002A0926A
:10F9E000E102B092E2024091A4174C2B4093A4177D
:10F9F00081E0D5CF4F925F926F927F928F929F92CC
:10FA0000AF92BF92CF92DF92EF92FF920F931F932C
:10FA1000CF93DF93EC01423051056105710590F4FD
:10FA200080E0DF91CF911F910F91FF90EF90DF90D9
:10FA3000CF90BF90AF909F908F907F906F905F908E
:10FA40004F90089589859A85AB85BC850196A11D47
:10FA5000B11D84179507A607B70710F3CB88DC887C
:10FA6000ED88FE888F89803109F042C0BB27A72F1F
:10FA7000962F852F480159012A013B01C80ED91E36
:10FA8000EA1EFB1E8091DF029091E002A091E1024C
:10FA9000B091E202C816D906EA06FB0699F58F89ED
:10FAA0008031C1F5B301A201552766277727440F9E
:10FAB000551F4C5F524FFA01918280828091A417AA
:10FAC00081608093A4178A89823080F08D819E8125
:10FAD000AF81B8858C0D9D1DAE1DBF1D8093A517F0
:10FAE0009093A617A093A717B093A81781E099CF7A
:10FAF000DB01CA01E7E0B695A79597958795EA954A
:10FB0000D1F7B8CF40E0C701B6010E94B17C8111A6
:10FB1000C6CF86CFB301A2014F7755276627772737
:10FB2000440F551F440F551F4C5F524FFA018082FE
:10FB30009182A282B382C2CF8F929F92AF92BF92E4
:10FB4000CF92DF92EF92FF920F931F93CF93DF93A9
:10FB5000FC0181859285A385B4850196A11DB11D07
:10FB600084179507A607B70770F480E0DF91CF915F
:10FB70001F910F91FF90EF90DF90CF90BF90AF90CB
:10FB80009F908F90089583889488A588B6888789E8
:10FB9000803189F5BB27A72F962F852FE9016A01B0
:10FBA0007B018F01BC01CD01680D791D8A1D9B1D54
:10FBB0008090DF029090E002A090E102B090E2021B
:10FBC00086169706A806B90601F5F80187898031DF
:10FBD00011F5DD24EE24FF24F601EE0FFF1FEC5F8C
:10FBE000F24F80819181B0E0A0E088839983AA835D
:10FBF000BB8381E0BBCFDB01CA01C7E0B695A79507
:10FC000097958795CA95D1F7C9CF40E00E94B17CFE
:10FC10008111DBCFAACFE894C7F8DD24EE24FF24BE
:10FC2000F601EE0FFF1FEE0FFF1FEC5FF24F80811A
:10FC30009181A281B381BF70D8CF4F925F926F92B2
:10FC40007F92AF92BF92CF92DF92EF92FF920F938B
:10FC50001F93CF93DF9300D01F92CDB7DEB78C01F7
:10FC600049835A836B837C835901C12CD12C760143
:10FC7000412C82E0582E612C712C49815A816B8174
:10FC80007C819E012F5F3F4FC8010E949C7D88238D
:10FC900039F1F8018585A301920104C0220F331FB9
:10FCA000441F551F8A95D2F7DA01C901C80ED91E23
:10FCB000EA1EFB1E49815A816B817C8187898031D4
:10FCC00011F188EF9FEFAFEFBFE0481759076A07C0
:10FCD0007B0798F2F501C082D182E282F38281E053
:10FCE0000F900F900F900F90DF91CF911F910F9178
:10FCF000FF90EF90DF90CF90BF90AF907F906F908C
:10FD00005F904F90089588EF9FEFA0E0B0E0DDCFC7
:10FD1000CF92DF92EF92FF921F93CF93DF93EC018C
:10FD200080E2689FF0011124EC5FF24F938591719E
:10FD300061F0842F827449F080E0DF91CF911F91B0
:10FD4000FF90EF90DF90CF900895142F6A8B8091F1
:10FD5000DF029091E002A091E102B091E2028E8771
:10FD60009F87A88BB98BC488D588F12CE12C7601AC
:10FD7000DD24CC24CF8AD88EE98EFA8E828D938DA5
:10FD8000B0E0A0E0AC01BD014C295D296E297F29BE
:10FD90004F8B588F698F7A8F83858871B1F4848DEA
:10FDA000958DA68DB78D8B8B9C8BAD8BBE8B81E09B
:10FDB0008D831F701C831E821F82188619861A86E7
:10FDC0001B861C861D8681E0B8CF803109F0B4CF38
:10FDD0009E012D5E3F4F8B8D9C8D0E941D7E882342
:10FDE00009F4AACF84E0E4CF8F929F92AF92BF92A2
:10FDF000CF92DF92EF92FF920F931F93CF93DF93F7
:10FE0000EC018D8181110EC080E0DF91CF911F91B7
:10FE10000F91FF90EF90DF90CF90BF90AF909F90A9
:10FE20008F9008950B891C892D893E890417150729
:10FE30002607370748F34A015B01823031F48A868E
:10FE40009B86AC86BD8681E0E0CF81149104A1043D
:10FE5000B10449F41E821F82188619861A861B86F1
:10FE60001C861D86F0CF0A851B852C853D85EB8D74
:10FE7000FC8D858590E00996B901A8014150510992
:10FE800061097109082E04C07695679557954795C5
:10FE90000A94D2F775016401E1E0CE1AD108E108B5
:10FEA000F10804C0F694E794D794C7948A95D2F7E2
:10FEB000C416D506E606F70620F0012B022B032B0D
:10FEC00011F58F89988DA98DBA8D8E839F83A88710
:10FED000B9878E010A5F1F4FC114D104E104F104F8
:10FEE00009F4ADCF4E815F816885798598018B8D4E
:10FEF0009C8D0E949C7D91E0C91AD108E108F1080F
:10FF00008111EACF81CFC41AD50AE60AF70AE1CFF8
:10FF10003F924F925F926F927F928F929F92AF9299
:10FF2000BF92CF92DF92EF92FF920F931F93CF93E6
:10FF3000DF93CDB7DEB72C970FB6F894DEBF0FBEB8
:10FF4000CDBF5C01DC015B968D909C905C97169612
:10FF50004D905D906D907C9019974114510461040F
:10FF6000710409F468C0BFEF4B1A5B0A6B0A7B0A85
:10FF7000312CF40181859285A385B4859C01AD0166
:10FF80002F5F3F4F4F4F5F4F29873A874B875C87E3
:10FF9000730162011D821E821F821886F401818511
:10FFA0009285A385B4852D813E814F815885281780
:10FFB00039074A075B0708F056C089859A85AB85E3
:10FFC000BC858C159D05AE05BF0550F482E0C82E9A
:10FFD000D12CE12CF12C92E0492E512C612C712C6A
:10FFE0009E012F5F3F4FB701A601C4010E949C7D77
:10FFF0008823C9F189819A81AB81BC81892B8A2BA5
:020000021000EC
:100000008B2B09F1260137019FEF491A590A690A1A
:10001000790A2D813E814F8158852F5F3F4F4F4F89
:100020005F4F2D833E834F8358873FEFC31AD30A18
:10003000E30AF30AB3CFF4014080518062807380F9
:100040003324339496CFC414D504E604F70409F797
:100050000FEF1FEF2FEF3FE0B701A601C4010E9491
:10006000FA7C811119C080E02C960FB6F894DEBF9F
:100070000FBECDBFDF91CF911F910F91FF90EF90F9
:10008000DF90CF90BF90AF909F908F907F906F90B8
:100090005F904F903F900895F501468157816085AC
:1000A0007185411551056105710539F0970186018A
:1000B000C4010E94FA7C8823B1F2D5011696CD9234
:1000C000DD92ED92FC921997332051F0D701C601D1
:1000D0000196A11DB11DF40180839183A283B38396
:1000E000F5018789908DA18DB28D892B8A2B8B2B61
:1000F00039F4C78AD08EE18EF28E84818068848341
:1001000081E0B2CF2F923F924F925F926F927F9297
:100110008F929F92AF92BF92CF92DF92EF92FF9217
:100120000F931F93CF93DF93EC015B012A018D8125
:10013000811115C08FEF9FEFDF91CF911F910F912C
:10014000FF90EF90DF90CF90BF90AF909F908F90F7
:100150007F906F905F904F903F902F9008958C818B
:1001600080FFE8CF0B891C892D893E894A855B85F4
:100170006C857D85C201B0E0A0E068017901C41AF8
:10018000D50AE60AF70AC816D906EA06FB0618F4E5
:100190002801441A550A42011E0126E0220E311C94
:1001A0008114910409F4B3C04A855B856C857D8513
:1001B0006A0181E0D8228B8D9C8D8A019B01E9E048
:1001C0003695279517950795EA95D1F7ED81E23099
:1001D000E1F5FC01628D738D848D958D600F711F2B
:1001E000821F931F612C22E0722E6C187D088614EA
:1001F000970408F434012C8126FD04C06114F2E058
:100200007F0671F40091DF021091E0022091E1027B
:100210003091E202061717072807390709F053C083
:1002200040E00E94B17C882309F484CFC6018C5F32
:10023000924FD5019C01260D371DFC012E173F075B
:1002400009F460C041914D93F9CFFC0174807A9418
:100250007022C114D10471F471100CC0452B462BCF
:10026000472B39F58F89988DA98DBA8D8E839F8301
:10027000A887B987EB8DFC8D6E817F8188859985F4
:100280006250710981099109258504C0660F771FA5
:10029000881F991F2A95D2F70685178520893189ED
:1002A000600F711F821F931F670D711D811D911DAE
:1002B00099CF4E815F816885798591010E949C7DEF
:1002C0008111D8CF37CF750183019601AB01BC01F5
:1002D0008091F60C9091F70C0E94627B882309F4C0
:1002E00029CFA60CB71C8A859B85AC85BD85860D5C
:1002F000971DA11DB11D8A879B87AC87BD87861876
:1003000097084ECF281B390BA20EB31EECCFC201AB
:1003100013CFCF93DF931F92CDB7DEB741E050E00C
:10032000BE016F5F7F4F0E948280019731F4898107
:1003300090E00F90DF91CF9108958FEF9FEFF9CF6D
:10034000FC01818D928D009711F00C9489818FEFC3
:100350009FEF08950F931F93CF93DF93EC01898D47
:100360009A8D10E000E0009799F00E9489818C013D
:100370000F3F100769F0898D9A8DFC0142855385E6
:100380006485758541505109610971090E94F47EA7
:10039000C801DF91CF911F910F910895CF93DF9303
:1003A000EC018D81882329F18C8187FF1EC0CE014D
:1003B0000E94145FFC01892BE1F08D81823040F4B2
:1003C0008B899C89AD89BE89848F958FA68FB78FC5
:1003D0008F89988D938F828F8F89988DA98DBA8DF3
:1003E000B58BA48B8C818F778C83DF91CF910C940C
:1003F000767C80E0DF91CF910895CF93DF93EC017D
:100400000E94CE81882311F01D8281E0DF91CF917F
:100410000895FC01818D928D009711F00C94CE818E
:1004200008953F924F925F926F927F928F929F9228
:10043000AF92BF92CF92DF92EF92FF920F931F93F2
:10044000CF93DF9300D000D000D01F921F92CDB782
:10045000DEB77C01DC0115968C91811115C0FE017F
:100460003196CE010C966F0130E23193E817F9070F
:10047000E1F7DA0130E087E09D91B92E992329F167
:100480009E3239F48A3011F480E0D9C038E08AE035
:10049000F3CFE5EEFDE04491442321F0319694132F
:1004A000FACFF2CF831780F34FED490F4E3560F747
:1004B0004FE9490F4A3118F440EEB42EB90EF60157
:1004C000E30FF11DB0823F5FD7CF89818032E1F227
:1004D000322E8B01FB01838D948DD7015C969C930A
:1004E0008E935B971682178210861186128613866A
:1004F00014861586F80182859385A485B585438980
:1005000054896589768984179507A607B70708F087
:100510004DC025E0B695A795979587952A95D1F773
:10052000F82FFF70AF2ED80115968C91823008F409
:10053000ABCFC8010E94898197FDA6CFF8018285C3
:100540009385A485B5854F96A11DB11D828793879C
:10055000A487B587F0E2AF9EB00111246C5F724FA3
:100560006115710509F490CFDB018C91882341F06E
:10057000853E09F057C0BB2029F0BB24B394BACF05
:10058000B1100EC0F701A28A8091DF029091E002C3
:10059000A091E102B091E20286879787A08BB18B90
:1005A000DB018C918111E9CFBB24B394832D82713F
:1005B000823109F069CFBB2009F459C0C7010E94FC
:1005C000145F009709F460CF20E2FC0111922A9594
:1005D000E9F72BE0F601DC0101900D922A95E1F795
:1005E00021E238E2DC0151963C932E93509740E093
:1005F00058E01F965C934E931E9753963C932E9310
:10060000529759963C932E93589757965C934E93D6
:1006100056970E94767C882309F436CF432DF70144
:1006200062890AC04BE050E0C6010E948DBC892B54
:1006300009F060CF432D6A2DC7010E94887E2B965A
:100640000FB6F894DEBF0FBECDBFDF91CF911F91E3
:100650000F91FF90EF90DF90CF90BF90AF909F9061
:100660008F907F906F905F904F903F900895F8012A
:100670008581823009F408CFC8010E94887F8823D1
:1006800009F402CFD8015B96ED91FC915C97169628
:100690008D909D90AD90BC901997B2E08B1A910807
:1006A000A108B108858504C0880C991CAA1CBB1C34
:1006B0008A95D2F786859785A089B189880E991E7B
:1006C000AA1EBB1E848124013501480E511C611CE9
:1006D000711C84149504A604B70401F1E1E04E1ADC
:1006E0005108610871080E94767C882309F4CCCEF9
:1006F000E4E0FDE0119284E09FE08E179F07D1F7C0
:100700004092DF025092E0026092E1027092E202B7
:100710008091A41781608093A417DBCFD8015B96EA
:10072000ED91FC91258580E092E0A0E0B0E004C06E
:10073000880F991FAA1FBB1F2A95D2F7F80143897A
:10074000548965897689840F951FA61FB71F838BEF
:10075000948BA58BB68BD70152961C9284E09DE0BA
:1007600033CF1F93CF93DF93CDB7DEB76D970FB61F
:10077000F894DEBF0FBECDBFAB011C821B8220E808
:1007800033E03A8329831E8221E0BC01CE01019629
:100790000E94118211E081110CC010E0812F6D9632
:1007A0000FB6F894DEBF0FBECDBFDF91CF911F9182
:1007B0000895CE0101960E94FD81F0CFCF93DF9383
:1007C000CDB7DEB76D970FB6F894DEBF0FBECDBFC5
:1007D000442391F1AB01BC011C821B8280E893E0B1
:1007E0009A8389831E8222E0CE0101960E941182A3
:1007F00081110EC090E081E0911101C080E06D9602
:100800000FB6F894DEBF0FBECDBFDF91CF91089534
:10081000CE0101960E942D5F882361F3CE010196DF
:100820000E94145F009731F325EEFC0120831E82A5
:100830000E94767C982FDFCF81E0E1CF2F923F920C
:100840004F925F926F927F928F929F92AF92BF92E0
:10085000CF92DF92EF92FF920F931F93CF93DF938C
:1008600000D01F92CDB7DEB78C015B011A01DC010D
:1008700015968C911597813009F0C8C014968C910B
:1008800081FFC4C082FDAEC06101D8011A964D91AE
:100890005D916D917C911D97C114D10409F429C11A
:1008A0005B968D919C915C97FC0174802FEF270DD6
:1008B0002A013B0139E076946794579447943A951E
:1008C000D1F7722E74207A01F1E0FF22711020C05E
:1008D000E114F104E9F416964D915D916D917C91CE
:1008E0001997411551056105710509F098C0579692
:1008F0008D919D910D90BC91A02D0097A105B10502
:1009000009F0AFC0C8010E94887F882309F47EC027
:1009100080E092E08E199F0946018C159D0508F430
:100920004C01D8015B964D915C915C9716968D9128
:100930009D910D90BC91A02D0297A109B109FA01DA
:10094000258504C0880F991FAA1FBB1F2A95D2F7BF
:100950004685578560897189840F951FA61FB71F2B
:100960009C01AD01270D311D411D511D29013A0189
:10097000811432E0930609F07AC08091DF029091F1
:10098000E002A091E102B091E20284159505A6056E
:10099000B70559F48FEF9FEFDC018093DF0290934E
:1009A000E002A093E102B093E2029501B301A2013B
:1009B0008091F60C9091F70C0E94097C882331F10C
:1009C0009EEFB91AC818D908F80182859385A485C5
:1009D000B585880D991DA11DB11D82879387A487B8
:1009E000B58753CFF8014389548965897689828513
:1009F0009385A485B585481759076A077B0709F4CD
:100A000043CFC8010E94F47E81113ECF81E090E087
:100A1000D80113969C938E93129780E007C09E0195
:100A20002F5F3F4F0E949C7D811102C090E077C0F4
:100A300089819A81AB81BC81F801238D348DF901C4
:100A4000278948EF5FEF60E070E0203121F048EF48
:100A50005FEF6FEF7FE084179507A607B70708F0F1
:100A600051CFF80186839783A087B18751CFE114D6
:100A7000F10491F5D8011A964D915D916D917C919B
:100A80001D9753968D919D910D90BC91A02D481767
:100A900059076A077B0700F10E94767C882309F4D6
:100AA000B5CF4092DF025092E0026092E102709274
:100AB000E2028091A41781608093A41797012C5FB4
:100AC000324FD501C901880D991DF9018E179F0775
:100AD00059F04D914193FACF41E0C301B2010E9418
:100AE000B17C8111EBCF92CF821B930BA80EB91E64
:100AF00069CFF80183899489A589B68984179507F8
:100B0000A607B70738F48481438B548B658B768BAB
:100B100080688483F801848183FD18C0C1010F902F
:100B20000F900F900F90DF91CF911F910F91FF9039
:100B3000EF90DF90CF90BF90AF909F908F907F907D
:100B40006F905F904F903F902F900895C8010E9442
:100B5000CE81882309F45ACFE1CFCF93DF931F9240
:100B6000CDB7DEB7698341E050E0BE016F5F7F4FD4
:100B70000E941E840F90DF91CF910895CF93DF9351
:100B8000EC01E98DFA8D309749F481E090E09B8388
:100B90008A8390E080E0DF91CF91089513821282E2
:100BA000898D9A8D0E941E84E98DFA8D2281338170
:100BB000232B59F7F0CFFC01DB0112968D919C910C
:100BC00013979383828380E893E0918380831496C4
:100BD0008C911497848315968C911597858316961E
:100BE0004D915D916D917C911997468357836087F4
:100BF00071871A964D915D916D917C911D974287F9
:100C00005387648775871E964D915D916D917C9198
:100C1000519746875787608B718B52968C9152976C
:100C2000828B53964D915D916D917C915697438B3C
:100C3000548B658B768B57964D915D916D917C9120
:100C40005A97478B508F618F728F5B968D919C91D5
:100C5000948F838F0895DC015996ED91FC91309724
:100C600021F081E09581911101C080E00895CF933A
:100C7000DF93EC01898D9A8D009741F00E94FD81F0
:100C8000898D9A8D0E9416BB1A8E198EDF91CF9195
:100C90000895EF92FF920F931F93CF93DF93EC0190
:100CA0007B018A011B821A8288EE93E0A0E0B0E00B
:100CB0008C839D83AE83BF8382E094E09983888395
:100CC0008DE190E00E947ABA9A8F898F009779F02F
:100CD0002DE1F701DC0101900D922A95E1F74CE03E
:100CE00050E0B801CE010C960E94E5BC188EDF9151
:100CF000CF911F910F91FF90EF900895E091F90C23
:100D0000F091FA0C80819091F80C892B80830895E2
:100D1000AF92BF92CF92DF92EF92FF920F931F9309
:100D2000CF93DF9300D01F92CDB7DEB78C016B015C
:100D30007A018091FB0C8333E9F45B016801C40EF6
:100D4000D51EC016D106A9F10E94C3768FE00E947D
:100D5000CE76812F0E94CE76802F0E94CE760F5FB6
:100D60001F4F80E00E94CE76F50181935F010E94C3
:100D70007E86E7CF843369F50E94C37619830A83A0
:100D80008F2D8F778B83EC8264E070E0CE0101962B
:100D90000E94A976A70170E060E0C6010E94B5BC80
:100DA000E114F10421F0B701C6010E94A9760E9466
:100DB0007E86C7010F900F900F900F90DF91CF911B
:100DC0001F910F91FF90EF90DF90CF90BF90AF9069
:100DD00008950E94C3760F3F110509F030F419827F
:100DE0000A831B8263E070E0D1CF17FD0BC019822C
:100DF0000A8333E0169507953A95E1F7007E08607F
:100E00000B83F0CFC80126E0969587952A95E1F7E8
:100E1000807E19830A830115104C18F480618B833E
:100E2000E1CF8861FCCFCF93DF931F92CDB7DEB7C0
:100E30002091FC0C30E0322F2227260F371F90E044
:100E4000982F882741E050E0BE016F5F7F4F820FEF
:100E5000931F0E94888689810F90DF91CF9108951A
:100E6000AF92BF92CF92DF92EF92FF920F931F93B8
:100E7000CF93DF9300D000D01F921F92CDB7DEB783
:100E80008C017B016A018091FB0C8333E1F45801F2
:100E9000A40EB51EA016B10609F46FC00E94C37659
:100EA00080EF0E94CE76812F0E94CE76802F0E9406
:100EB000CE760F5F1F4FF70181917F010E94CE76A2
:100EC0000E947E86E7CF5B01A40EB51E8433C1F479
:100ED0000E94C37619830A838D2D80688B83CC8210
:100EE00064E070E0CE0101960E94A976AE14BF04C2
:100EF00009F441C0F70181917F010E94CE76F6CFBF
:100F00000E94C3760F3F110509F028F419820A8365
:100F100084E08B830CC017FD17C019820A8333E06D
:100F2000169507953A95E1F7007E0C600B8386E0F5
:100F3000C816D104A0F5F701DE011496EA15FB05E9
:100F400099F081918D93FACFC80126E09695879507
:100F50002A95E1F7807E19830A830115104C10F45D
:100F60008461D7CF8C61D5CFB6016D5F7F4FCE0145
:100F700001960E94A9760E947E86C60128960FB629
:100F8000F894DEBF0FBECDBFDF91CF911F910F91BF
:100F9000FF90EF90DF90CF90BF90AF90089563E007
:100FA00070E0CE0101960E94A976F70181917F0140
:100FB0000E94CE76AE14BF04C1F7DDCFCF93DF938E
:100FC0001F92CDB7DEB741E050E0BE016F5F7F4FAB
:100FD00090E080E00E94888689810F90DF91CF9118
:100FE0000895CF93DF93C4E1D0E00E94DE87882389
:100FF00061F061E070E080E090E00E94C0692197BC
:10100000A1F780E0DF91CF91089581E0FBCFCF93EE
:10101000DF931F92CDB7DEB7898341E050E0BE0178
:101020006F5F7F4F90E080E00E9430870F90DF91EC
:10103000CF91089563E070E00C941387DA01E0919A
:10104000FC0CF0E0FE2FEE27E60FF71F90E0982F44
:101050008827A901BD018E0F9F1F0C943087CF9365
:10106000DF931F921F92CDB7DEB779836A8322E0A8
:1010700030E0AE014F5F5F4F60E170E00E941E887C
:101080000F900F90DF91CF910895CF93DF931F9230
:101090001F92CDB7DEB779836A8322E030E0AE01DC
:1010A0004F5F5F4F64E070E00E941E880F900F90CA
:1010B000DF91CF910895CF93DF931F92CDB7DEB725
:1010C0002091FC0C30E0322F2227260F371F90E0B2
:1010D000982F8827498341E050E0BE016F5F7F4F22
:1010E000820F931F0E9430870F90DF91CF91089558
:1010F000CF93C82F462F61E070E00E945B8861E0CB
:1011000070E08C2F0E9413878111F9CFCF91089541
:10111000DA01E091FC0CF0E0FE2FEE27E60FF71F5E
:1011200090E0982F8827A901BD018E0F9F1F0C9476
:1011300088866F927F929F92AF92BF92CF92DF92FA
:10114000EF92FF920F931F93CF93DF931F921F9203
:10115000CDB7DEB7982E8B013A01690122E030E06D
:10116000AE014F5F5F4F64E270E00E948888E980C3
:10117000FA80FE24EF24FE24E00EF11E9701377062
:101180004091FB0C092D10E0C801433309F04CC01D
:101190000896982F8827990F990F990F820F931F00
:1011A000473309F446C0A9014C0D5D1D413058403C
:1011B00008F43FC060E078E05B01A21AB30AA50121
:1011C000B3010E943087A6014A195B09B3016A0D79
:1011D0007B1D8091FB0C833349F5085F1F4F000F87
:1011E000000F000F80E0902F0E943087EC0CFD1C58
:1011F000F982EA8222E030E0AE014F5F5F4F64E2A5
:1012000070E0892D0E941E880F900F90DF91CF9182
:101210001F910F91FF90EF90DF90CF90BF90AF9014
:101220009F907F906F9008954096B3CF005F1F4FBF
:10123000D6CFA601B301D8CFEF92FF921F93CF93E1
:10124000DF931F921F92CDB7DEB7182F22E030E058
:10125000AE014F5F5F4F60E270E00E948888E980D6
:10126000FA80FE24EF24FE2422E030E0AE014F5F3E
:101270005F4F60E270E0812F0E94888889819A81A7
:10128000982789279827E816F90689F487E0189F98
:10129000F0011124E855F34FF582E482C7010F9065
:1012A0000F90DF91CF911F91FF90EF9008957C01F7
:1012B000DBCFFF920F931F93CF93DF931F921F9269
:1012C000CDB7DEB7F82E22E030E0AE014F5F5F4FC2
:1012D00066E270E00E94888809811A811027012740
:1012E000102722E030E0AE014F5F5F4F66E270E012
:1012F0008F2D0E94888889819A819827892798272D
:101300000817190749F4C8010F900F90DF91CF918A
:101310001F910F91FF9008958C01E3CF44E050E0BE
:10132000BC018FE090E00C94308708951F93CF9319
:10133000DF93182F80E591E00E944D5C812F0E9481
:101340001C89EC01812F0E941A88873121F08C3191
:1013500011F0D0E0C0E0CE01DF91CF911F91089550
:10136000FC018485883010F40C94968990E080E02C
:101370000895CF92DF92EF92FF921F93CF93DF9366
:10138000182F7B01EA014130584010F0C0E0D8E04E
:1013900080E591E00E944D5C812F0E941C896C01C8
:1013A000812F0E941A88873111F08C3121F5CC16DB
:1013B000DD0670F380E591E00E944D5C9E01A7017F
:1013C00070E060E0812F0E94998860E270E0812FD8
:1013D0000E94788862E070E0812F0E94138784FD6C
:1013E0000DC0812F0E941A888823B9F080E591E012
:1013F0000E944D5CEFCFD0E0C0E0DCCF40E162E086
:1014000070E0812F0E945B88CE01DF91CF911F9108
:10141000FF90EF90DF90CF900895D0E0C0E0F4CF40
:101420000F931F93CF93DF938C01EA01FC01848516
:10143000883048F40E94B989892B39F481E090E022
:10144000F80193838283D0E0C0E0CE01DF91CF9199
:101450001F910F9108951F93CF93DF931F92CDB7E4
:10146000DEB7182F80E591E00E944D5C812F0E942D
:10147000D57627E0129FF0011124E855F34F228121
:101480003381377041E050E0BE016F5F7F4F820FC4
:10149000931F0E94888689810F90DF91CF911F91C1
:1014A0000895FC01808D883040F4218D328D232BEE
:1014B00021F00E942B8A90E008958FEF9FEF08950E
:1014C000CF93DF93FC012485283028F08FEF9FEF26
:1014D000DF91CF910895EC010190F081E02D00841F
:1014E000F185E02D1995892B89F38C850E942B8A33
:1014F00090E0EECF1F93CF93DF93182F87E0189FD4
:10150000E0011124C855D34F88819981009761F477
:1015100080E591E00E944D5C812F0E9459892E81C7
:10152000821B910999838883DF91CF911F91089540
:10153000FC018485883010F40C947A8A90E080E075
:1015400008954F925F927F928F929F92AF92BF9237
:10155000CF92DF92EF92FF920F931F93CF93DF937F
:101560001F921F92CDB7DEB7782E6B014A01A82ECD
:10157000B12C27E0829FC0011124FC01E855F34FF4
:101580007F010081118180E591E00E944D5C08158A
:10159000190554F4872D0E945989F70126818C0181
:1015A000021B1109118300830115110519F5872DFF
:1015B0000E941A88843159F0882349F001E010E034
:1015C0008C3111F410E000E0119501951109C8016A
:1015D0000F900F90DF91CF911F910F91FF90EF909F
:1015E000DF90CF90BF90AF909F908F907F905F9053
:1015F0004F900895801691060CF4840187E08A9D2F
:10160000F0018B9DF00D1124E855F34FE280F3803B
:10161000C114D10451F12701F7E05F22872D0E9408
:10162000D576840D951D2091FB0C273309F453C00A
:101630009801240D351D2130384008F44CC020E0BD
:1016400038E0490184189508A401B6010E948886F3
:101650002601480C591C6801C818D908872D0E941A
:10166000D576A601B2010E948886E00EF11E87E0C1
:101670008A9DF0018B9DF00D1124E855F34FF38204
:10168000E28220813181201B310B318320838681CE
:10169000800F912F911D8A3F910510F4232BF1F4B7
:1016A00087E08A9DF0018B9DF00D1124E855F34FE2
:1016B0001682F982EA8222E030E0AE014F5F5F4F8E
:1016C00068E270E0872D0E941E8860E470E0872D3C
:1016D0000E9478887CCFA801B601C5CF868377CFDA
:1016E000CF93DF93FC01218D328D2115310529F433
:1016F0008FEF9FEFDF91CF910895EC01808D42171E
:10170000530708F0A9010E94A18A1816190684F748
:10171000298D3A8D281B390B3A8F298FEBCF0F93E8
:101720001F93CF93DF931F92CDB7DEB7FC01218DBE
:10173000328D232B41F48FEF9FEF0F90DF91CF91EC
:101740001F910F9108958C0141E050E0BE016F5F41
:101750007F4FFC01808D0E94A18A181619065CF744
:10176000F801818D928D0197928F818F898190E010
:10177000E4CF0F931F93CF93DF9300D000D01F923D
:101780001F92CDB7DEB78C01D80159964D915C916F
:101790005A974115510551F0ED91FC91048CF58D4E
:1017A000E02D70E060E0C8011995EECFF801808D62
:1017B0000E947A8A892BB1F148E050E0BE016F5F48
:1017C0007F4FD80158968C910E94A18A181619064D
:1017D000F4F4D801509684E0FE01319601900D9208
:1017E0008A95E1F78D8190E0982F88272E81820FCE
:1017F000911DF801958B848B8F81282F30E0322F3B
:1018000022278885820F932F911D928F818F289692
:101810000FB6F894DEBF0FBECDBFDF91CF911F9101
:101820000F91089590E080E0F2CFCF93DF931F9265
:10183000CDB7DEB741E050E0BE016F5F7F4FFC01E6
:1018400084850E94A18A1816190634F4898190E0D3
:101850000F90DF91CF9108958FEF9FEFF9CFFC01AB
:101860008485883010F40C94A18A90E080E008957B
:10187000CF93C82F80E591E00E944D5C68E070E056
:101880008C2FCF910C947888CF93C82F80E591E06E
:101890000E944D5C60E170E08C2FCF910C947888B1
:1018A000CF92DF92EF92FF920F931F93CF93DF932C
:1018B00000D000D0CDB7DEB78C016B017A01FC01FE
:1018C000808D883010F40E94448C80E294E09A83EA
:1018D0008983F60182819381A481B5818B839C8366
:1018E000AD83BE83B701CE0101960E94E861F80185
:1018F000808F8830A0F4F586E486128E118E81E008
:1019000026960FB6F894DEBF0FBECDBFDF91CF9104
:101910001F910F91FF90EF90DF90CF90089580E09E
:10192000EFCFCF93DF93EC01888D883020F40E94B5
:10193000448C88E0888FDF91CF910895CF93C82F92
:1019400080E591E00E944D5C8C2FCF910C941A8819
:10195000EF92FF920F931F93CF93DF937C018091BF
:10196000FB0CD4E0833309F0D8E000EE1CE0C0E0CB
:10197000F801219131918F01F70184819581281718
:10198000390729F0CF5FDC13F3CF80E006C08C2F3E
:101990000E949E8C8431B1F781E0DF91CF911F913D
:1019A0000F91FF90EF9008959F92AF92BF92CF92C8
:1019B000DF92EF92FF920F931F93CF93DF93EC018F
:1019C0007B018091FB0C811121C01B821A8288EE61
:1019D00093E0A0E0B0E08C839D83AE83BF8384ED71
:1019E00093E09983888388E08C8788EE93E09E87D4
:1019F0008D87CE01DF91CF911F910F91FF90EF90D6
:101A0000DF90CF90BF90AF909F90089534E0932ED9
:101A1000833311F028E0922E80EEC82E8CE0D82E71
:101A200010E098E0B92EA12CD6012D913D916D01C9
:101A3000F701848195812817390791F4812F0E943D
:101A40009E8C082F873111F08C3139F5812F0E943F
:101A50007A8A892B59F50C3119F4812F0E94388C20
:101A60001F5F9112E1CFA11008C0D701ED91FC9149
:101A70000084F185E02DC70119951B821A8288EE3A
:101A800093E0A0E0B0E08C839D83AE83BF8384EDC0
:101A900093E099838883BC86A8CF843149F0811173
:101AA000DFCFF601329711821082DACFB12ED8CF74
:101AB000AA24A394D5CF8F929F92AF92BF92CF9238
:101AC000DF92EF92FF920F931F93CF93DF93CDB7E7
:101AD000DEB72F970FB6F894DEBF0FBECDBF5C0107
:101AE0004B017A018091FB0C8823C9F104E0833318
:101AF00009F008E0B501CE0101960E94D48C80EE79
:101B0000C82E8CE0D82E10E0F601219131916F01A2
:101B1000F501848195812817390751F4812F0E949E
:101B20009E8C873129F4A701B401812F0E94B989C5
:101B30001F5F0113E9CFC7012F960FB6F894DEBFE0
:101B40000FBECDBFDF91CF911F910F91FF90EF900E
:101B5000DF90CF90BF90AF909F908F900895F12C21
:101B6000E12CE9CFCF93DF93EC018C858830D0F462
:101B70000E949E8C843189F0882379F0883169F045
:101B800021E08C3159F4E881F9810084F185E02D60
:101B9000CE01199521E0892B09F420E0822FDF91F5
:101BA000CF91089580E0FBCFCF92DF92EF92FF922A
:101BB000CF93DF93EC018C85883068F40E94388CD9
:101BC0000E948F6C6B017C018C850E949E8C811120
:101BD00009C088E08C87DF91CF91FF90EF90DF9074
:101BE000CF90089561E070E080E090E00E94C069CD
:101BF0000E948F6CAB01BC014C195D096E097F0915
:101C00008D859E85B0E0A0E0481759076A077B07DD
